Archive member included to satisfy reference by file (symbol)

d:/programfiles/nxp/mcuxpressoide_11.1.0_3209/ide/plugins/com.nxp.mcuxpresso.tools.win32_11.1.0.201909161352/tools/bin/../lib/gcc/arm-none-eabi/8.3.1/thumb/v7e-m+fp/hard\libgcc.a(_arm_addsubdf3.o)
                              ./open62541/open62541.o (__aeabi_ul2d)
d:/programfiles/nxp/mcuxpressoide_11.1.0_3209/ide/plugins/com.nxp.mcuxpresso.tools.win32_11.1.0.201909161352/tools/bin/../lib/gcc/arm-none-eabi/8.3.1/thumb/v7e-m+fp/hard\libgcc.a(_aeabi_ldivmod.o)
                              ./utilities/fsl_str.o (__aeabi_ldivmod)
d:/programfiles/nxp/mcuxpressoide_11.1.0_3209/ide/plugins/com.nxp.mcuxpresso.tools.win32_11.1.0.201909161352/tools/bin/../lib/gcc/arm-none-eabi/8.3.1/thumb/v7e-m+fp/hard\libgcc.a(_aeabi_uldivmod.o)
                              ./utilities/fsl_str.o (__aeabi_uldivmod)
d:/programfiles/nxp/mcuxpressoide_11.1.0_3209/ide/plugins/com.nxp.mcuxpresso.tools.win32_11.1.0.201909161352/tools/bin/../lib/gcc/arm-none-eabi/8.3.1/thumb/v7e-m+fp/hard\libgcc.a(_fixdfdi.o)
                              ./open62541/open62541.o (__aeabi_d2lz)
d:/programfiles/nxp/mcuxpressoide_11.1.0_3209/ide/plugins/com.nxp.mcuxpresso.tools.win32_11.1.0.201909161352/tools/bin/../lib/gcc/arm-none-eabi/8.3.1/thumb/v7e-m+fp/hard\libgcc.a(_fixunsdfdi.o)
                              ./open62541/open62541.o (__aeabi_d2ulz)
d:/programfiles/nxp/mcuxpressoide_11.1.0_3209/ide/plugins/com.nxp.mcuxpresso.tools.win32_11.1.0.201909161352/tools/bin/../lib/gcc/arm-none-eabi/8.3.1/thumb/v7e-m+fp/hard\libgcc.a(_udivmoddi4.o)
                              d:/programfiles/nxp/mcuxpressoide_11.1.0_3209/ide/plugins/com.nxp.mcuxpresso.tools.win32_11.1.0.201909161352/tools/bin/../lib/gcc/arm-none-eabi/8.3.1/thumb/v7e-m+fp/hard\libgcc.a(_aeabi_ldivmod.o) (__udivmoddi4)
d:/programfiles/nxp/mcuxpressoide_11.1.0_3209/ide/plugins/com.nxp.mcuxpresso.tools.win32_11.1.0.201909161352/tools/bin/../lib/gcc/arm-none-eabi/8.3.1/thumb/v7e-m+fp/hard\libgcc.a(_dvmd_tls.o)
                              d:/programfiles/nxp/mcuxpressoide_11.1.0_3209/ide/plugins/com.nxp.mcuxpresso.tools.win32_11.1.0.201909161352/tools/bin/../lib/gcc/arm-none-eabi/8.3.1/thumb/v7e-m+fp/hard\libgcc.a(_aeabi_ldivmod.o) (__aeabi_ldiv0)
d:/programfiles/nxp/mcuxpressoide_11.1.0_3209/ide/plugins/com.nxp.mcuxpresso.tools.win32_11.1.0.201909161352/tools/bin/../lib/gcc/arm-none-eabi/8.3.1/thumb/v7e-m+fp/hard\libgcc.a(_arm_muldivdf3.o)
                              d:/programfiles/nxp/mcuxpressoide_11.1.0_3209/ide/plugins/com.nxp.mcuxpresso.tools.win32_11.1.0.201909161352/tools/bin/../lib/gcc/arm-none-eabi/8.3.1/thumb/v7e-m+fp/hard\libgcc.a(_fixunsdfdi.o) (__aeabi_dmul)
d:/programfiles/nxp/mcuxpressoide_11.1.0_3209/ide/plugins/com.nxp.mcuxpresso.tools.win32_11.1.0.201909161352/tools/bin/../lib/gcc/arm-none-eabi/8.3.1/thumb/v7e-m+fp/hard\libgcc.a(_arm_cmpdf2.o)
                              d:/programfiles/nxp/mcuxpressoide_11.1.0_3209/ide/plugins/com.nxp.mcuxpresso.tools.win32_11.1.0.201909161352/tools/bin/../lib/gcc/arm-none-eabi/8.3.1/thumb/v7e-m+fp/hard\libgcc.a(_fixdfdi.o) (__aeabi_dcmplt)
d:/programfiles/nxp/mcuxpressoide_11.1.0_3209/ide/plugins/com.nxp.mcuxpresso.tools.win32_11.1.0.201909161352/tools/bin/../lib/gcc/arm-none-eabi/8.3.1/thumb/v7e-m+fp/hard\libgcc.a(_arm_fixunsdfsi.o)
                              d:/programfiles/nxp/mcuxpressoide_11.1.0_3209/ide/plugins/com.nxp.mcuxpresso.tools.win32_11.1.0.201909161352/tools/bin/../lib/gcc/arm-none-eabi/8.3.1/thumb/v7e-m+fp/hard\libgcc.a(_fixunsdfdi.o) (__aeabi_d2uiz)
d:/programfiles/nxp/mcuxpressoide_11.1.0_3209/ide/plugins/com.nxp.mcuxpresso.tools.win32_11.1.0.201909161352/tools/bin/../lib/gcc/arm-none-eabi/8.3.1/../../../../arm-none-eabi/lib/thumb/v7e-m+fp/hard\libc.a(lib_a-atoi.o)
                              ./lwip/src/core/netif.o (atoi)
d:/programfiles/nxp/mcuxpressoide_11.1.0_3209/ide/plugins/com.nxp.mcuxpresso.tools.win32_11.1.0.201909161352/tools/bin/../lib/gcc/arm-none-eabi/8.3.1/../../../../arm-none-eabi/lib/thumb/v7e-m+fp/hard\libc.a(lib_a-ctype_.o)
                              ./lwip/src/core/ipv4/ip4_addr.o (_ctype_)
d:/programfiles/nxp/mcuxpressoide_11.1.0_3209/ide/plugins/com.nxp.mcuxpresso.tools.win32_11.1.0.201909161352/tools/bin/../lib/gcc/arm-none-eabi/8.3.1/../../../../arm-none-eabi/lib/thumb/v7e-m+fp/hard\libc.a(lib_a-fflush.o)
                              ./open62541/open62541.o (fflush)
d:/programfiles/nxp/mcuxpressoide_11.1.0_3209/ide/plugins/com.nxp.mcuxpresso.tools.win32_11.1.0.201909161352/tools/bin/../lib/gcc/arm-none-eabi/8.3.1/../../../../arm-none-eabi/lib/thumb/v7e-m+fp/hard\libc.a(lib_a-findfp.o)
                              d:/programfiles/nxp/mcuxpressoide_11.1.0_3209/ide/plugins/com.nxp.mcuxpresso.tools.win32_11.1.0.201909161352/tools/bin/../lib/gcc/arm-none-eabi/8.3.1/../../../../arm-none-eabi/lib/thumb/v7e-m+fp/hard\libc.a(lib_a-fflush.o) (__sinit)
d:/programfiles/nxp/mcuxpressoide_11.1.0_3209/ide/plugins/com.nxp.mcuxpresso.tools.win32_11.1.0.201909161352/tools/bin/../lib/gcc/arm-none-eabi/8.3.1/../../../../arm-none-eabi/lib/thumb/v7e-m+fp/hard\libc.a(lib_a-freer.o)
                              d:/programfiles/nxp/mcuxpressoide_11.1.0_3209/ide/plugins/com.nxp.mcuxpresso.tools.win32_11.1.0.201909161352/tools/bin/../lib/gcc/arm-none-eabi/8.3.1/../../../../arm-none-eabi/lib/thumb/v7e-m+fp/hard\libc.a(lib_a-fflush.o) (_free_r)
d:/programfiles/nxp/mcuxpressoide_11.1.0_3209/ide/plugins/com.nxp.mcuxpresso.tools.win32_11.1.0.201909161352/tools/bin/../lib/gcc/arm-none-eabi/8.3.1/../../../../arm-none-eabi/lib/thumb/v7e-m+fp/hard\libc.a(lib_a-fwalk.o)
                              d:/programfiles/nxp/mcuxpressoide_11.1.0_3209/ide/plugins/com.nxp.mcuxpresso.tools.win32_11.1.0.201909161352/tools/bin/../lib/gcc/arm-none-eabi/8.3.1/../../../../arm-none-eabi/lib/thumb/v7e-m+fp/hard\libc.a(lib_a-findfp.o) (_fwalk)
d:/programfiles/nxp/mcuxpressoide_11.1.0_3209/ide/plugins/com.nxp.mcuxpresso.tools.win32_11.1.0.201909161352/tools/bin/../lib/gcc/arm-none-eabi/8.3.1/../../../../arm-none-eabi/lib/thumb/v7e-m+fp/hard\libc.a(lib_a-impure.o)
                              d:/programfiles/nxp/mcuxpressoide_11.1.0_3209/ide/plugins/com.nxp.mcuxpresso.tools.win32_11.1.0.201909161352/tools/bin/../lib/gcc/arm-none-eabi/8.3.1/../../../../arm-none-eabi/lib/thumb/v7e-m+fp/hard\libc.a(lib_a-fflush.o) (_global_impure_ptr)
d:/programfiles/nxp/mcuxpressoide_11.1.0_3209/ide/plugins/com.nxp.mcuxpresso.tools.win32_11.1.0.201909161352/tools/bin/../lib/gcc/arm-none-eabi/8.3.1/../../../../arm-none-eabi/lib/thumb/v7e-m+fp/hard\libc.a(lib_a-lock.o)
                              d:/programfiles/nxp/mcuxpressoide_11.1.0_3209/ide/plugins/com.nxp.mcuxpresso.tools.win32_11.1.0.201909161352/tools/bin/../lib/gcc/arm-none-eabi/8.3.1/../../../../arm-none-eabi/lib/thumb/v7e-m+fp/hard\libc.a(lib_a-findfp.o) (__retarget_lock_init_recursive)
d:/programfiles/nxp/mcuxpressoide_11.1.0_3209/ide/plugins/com.nxp.mcuxpresso.tools.win32_11.1.0.201909161352/tools/bin/../lib/gcc/arm-none-eabi/8.3.1/../../../../arm-none-eabi/lib/thumb/v7e-m+fp/hard\libc.a(lib_a-malloc.o)
                              ./source/cpp_config.o (malloc)
d:/programfiles/nxp/mcuxpressoide_11.1.0_3209/ide/plugins/com.nxp.mcuxpresso.tools.win32_11.1.0.201909161352/tools/bin/../lib/gcc/arm-none-eabi/8.3.1/../../../../arm-none-eabi/lib/thumb/v7e-m+fp/hard\libc.a(lib_a-mallocr.o)
                              d:/programfiles/nxp/mcuxpressoide_11.1.0_3209/ide/plugins/com.nxp.mcuxpresso.tools.win32_11.1.0.201909161352/tools/bin/../lib/gcc/arm-none-eabi/8.3.1/../../../../arm-none-eabi/lib/thumb/v7e-m+fp/hard\libc.a(lib_a-findfp.o) (_malloc_r)
d:/programfiles/nxp/mcuxpressoide_11.1.0_3209/ide/plugins/com.nxp.mcuxpresso.tools.win32_11.1.0.201909161352/tools/bin/../lib/gcc/arm-none-eabi/8.3.1/../../../../arm-none-eabi/lib/thumb/v7e-m+fp/hard\libc.a(lib_a-memcmp.o)
                              ./open62541/open62541.o (memcmp)
d:/programfiles/nxp/mcuxpressoide_11.1.0_3209/ide/plugins/com.nxp.mcuxpresso.tools.win32_11.1.0.201909161352/tools/bin/../lib/gcc/arm-none-eabi/8.3.1/../../../../arm-none-eabi/lib/thumb/v7e-m+fp/hard\libc.a(lib_a-memcpy.o)
                              ./source/commands.o (memcpy)
d:/programfiles/nxp/mcuxpressoide_11.1.0_3209/ide/plugins/com.nxp.mcuxpresso.tools.win32_11.1.0.201909161352/tools/bin/../lib/gcc/arm-none-eabi/8.3.1/../../../../arm-none-eabi/lib/thumb/v7e-m+fp/hard\libc.a(lib_a-memmove.o)
                              ./open62541/open62541.o (memmove)
d:/programfiles/nxp/mcuxpressoide_11.1.0_3209/ide/plugins/com.nxp.mcuxpresso.tools.win32_11.1.0.201909161352/tools/bin/../lib/gcc/arm-none-eabi/8.3.1/../../../../arm-none-eabi/lib/thumb/v7e-m+fp/hard\libc.a(lib_a-memset.o)
                              ./source/commands.o (memset)
d:/programfiles/nxp/mcuxpressoide_11.1.0_3209/ide/plugins/com.nxp.mcuxpresso.tools.win32_11.1.0.201909161352/tools/bin/../lib/gcc/arm-none-eabi/8.3.1/../../../../arm-none-eabi/lib/thumb/v7e-m+fp/hard\libc.a(lib_a-mlock.o)
                              d:/programfiles/nxp/mcuxpressoide_11.1.0_3209/ide/plugins/com.nxp.mcuxpresso.tools.win32_11.1.0.201909161352/tools/bin/../lib/gcc/arm-none-eabi/8.3.1/../../../../arm-none-eabi/lib/thumb/v7e-m+fp/hard\libc.a(lib_a-freer.o) (__malloc_lock)
d:/programfiles/nxp/mcuxpressoide_11.1.0_3209/ide/plugins/com.nxp.mcuxpresso.tools.win32_11.1.0.201909161352/tools/bin/../lib/gcc/arm-none-eabi/8.3.1/../../../../arm-none-eabi/lib/thumb/v7e-m+fp/hard\libc.a(lib_a-printf.o)
                              ./utilities/fsl_assert.o (printf)
d:/programfiles/nxp/mcuxpressoide_11.1.0_3209/ide/plugins/com.nxp.mcuxpresso.tools.win32_11.1.0.201909161352/tools/bin/../lib/gcc/arm-none-eabi/8.3.1/../../../../arm-none-eabi/lib/thumb/v7e-m+fp/hard\libc.a(lib_a-sbrkr.o)
                              d:/programfiles/nxp/mcuxpressoide_11.1.0_3209/ide/plugins/com.nxp.mcuxpresso.tools.win32_11.1.0.201909161352/tools/bin/../lib/gcc/arm-none-eabi/8.3.1/../../../../arm-none-eabi/lib/thumb/v7e-m+fp/hard\libc.a(lib_a-freer.o) (_sbrk_r)
d:/programfiles/nxp/mcuxpressoide_11.1.0_3209/ide/plugins/com.nxp.mcuxpresso.tools.win32_11.1.0.201909161352/tools/bin/../lib/gcc/arm-none-eabi/8.3.1/../../../../arm-none-eabi/lib/thumb/v7e-m+fp/hard\libc.a(lib_a-snprintf.o)
                              ./open62541/open62541.o (snprintf)
d:/programfiles/nxp/mcuxpressoide_11.1.0_3209/ide/plugins/com.nxp.mcuxpresso.tools.win32_11.1.0.201909161352/tools/bin/../lib/gcc/arm-none-eabi/8.3.1/../../../../arm-none-eabi/lib/thumb/v7e-m+fp/hard\libc.a(lib_a-sprintf.o)
                              ./source/commands.o (sprintf)
d:/programfiles/nxp/mcuxpressoide_11.1.0_3209/ide/plugins/com.nxp.mcuxpresso.tools.win32_11.1.0.201909161352/tools/bin/../lib/gcc/arm-none-eabi/8.3.1/../../../../arm-none-eabi/lib/thumb/v7e-m+fp/hard\libc.a(lib_a-stdio.o)
                              d:/programfiles/nxp/mcuxpressoide_11.1.0_3209/ide/plugins/com.nxp.mcuxpresso.tools.win32_11.1.0.201909161352/tools/bin/../lib/gcc/arm-none-eabi/8.3.1/../../../../arm-none-eabi/lib/thumb/v7e-m+fp/hard\libc.a(lib_a-findfp.o) (__sread)
d:/programfiles/nxp/mcuxpressoide_11.1.0_3209/ide/plugins/com.nxp.mcuxpresso.tools.win32_11.1.0.201909161352/tools/bin/../lib/gcc/arm-none-eabi/8.3.1/../../../../arm-none-eabi/lib/thumb/v7e-m+fp/hard\libc.a(lib_a-strcmp.o)
                              ./source/commands.o (strcmp)
d:/programfiles/nxp/mcuxpressoide_11.1.0_3209/ide/plugins/com.nxp.mcuxpresso.tools.win32_11.1.0.201909161352/tools/bin/../lib/gcc/arm-none-eabi/8.3.1/../../../../arm-none-eabi/lib/thumb/v7e-m+fp/hard\libc.a(lib_a-strcpy.o)
                              ./amazon-freertos/freertos_kernel/tasks.o (strcpy)
d:/programfiles/nxp/mcuxpressoide_11.1.0_3209/ide/plugins/com.nxp.mcuxpresso.tools.win32_11.1.0.201909161352/tools/bin/../lib/gcc/arm-none-eabi/8.3.1/../../../../arm-none-eabi/lib/thumb/v7e-m+fp/hard\libc.a(lib_a-strerror.o)
                              ./open62541/open62541.o (strerror)
d:/programfiles/nxp/mcuxpressoide_11.1.0_3209/ide/plugins/com.nxp.mcuxpresso.tools.win32_11.1.0.201909161352/tools/bin/../lib/gcc/arm-none-eabi/8.3.1/../../../../arm-none-eabi/lib/thumb/v7e-m+fp/hard\libc.a(lib_a-strlen.o)
                              ./utilities/fsl_str.o (strlen)
d:/programfiles/nxp/mcuxpressoide_11.1.0_3209/ide/plugins/com.nxp.mcuxpresso.tools.win32_11.1.0.201909161352/tools/bin/../lib/gcc/arm-none-eabi/8.3.1/../../../../arm-none-eabi/lib/thumb/v7e-m+fp/hard\libc.a(lib_a-strncmp.o)
                              ./open62541/open62541.o (strncmp)
d:/programfiles/nxp/mcuxpressoide_11.1.0_3209/ide/plugins/com.nxp.mcuxpresso.tools.win32_11.1.0.201909161352/tools/bin/../lib/gcc/arm-none-eabi/8.3.1/../../../../arm-none-eabi/lib/thumb/v7e-m+fp/hard\libc.a(lib_a-strncpy.o)
                              ./lwip/src/api/netdb.o (strncpy)
d:/programfiles/nxp/mcuxpressoide_11.1.0_3209/ide/plugins/com.nxp.mcuxpresso.tools.win32_11.1.0.201909161352/tools/bin/../lib/gcc/arm-none-eabi/8.3.1/../../../../arm-none-eabi/lib/thumb/v7e-m+fp/hard\libc.a(lib_a-strtol.o)
                              d:/programfiles/nxp/mcuxpressoide_11.1.0_3209/ide/plugins/com.nxp.mcuxpresso.tools.win32_11.1.0.201909161352/tools/bin/../lib/gcc/arm-none-eabi/8.3.1/../../../../arm-none-eabi/lib/thumb/v7e-m+fp/hard\libc.a(lib_a-atoi.o) (_strtol_r)
d:/programfiles/nxp/mcuxpressoide_11.1.0_3209/ide/plugins/com.nxp.mcuxpresso.tools.win32_11.1.0.201909161352/tools/bin/../lib/gcc/arm-none-eabi/8.3.1/../../../../arm-none-eabi/lib/thumb/v7e-m+fp/hard\libc.a(lib_a-svfprintf.o)
                              d:/programfiles/nxp/mcuxpressoide_11.1.0_3209/ide/plugins/com.nxp.mcuxpresso.tools.win32_11.1.0.201909161352/tools/bin/../lib/gcc/arm-none-eabi/8.3.1/../../../../arm-none-eabi/lib/thumb/v7e-m+fp/hard\libc.a(lib_a-snprintf.o) (_svfprintf_r)
d:/programfiles/nxp/mcuxpressoide_11.1.0_3209/ide/plugins/com.nxp.mcuxpresso.tools.win32_11.1.0.201909161352/tools/bin/../lib/gcc/arm-none-eabi/8.3.1/../../../../arm-none-eabi/lib/thumb/v7e-m+fp/hard\libc.a(lib_a-u_strerr.o)
                              d:/programfiles/nxp/mcuxpressoide_11.1.0_3209/ide/plugins/com.nxp.mcuxpresso.tools.win32_11.1.0.201909161352/tools/bin/../lib/gcc/arm-none-eabi/8.3.1/../../../../arm-none-eabi/lib/thumb/v7e-m+fp/hard\libc.a(lib_a-strerror.o) (_user_strerror)
d:/programfiles/nxp/mcuxpressoide_11.1.0_3209/ide/plugins/com.nxp.mcuxpresso.tools.win32_11.1.0.201909161352/tools/bin/../lib/gcc/arm-none-eabi/8.3.1/../../../../arm-none-eabi/lib/thumb/v7e-m+fp/hard\libc.a(lib_a-vfprintf.o)
                              d:/programfiles/nxp/mcuxpressoide_11.1.0_3209/ide/plugins/com.nxp.mcuxpresso.tools.win32_11.1.0.201909161352/tools/bin/../lib/gcc/arm-none-eabi/8.3.1/../../../../arm-none-eabi/lib/thumb/v7e-m+fp/hard\libc.a(lib_a-printf.o) (_vfprintf_r)
d:/programfiles/nxp/mcuxpressoide_11.1.0_3209/ide/plugins/com.nxp.mcuxpresso.tools.win32_11.1.0.201909161352/tools/bin/../lib/gcc/arm-none-eabi/8.3.1/../../../../arm-none-eabi/lib/thumb/v7e-m+fp/hard\libc.a(lib_a-vprintf.o)
                              ./open62541/open62541.o (vprintf)
d:/programfiles/nxp/mcuxpressoide_11.1.0_3209/ide/plugins/com.nxp.mcuxpresso.tools.win32_11.1.0.201909161352/tools/bin/../lib/gcc/arm-none-eabi/8.3.1/../../../../arm-none-eabi/lib/thumb/v7e-m+fp/hard\libc.a(lib_a-vsnprintf.o)
                              ./source/node.o (vsnprintf)
d:/programfiles/nxp/mcuxpressoide_11.1.0_3209/ide/plugins/com.nxp.mcuxpresso.tools.win32_11.1.0.201909161352/tools/bin/../lib/gcc/arm-none-eabi/8.3.1/../../../../arm-none-eabi/lib/thumb/v7e-m+fp/hard\libc.a(lib_a-writer.o)
                              d:/programfiles/nxp/mcuxpressoide_11.1.0_3209/ide/plugins/com.nxp.mcuxpresso.tools.win32_11.1.0.201909161352/tools/bin/../lib/gcc/arm-none-eabi/8.3.1/../../../../arm-none-eabi/lib/thumb/v7e-m+fp/hard\libc.a(lib_a-stdio.o) (_write_r)
d:/programfiles/nxp/mcuxpressoide_11.1.0_3209/ide/plugins/com.nxp.mcuxpresso.tools.win32_11.1.0.201909161352/tools/bin/../lib/gcc/arm-none-eabi/8.3.1/../../../../arm-none-eabi/lib/thumb/v7e-m+fp/hard\libc.a(lib_a-wsetup.o)
                              d:/programfiles/nxp/mcuxpressoide_11.1.0_3209/ide/plugins/com.nxp.mcuxpresso.tools.win32_11.1.0.201909161352/tools/bin/../lib/gcc/arm-none-eabi/8.3.1/../../../../arm-none-eabi/lib/thumb/v7e-m+fp/hard\libc.a(lib_a-vfprintf.o) (__swsetup_r)
d:/programfiles/nxp/mcuxpressoide_11.1.0_3209/ide/plugins/com.nxp.mcuxpresso.tools.win32_11.1.0.201909161352/tools/bin/../lib/gcc/arm-none-eabi/8.3.1/../../../../arm-none-eabi/lib/thumb/v7e-m+fp/hard\libc.a(lib_a-closer.o)
                              d:/programfiles/nxp/mcuxpressoide_11.1.0_3209/ide/plugins/com.nxp.mcuxpresso.tools.win32_11.1.0.201909161352/tools/bin/../lib/gcc/arm-none-eabi/8.3.1/../../../../arm-none-eabi/lib/thumb/v7e-m+fp/hard\libc.a(lib_a-stdio.o) (_close_r)
d:/programfiles/nxp/mcuxpressoide_11.1.0_3209/ide/plugins/com.nxp.mcuxpresso.tools.win32_11.1.0.201909161352/tools/bin/../lib/gcc/arm-none-eabi/8.3.1/../../../../arm-none-eabi/lib/thumb/v7e-m+fp/hard\libc.a(lib_a-dtoa.o)
                              d:/programfiles/nxp/mcuxpressoide_11.1.0_3209/ide/plugins/com.nxp.mcuxpresso.tools.win32_11.1.0.201909161352/tools/bin/../lib/gcc/arm-none-eabi/8.3.1/../../../../arm-none-eabi/lib/thumb/v7e-m+fp/hard\libc.a(lib_a-svfprintf.o) (_dtoa_r)
d:/programfiles/nxp/mcuxpressoide_11.1.0_3209/ide/plugins/com.nxp.mcuxpresso.tools.win32_11.1.0.201909161352/tools/bin/../lib/gcc/arm-none-eabi/8.3.1/../../../../arm-none-eabi/lib/thumb/v7e-m+fp/hard\libc.a(lib_a-fclose.o)
                              d:/programfiles/nxp/mcuxpressoide_11.1.0_3209/ide/plugins/com.nxp.mcuxpresso.tools.win32_11.1.0.201909161352/tools/bin/../lib/gcc/arm-none-eabi/8.3.1/../../../../arm-none-eabi/lib/thumb/v7e-m+fp/hard\libc.a(lib_a-findfp.o) (_fclose_r)
d:/programfiles/nxp/mcuxpressoide_11.1.0_3209/ide/plugins/com.nxp.mcuxpresso.tools.win32_11.1.0.201909161352/tools/bin/../lib/gcc/arm-none-eabi/8.3.1/../../../../arm-none-eabi/lib/thumb/v7e-m+fp/hard\libc.a(lib_a-localeconv.o)
                              d:/programfiles/nxp/mcuxpressoide_11.1.0_3209/ide/plugins/com.nxp.mcuxpresso.tools.win32_11.1.0.201909161352/tools/bin/../lib/gcc/arm-none-eabi/8.3.1/../../../../arm-none-eabi/lib/thumb/v7e-m+fp/hard\libc.a(lib_a-svfprintf.o) (_localeconv_r)
d:/programfiles/nxp/mcuxpressoide_11.1.0_3209/ide/plugins/com.nxp.mcuxpresso.tools.win32_11.1.0.201909161352/tools/bin/../lib/gcc/arm-none-eabi/8.3.1/../../../../arm-none-eabi/lib/thumb/v7e-m+fp/hard\libc.a(lib_a-lseekr.o)
                              d:/programfiles/nxp/mcuxpressoide_11.1.0_3209/ide/plugins/com.nxp.mcuxpresso.tools.win32_11.1.0.201909161352/tools/bin/../lib/gcc/arm-none-eabi/8.3.1/../../../../arm-none-eabi/lib/thumb/v7e-m+fp/hard\libc.a(lib_a-stdio.o) (_lseek_r)
d:/programfiles/nxp/mcuxpressoide_11.1.0_3209/ide/plugins/com.nxp.mcuxpresso.tools.win32_11.1.0.201909161352/tools/bin/../lib/gcc/arm-none-eabi/8.3.1/../../../../arm-none-eabi/lib/thumb/v7e-m+fp/hard\libc.a(lib_a-makebuf.o)
                              d:/programfiles/nxp/mcuxpressoide_11.1.0_3209/ide/plugins/com.nxp.mcuxpresso.tools.win32_11.1.0.201909161352/tools/bin/../lib/gcc/arm-none-eabi/8.3.1/../../../../arm-none-eabi/lib/thumb/v7e-m+fp/hard\libc.a(lib_a-wsetup.o) (__smakebuf_r)
d:/programfiles/nxp/mcuxpressoide_11.1.0_3209/ide/plugins/com.nxp.mcuxpresso.tools.win32_11.1.0.201909161352/tools/bin/../lib/gcc/arm-none-eabi/8.3.1/../../../../arm-none-eabi/lib/thumb/v7e-m+fp/hard\libc.a(lib_a-memchr.o)
                              d:/programfiles/nxp/mcuxpressoide_11.1.0_3209/ide/plugins/com.nxp.mcuxpresso.tools.win32_11.1.0.201909161352/tools/bin/../lib/gcc/arm-none-eabi/8.3.1/../../../../arm-none-eabi/lib/thumb/v7e-m+fp/hard\libc.a(lib_a-svfprintf.o) (memchr)
d:/programfiles/nxp/mcuxpressoide_11.1.0_3209/ide/plugins/com.nxp.mcuxpresso.tools.win32_11.1.0.201909161352/tools/bin/../lib/gcc/arm-none-eabi/8.3.1/../../../../arm-none-eabi/lib/thumb/v7e-m+fp/hard\libc.a(lib_a-mprec.o)
                              d:/programfiles/nxp/mcuxpressoide_11.1.0_3209/ide/plugins/com.nxp.mcuxpresso.tools.win32_11.1.0.201909161352/tools/bin/../lib/gcc/arm-none-eabi/8.3.1/../../../../arm-none-eabi/lib/thumb/v7e-m+fp/hard\libc.a(lib_a-dtoa.o) (_Balloc)
d:/programfiles/nxp/mcuxpressoide_11.1.0_3209/ide/plugins/com.nxp.mcuxpresso.tools.win32_11.1.0.201909161352/tools/bin/../lib/gcc/arm-none-eabi/8.3.1/../../../../arm-none-eabi/lib/thumb/v7e-m+fp/hard\libc.a(lib_a-readr.o)
                              d:/programfiles/nxp/mcuxpressoide_11.1.0_3209/ide/plugins/com.nxp.mcuxpresso.tools.win32_11.1.0.201909161352/tools/bin/../lib/gcc/arm-none-eabi/8.3.1/../../../../arm-none-eabi/lib/thumb/v7e-m+fp/hard\libc.a(lib_a-stdio.o) (_read_r)
d:/programfiles/nxp/mcuxpressoide_11.1.0_3209/ide/plugins/com.nxp.mcuxpresso.tools.win32_11.1.0.201909161352/tools/bin/../lib/gcc/arm-none-eabi/8.3.1/../../../../arm-none-eabi/lib/thumb/v7e-m+fp/hard\libc.a(lib_a-s_frexp.o)
                              d:/programfiles/nxp/mcuxpressoide_11.1.0_3209/ide/plugins/com.nxp.mcuxpresso.tools.win32_11.1.0.201909161352/tools/bin/../lib/gcc/arm-none-eabi/8.3.1/../../../../arm-none-eabi/lib/thumb/v7e-m+fp/hard\libc.a(lib_a-svfprintf.o) (frexp)
d:/programfiles/nxp/mcuxpressoide_11.1.0_3209/ide/plugins/com.nxp.mcuxpresso.tools.win32_11.1.0.201909161352/tools/bin/../lib/gcc/arm-none-eabi/8.3.1/../../../../arm-none-eabi/lib/thumb/v7e-m+fp/hard\libc.a(lib_a-svfiprintf.o)
                              d:/programfiles/nxp/mcuxpressoide_11.1.0_3209/ide/plugins/com.nxp.mcuxpresso.tools.win32_11.1.0.201909161352/tools/bin/../lib/gcc/arm-none-eabi/8.3.1/../../../../arm-none-eabi/lib/thumb/v7e-m+fp/hard\libc.a(lib_a-svfprintf.o) (__ssprint_r)
d:/programfiles/nxp/mcuxpressoide_11.1.0_3209/ide/plugins/com.nxp.mcuxpresso.tools.win32_11.1.0.201909161352/tools/bin/../lib/gcc/arm-none-eabi/8.3.1/../../../../arm-none-eabi/lib/thumb/v7e-m+fp/hard\libc.a(lib_a-vfiprintf.o)
                              d:/programfiles/nxp/mcuxpressoide_11.1.0_3209/ide/plugins/com.nxp.mcuxpresso.tools.win32_11.1.0.201909161352/tools/bin/../lib/gcc/arm-none-eabi/8.3.1/../../../../arm-none-eabi/lib/thumb/v7e-m+fp/hard\libc.a(lib_a-vfprintf.o) (__sprint_r)
d:/programfiles/nxp/mcuxpressoide_11.1.0_3209/ide/plugins/com.nxp.mcuxpresso.tools.win32_11.1.0.201909161352/tools/bin/../lib/gcc/arm-none-eabi/8.3.1/../../../../arm-none-eabi/lib/thumb/v7e-m+fp/hard\libc.a(lib_a-callocr.o)
                              d:/programfiles/nxp/mcuxpressoide_11.1.0_3209/ide/plugins/com.nxp.mcuxpresso.tools.win32_11.1.0.201909161352/tools/bin/../lib/gcc/arm-none-eabi/8.3.1/../../../../arm-none-eabi/lib/thumb/v7e-m+fp/hard\libc.a(lib_a-mprec.o) (_calloc_r)
d:/programfiles/nxp/mcuxpressoide_11.1.0_3209/ide/plugins/com.nxp.mcuxpresso.tools.win32_11.1.0.201909161352/tools/bin/../lib/gcc/arm-none-eabi/8.3.1/../../../../arm-none-eabi/lib/thumb/v7e-m+fp/hard\libc.a(lib_a-fputwc.o)
                              d:/programfiles/nxp/mcuxpressoide_11.1.0_3209/ide/plugins/com.nxp.mcuxpresso.tools.win32_11.1.0.201909161352/tools/bin/../lib/gcc/arm-none-eabi/8.3.1/../../../../arm-none-eabi/lib/thumb/v7e-m+fp/hard\libc.a(lib_a-vfiprintf.o) (_fputwc_r)
d:/programfiles/nxp/mcuxpressoide_11.1.0_3209/ide/plugins/com.nxp.mcuxpresso.tools.win32_11.1.0.201909161352/tools/bin/../lib/gcc/arm-none-eabi/8.3.1/../../../../arm-none-eabi/lib/thumb/v7e-m+fp/hard\libc.a(lib_a-fstatr.o)
                              d:/programfiles/nxp/mcuxpressoide_11.1.0_3209/ide/plugins/com.nxp.mcuxpresso.tools.win32_11.1.0.201909161352/tools/bin/../lib/gcc/arm-none-eabi/8.3.1/../../../../arm-none-eabi/lib/thumb/v7e-m+fp/hard\libc.a(lib_a-makebuf.o) (_fstat_r)
d:/programfiles/nxp/mcuxpressoide_11.1.0_3209/ide/plugins/com.nxp.mcuxpresso.tools.win32_11.1.0.201909161352/tools/bin/../lib/gcc/arm-none-eabi/8.3.1/../../../../arm-none-eabi/lib/thumb/v7e-m+fp/hard\libc.a(lib_a-fvwrite.o)
                              d:/programfiles/nxp/mcuxpressoide_11.1.0_3209/ide/plugins/com.nxp.mcuxpresso.tools.win32_11.1.0.201909161352/tools/bin/../lib/gcc/arm-none-eabi/8.3.1/../../../../arm-none-eabi/lib/thumb/v7e-m+fp/hard\libc.a(lib_a-vfiprintf.o) (__sfvwrite_r)
d:/programfiles/nxp/mcuxpressoide_11.1.0_3209/ide/plugins/com.nxp.mcuxpresso.tools.win32_11.1.0.201909161352/tools/bin/../lib/gcc/arm-none-eabi/8.3.1/../../../../arm-none-eabi/lib/thumb/v7e-m+fp/hard\libc.a(lib_a-isattyr.o)
                              d:/programfiles/nxp/mcuxpressoide_11.1.0_3209/ide/plugins/com.nxp.mcuxpresso.tools.win32_11.1.0.201909161352/tools/bin/../lib/gcc/arm-none-eabi/8.3.1/../../../../arm-none-eabi/lib/thumb/v7e-m+fp/hard\libc.a(lib_a-makebuf.o) (_isatty_r)
d:/programfiles/nxp/mcuxpressoide_11.1.0_3209/ide/plugins/com.nxp.mcuxpresso.tools.win32_11.1.0.201909161352/tools/bin/../lib/gcc/arm-none-eabi/8.3.1/../../../../arm-none-eabi/lib/thumb/v7e-m+fp/hard\libc.a(lib_a-locale.o)
                              d:/programfiles/nxp/mcuxpressoide_11.1.0_3209/ide/plugins/com.nxp.mcuxpresso.tools.win32_11.1.0.201909161352/tools/bin/../lib/gcc/arm-none-eabi/8.3.1/../../../../arm-none-eabi/lib/thumb/v7e-m+fp/hard\libc.a(lib_a-fputwc.o) (__locale_mb_cur_max)
d:/programfiles/nxp/mcuxpressoide_11.1.0_3209/ide/plugins/com.nxp.mcuxpresso.tools.win32_11.1.0.201909161352/tools/bin/../lib/gcc/arm-none-eabi/8.3.1/../../../../arm-none-eabi/lib/thumb/v7e-m+fp/hard\libc.a(lib_a-mbtowc_r.o)
                              d:/programfiles/nxp/mcuxpressoide_11.1.0_3209/ide/plugins/com.nxp.mcuxpresso.tools.win32_11.1.0.201909161352/tools/bin/../lib/gcc/arm-none-eabi/8.3.1/../../../../arm-none-eabi/lib/thumb/v7e-m+fp/hard\libc.a(lib_a-locale.o) (__ascii_mbtowc)
d:/programfiles/nxp/mcuxpressoide_11.1.0_3209/ide/plugins/com.nxp.mcuxpresso.tools.win32_11.1.0.201909161352/tools/bin/../lib/gcc/arm-none-eabi/8.3.1/../../../../arm-none-eabi/lib/thumb/v7e-m+fp/hard\libc.a(lib_a-reallocr.o)
                              d:/programfiles/nxp/mcuxpressoide_11.1.0_3209/ide/plugins/com.nxp.mcuxpresso.tools.win32_11.1.0.201909161352/tools/bin/../lib/gcc/arm-none-eabi/8.3.1/../../../../arm-none-eabi/lib/thumb/v7e-m+fp/hard\libc.a(lib_a-svfiprintf.o) (_realloc_r)
d:/programfiles/nxp/mcuxpressoide_11.1.0_3209/ide/plugins/com.nxp.mcuxpresso.tools.win32_11.1.0.201909161352/tools/bin/../lib/gcc/arm-none-eabi/8.3.1/../../../../arm-none-eabi/lib/thumb/v7e-m+fp/hard\libc.a(lib_a-wbuf.o)
                              d:/programfiles/nxp/mcuxpressoide_11.1.0_3209/ide/plugins/com.nxp.mcuxpresso.tools.win32_11.1.0.201909161352/tools/bin/../lib/gcc/arm-none-eabi/8.3.1/../../../../arm-none-eabi/lib/thumb/v7e-m+fp/hard\libc.a(lib_a-fputwc.o) (__swbuf_r)
d:/programfiles/nxp/mcuxpressoide_11.1.0_3209/ide/plugins/com.nxp.mcuxpresso.tools.win32_11.1.0.201909161352/tools/bin/../lib/gcc/arm-none-eabi/8.3.1/../../../../arm-none-eabi/lib/thumb/v7e-m+fp/hard\libc.a(lib_a-wcrtomb.o)
                              d:/programfiles/nxp/mcuxpressoide_11.1.0_3209/ide/plugins/com.nxp.mcuxpresso.tools.win32_11.1.0.201909161352/tools/bin/../lib/gcc/arm-none-eabi/8.3.1/../../../../arm-none-eabi/lib/thumb/v7e-m+fp/hard\libc.a(lib_a-fputwc.o) (_wcrtomb_r)
d:/programfiles/nxp/mcuxpressoide_11.1.0_3209/ide/plugins/com.nxp.mcuxpresso.tools.win32_11.1.0.201909161352/tools/bin/../lib/gcc/arm-none-eabi/8.3.1/../../../../arm-none-eabi/lib/thumb/v7e-m+fp/hard\libc.a(lib_a-wctomb_r.o)
                              d:/programfiles/nxp/mcuxpressoide_11.1.0_3209/ide/plugins/com.nxp.mcuxpresso.tools.win32_11.1.0.201909161352/tools/bin/../lib/gcc/arm-none-eabi/8.3.1/../../../../arm-none-eabi/lib/thumb/v7e-m+fp/hard\libc.a(lib_a-locale.o) (__ascii_wctomb)
d:/programfiles/nxp/mcuxpressoide_11.1.0_3209/ide/plugins/com.nxp.mcuxpresso.tools.win32_11.1.0.201909161352/tools/bin/../lib/gcc/arm-none-eabi/8.3.1/../../../../arm-none-eabi/lib/thumb/v7e-m+fp/hard\libstdc++.a(guard.o)
                              ./source/main_MandC.o (__cxa_guard_acquire)
d:/programfiles/nxp/mcuxpressoide_11.1.0_3209/ide/plugins/com.nxp.mcuxpresso.tools.win32_11.1.0.201909161352/tools/bin/../lib/gcc/arm-none-eabi/8.3.1/../../../../arm-none-eabi/lib/thumb/v7e-m+fp/hard\libstdc++.a(eh_alloc.o)
                              d:/programfiles/nxp/mcuxpressoide_11.1.0_3209/ide/plugins/com.nxp.mcuxpresso.tools.win32_11.1.0.201909161352/tools/bin/../lib/gcc/arm-none-eabi/8.3.1/../../../../arm-none-eabi/lib/thumb/v7e-m+fp/hard\libstdc++.a(guard.o) (__cxa_allocate_exception)
d:/programfiles/nxp/mcuxpressoide_11.1.0_3209/ide/plugins/com.nxp.mcuxpresso.tools.win32_11.1.0.201909161352/tools/bin/../lib/gcc/arm-none-eabi/8.3.1/../../../../arm-none-eabi/lib/thumb/v7e-m+fp/hard\libstdc++.a(eh_terminate.o)
                              d:/programfiles/nxp/mcuxpressoide_11.1.0_3209/ide/plugins/com.nxp.mcuxpresso.tools.win32_11.1.0.201909161352/tools/bin/../lib/gcc/arm-none-eabi/8.3.1/../../../../arm-none-eabi/lib/thumb/v7e-m+fp/hard\libstdc++.a(eh_alloc.o) (std::terminate())
d:/programfiles/nxp/mcuxpressoide_11.1.0_3209/ide/plugins/com.nxp.mcuxpresso.tools.win32_11.1.0.201909161352/tools/bin/../lib/gcc/arm-none-eabi/8.3.1/../../../../arm-none-eabi/lib/thumb/v7e-m+fp/hard\libstdc++.a(eh_arm.o)
                              d:/programfiles/nxp/mcuxpressoide_11.1.0_3209/ide/plugins/com.nxp.mcuxpresso.tools.win32_11.1.0.201909161352/tools/bin/../lib/gcc/arm-none-eabi/8.3.1/../../../../arm-none-eabi/lib/thumb/v7e-m+fp/hard\libstdc++.a(eh_terminate.o) (__cxa_end_cleanup)
d:/programfiles/nxp/mcuxpressoide_11.1.0_3209/ide/plugins/com.nxp.mcuxpresso.tools.win32_11.1.0.201909161352/tools/bin/../lib/gcc/arm-none-eabi/8.3.1/../../../../arm-none-eabi/lib/thumb/v7e-m+fp/hard\libstdc++.a(eh_throw.o)
                              d:/programfiles/nxp/mcuxpressoide_11.1.0_3209/ide/plugins/com.nxp.mcuxpresso.tools.win32_11.1.0.201909161352/tools/bin/../lib/gcc/arm-none-eabi/8.3.1/../../../../arm-none-eabi/lib/thumb/v7e-m+fp/hard\libstdc++.a(guard.o) (__cxa_throw)
d:/programfiles/nxp/mcuxpressoide_11.1.0_3209/ide/plugins/com.nxp.mcuxpresso.tools.win32_11.1.0.201909161352/tools/bin/../lib/gcc/arm-none-eabi/8.3.1/../../../../arm-none-eabi/lib/thumb/v7e-m+fp/hard\libstdc++.a(allocator-inst.o)
                              ./source/Devices.o (std::allocator<char>::allocator())
d:/programfiles/nxp/mcuxpressoide_11.1.0_3209/ide/plugins/com.nxp.mcuxpresso.tools.win32_11.1.0.201909161352/tools/bin/../lib/gcc/arm-none-eabi/8.3.1/../../../../arm-none-eabi/lib/thumb/v7e-m+fp/hard\libstdc++.a(string-inst.o)
                              ./source/node.o (std::__cxx11::basic_string<char, std::char_traits<char>, std::allocator<char> >::_M_data(char*))
d:/programfiles/nxp/mcuxpressoide_11.1.0_3209/ide/plugins/com.nxp.mcuxpresso.tools.win32_11.1.0.201909161352/tools/bin/../lib/gcc/arm-none-eabi/8.3.1/../../../../arm-none-eabi/lib/thumb/v7e-m+fp/hard\libstdc++.a(functexcept.o)
                              ./source/node.o (std::__throw_logic_error(char const*))
d:/programfiles/nxp/mcuxpressoide_11.1.0_3209/ide/plugins/com.nxp.mcuxpresso.tools.win32_11.1.0.201909161352/tools/bin/../lib/gcc/arm-none-eabi/8.3.1/../../../../arm-none-eabi/lib/thumb/v7e-m+fp/hard\libstdc++.a(guard_error.o)
                              d:/programfiles/nxp/mcuxpressoide_11.1.0_3209/ide/plugins/com.nxp.mcuxpresso.tools.win32_11.1.0.201909161352/tools/bin/../lib/gcc/arm-none-eabi/8.3.1/../../../../arm-none-eabi/lib/thumb/v7e-m+fp/hard\libstdc++.a(guard.o) (__gnu_cxx::recursive_init_error::~recursive_init_error())
d:/programfiles/nxp/mcuxpressoide_11.1.0_3209/ide/plugins/com.nxp.mcuxpresso.tools.win32_11.1.0.201909161352/tools/bin/../lib/gcc/arm-none-eabi/8.3.1/../../../../arm-none-eabi/lib/thumb/v7e-m+fp/hard\libstdc++.a(eh_exception.o)
                              d:/programfiles/nxp/mcuxpressoide_11.1.0_3209/ide/plugins/com.nxp.mcuxpresso.tools.win32_11.1.0.201909161352/tools/bin/../lib/gcc/arm-none-eabi/8.3.1/../../../../arm-none-eabi/lib/thumb/v7e-m+fp/hard\libstdc++.a(guard_error.o) (std::exception::~exception())
d:/programfiles/nxp/mcuxpressoide_11.1.0_3209/ide/plugins/com.nxp.mcuxpresso.tools.win32_11.1.0.201909161352/tools/bin/../lib/gcc/arm-none-eabi/8.3.1/../../../../arm-none-eabi/lib/thumb/v7e-m+fp/hard\libstdc++.a(eh_personality.o)
                              d:/programfiles/nxp/mcuxpressoide_11.1.0_3209/ide/plugins/com.nxp.mcuxpresso.tools.win32_11.1.0.201909161352/tools/bin/../lib/gcc/arm-none-eabi/8.3.1/../../../../arm-none-eabi/lib/thumb/v7e-m+fp/hard\libstdc++.a(eh_terminate.o) (__gxx_personality_v0)
d:/programfiles/nxp/mcuxpressoide_11.1.0_3209/ide/plugins/com.nxp.mcuxpresso.tools.win32_11.1.0.201909161352/tools/bin/../lib/gcc/arm-none-eabi/8.3.1/../../../../arm-none-eabi/lib/thumb/v7e-m+fp/hard\libstdc++.a(eh_term_handler.o)
                              d:/programfiles/nxp/mcuxpressoide_11.1.0_3209/ide/plugins/com.nxp.mcuxpresso.tools.win32_11.1.0.201909161352/tools/bin/../lib/gcc/arm-none-eabi/8.3.1/../../../../arm-none-eabi/lib/thumb/v7e-m+fp/hard\libstdc++.a(eh_terminate.o) (__cxxabiv1::__terminate_handler)
d:/programfiles/nxp/mcuxpressoide_11.1.0_3209/ide/plugins/com.nxp.mcuxpresso.tools.win32_11.1.0.201909161352/tools/bin/../lib/gcc/arm-none-eabi/8.3.1/../../../../arm-none-eabi/lib/thumb/v7e-m+fp/hard\libstdc++.a(bad_cast.o)
                              d:/programfiles/nxp/mcuxpressoide_11.1.0_3209/ide/plugins/com.nxp.mcuxpresso.tools.win32_11.1.0.201909161352/tools/bin/../lib/gcc/arm-none-eabi/8.3.1/../../../../arm-none-eabi/lib/thumb/v7e-m+fp/hard\libstdc++.a(functexcept.o) (std::bad_cast::~bad_cast())
d:/programfiles/nxp/mcuxpressoide_11.1.0_3209/ide/plugins/com.nxp.mcuxpresso.tools.win32_11.1.0.201909161352/tools/bin/../lib/gcc/arm-none-eabi/8.3.1/../../../../arm-none-eabi/lib/thumb/v7e-m+fp/hard\libstdc++.a(bad_alloc.o)
                              d:/programfiles/nxp/mcuxpressoide_11.1.0_3209/ide/plugins/com.nxp.mcuxpresso.tools.win32_11.1.0.201909161352/tools/bin/../lib/gcc/arm-none-eabi/8.3.1/../../../../arm-none-eabi/lib/thumb/v7e-m+fp/hard\libstdc++.a(functexcept.o) (std::bad_alloc::~bad_alloc())
d:/programfiles/nxp/mcuxpressoide_11.1.0_3209/ide/plugins/com.nxp.mcuxpresso.tools.win32_11.1.0.201909161352/tools/bin/../lib/gcc/arm-none-eabi/8.3.1/../../../../arm-none-eabi/lib/thumb/v7e-m+fp/hard\libstdc++.a(eh_call.o)
                              d:/programfiles/nxp/mcuxpressoide_11.1.0_3209/ide/plugins/com.nxp.mcuxpresso.tools.win32_11.1.0.201909161352/tools/bin/../lib/gcc/arm-none-eabi/8.3.1/../../../../arm-none-eabi/lib/thumb/v7e-m+fp/hard\libstdc++.a(eh_personality.o) (__cxa_call_terminate)
d:/programfiles/nxp/mcuxpressoide_11.1.0_3209/ide/plugins/com.nxp.mcuxpresso.tools.win32_11.1.0.201909161352/tools/bin/../lib/gcc/arm-none-eabi/8.3.1/../../../../arm-none-eabi/lib/thumb/v7e-m+fp/hard\libstdc++.a(pure.o)
                              d:/programfiles/nxp/mcuxpressoide_11.1.0_3209/ide/plugins/com.nxp.mcuxpresso.tools.win32_11.1.0.201909161352/tools/bin/../lib/gcc/arm-none-eabi/8.3.1/../../../../arm-none-eabi/lib/thumb/v7e-m+fp/hard\libstdc++.a(eh_exception.o) (__cxa_pure_virtual)
d:/programfiles/nxp/mcuxpressoide_11.1.0_3209/ide/plugins/com.nxp.mcuxpresso.tools.win32_11.1.0.201909161352/tools/bin/../lib/gcc/arm-none-eabi/8.3.1/../../../../arm-none-eabi/lib/thumb/v7e-m+fp/hard\libstdc++.a(eh_catch.o)
                              d:/programfiles/nxp/mcuxpressoide_11.1.0_3209/ide/plugins/com.nxp.mcuxpresso.tools.win32_11.1.0.201909161352/tools/bin/../lib/gcc/arm-none-eabi/8.3.1/../../../../arm-none-eabi/lib/thumb/v7e-m+fp/hard\libstdc++.a(eh_terminate.o) (__cxa_begin_catch)
d:/programfiles/nxp/mcuxpressoide_11.1.0_3209/ide/plugins/com.nxp.mcuxpresso.tools.win32_11.1.0.201909161352/tools/bin/../lib/gcc/arm-none-eabi/8.3.1/../../../../arm-none-eabi/lib/thumb/v7e-m+fp/hard\libstdc++.a(eh_unex_handler.o)
                              d:/programfiles/nxp/mcuxpressoide_11.1.0_3209/ide/plugins/com.nxp.mcuxpresso.tools.win32_11.1.0.201909161352/tools/bin/../lib/gcc/arm-none-eabi/8.3.1/../../../../arm-none-eabi/lib/thumb/v7e-m+fp/hard\libstdc++.a(eh_terminate.o) (__cxxabiv1::__unexpected_handler)
d:/programfiles/nxp/mcuxpressoide_11.1.0_3209/ide/plugins/com.nxp.mcuxpresso.tools.win32_11.1.0.201909161352/tools/bin/../lib/gcc/arm-none-eabi/8.3.1/../../../../arm-none-eabi/lib/thumb/v7e-m+fp/hard\libstdc++.a(eh_globals.o)
                              d:/programfiles/nxp/mcuxpressoide_11.1.0_3209/ide/plugins/com.nxp.mcuxpresso.tools.win32_11.1.0.201909161352/tools/bin/../lib/gcc/arm-none-eabi/8.3.1/../../../../arm-none-eabi/lib/thumb/v7e-m+fp/hard\libstdc++.a(eh_call.o) (__cxa_get_globals_fast)
d:/programfiles/nxp/mcuxpressoide_11.1.0_3209/ide/plugins/com.nxp.mcuxpresso.tools.win32_11.1.0.201909161352/tools/bin/../lib/gcc/arm-none-eabi/8.3.1/../../../../arm-none-eabi/lib/thumb/v7e-m+fp/hard\libstdc++.a(del_ops.o)
                              d:/programfiles/nxp/mcuxpressoide_11.1.0_3209/ide/plugins/com.nxp.mcuxpresso.tools.win32_11.1.0.201909161352/tools/bin/../lib/gcc/arm-none-eabi/8.3.1/../../../../arm-none-eabi/lib/thumb/v7e-m+fp/hard\libstdc++.a(guard_error.o) (operator delete(void*, unsigned int))
d:/programfiles/nxp/mcuxpressoide_11.1.0_3209/ide/plugins/com.nxp.mcuxpresso.tools.win32_11.1.0.201909161352/tools/bin/../lib/gcc/arm-none-eabi/8.3.1/../../../../arm-none-eabi/lib/thumb/v7e-m+fp/hard\libstdc++.a(bad_typeid.o)
                              d:/programfiles/nxp/mcuxpressoide_11.1.0_3209/ide/plugins/com.nxp.mcuxpresso.tools.win32_11.1.0.201909161352/tools/bin/../lib/gcc/arm-none-eabi/8.3.1/../../../../arm-none-eabi/lib/thumb/v7e-m+fp/hard\libstdc++.a(functexcept.o) (std::bad_typeid::~bad_typeid())
d:/programfiles/nxp/mcuxpressoide_11.1.0_3209/ide/plugins/com.nxp.mcuxpresso.tools.win32_11.1.0.201909161352/tools/bin/../lib/gcc/arm-none-eabi/8.3.1/../../../../arm-none-eabi/lib/thumb/v7e-m+fp/hard\libstdc++.a(si_class_type_info.o)
                              d:/programfiles/nxp/mcuxpressoide_11.1.0_3209/ide/plugins/com.nxp.mcuxpresso.tools.win32_11.1.0.201909161352/tools/bin/../lib/gcc/arm-none-eabi/8.3.1/../../../../arm-none-eabi/lib/thumb/v7e-m+fp/hard\libstdc++.a(guard_error.o) (vtable for __cxxabiv1::__si_class_type_info)
d:/programfiles/nxp/mcuxpressoide_11.1.0_3209/ide/plugins/com.nxp.mcuxpresso.tools.win32_11.1.0.201909161352/tools/bin/../lib/gcc/arm-none-eabi/8.3.1/../../../../arm-none-eabi/lib/thumb/v7e-m+fp/hard\libstdc++.a(tinfo.o)
                              d:/programfiles/nxp/mcuxpressoide_11.1.0_3209/ide/plugins/com.nxp.mcuxpresso.tools.win32_11.1.0.201909161352/tools/bin/../lib/gcc/arm-none-eabi/8.3.1/../../../../arm-none-eabi/lib/thumb/v7e-m+fp/hard\libstdc++.a(si_class_type_info.o) (std::type_info::__is_pointer_p() const)
d:/programfiles/nxp/mcuxpressoide_11.1.0_3209/ide/plugins/com.nxp.mcuxpresso.tools.win32_11.1.0.201909161352/tools/bin/../lib/gcc/arm-none-eabi/8.3.1/../../../../arm-none-eabi/lib/thumb/v7e-m+fp/hard\libstdc++.a(class_type_info.o)
                              d:/programfiles/nxp/mcuxpressoide_11.1.0_3209/ide/plugins/com.nxp.mcuxpresso.tools.win32_11.1.0.201909161352/tools/bin/../lib/gcc/arm-none-eabi/8.3.1/../../../../arm-none-eabi/lib/thumb/v7e-m+fp/hard\libstdc++.a(si_class_type_info.o) (__cxxabiv1::__class_type_info::__do_upcast(__cxxabiv1::__class_type_info const*, void**) const)
d:/programfiles/nxp/mcuxpressoide_11.1.0_3209/ide/plugins/com.nxp.mcuxpresso.tools.win32_11.1.0.201909161352/tools/bin/../lib/gcc/arm-none-eabi/8.3.1/../../../../arm-none-eabi/lib/thumb/v7e-m+fp/hard\libstdc++.a(stdexcept.o)
                              d:/programfiles/nxp/mcuxpressoide_11.1.0_3209/ide/plugins/com.nxp.mcuxpresso.tools.win32_11.1.0.201909161352/tools/bin/../lib/gcc/arm-none-eabi/8.3.1/../../../../arm-none-eabi/lib/thumb/v7e-m+fp/hard\libstdc++.a(functexcept.o) (std::logic_error::~logic_error())
d:/programfiles/nxp/mcuxpressoide_11.1.0_3209/ide/plugins/com.nxp.mcuxpresso.tools.win32_11.1.0.201909161352/tools/bin/../lib/gcc/arm-none-eabi/8.3.1/../../../../arm-none-eabi/lib/thumb/v7e-m+fp/hard\libstdc++.a(cow-string-inst.o)
                              d:/programfiles/nxp/mcuxpressoide_11.1.0_3209/ide/plugins/com.nxp.mcuxpresso.tools.win32_11.1.0.201909161352/tools/bin/../lib/gcc/arm-none-eabi/8.3.1/../../../../arm-none-eabi/lib/thumb/v7e-m+fp/hard\libstdc++.a(stdexcept.o) (std::string::_Rep::_S_empty_rep_storage)
d:/programfiles/nxp/mcuxpressoide_11.1.0_3209/ide/plugins/com.nxp.mcuxpresso.tools.win32_11.1.0.201909161352/tools/bin/../lib/gcc/arm-none-eabi/8.3.1/../../../../arm-none-eabi/lib/thumb/v7e-m+fp/hard\libstdc++.a(cow-stdexcept.o)
                              d:/programfiles/nxp/mcuxpressoide_11.1.0_3209/ide/plugins/com.nxp.mcuxpresso.tools.win32_11.1.0.201909161352/tools/bin/../lib/gcc/arm-none-eabi/8.3.1/../../../../arm-none-eabi/lib/thumb/v7e-m+fp/hard\libstdc++.a(functexcept.o) (std::logic_error::logic_error(char const*))
d:/programfiles/nxp/mcuxpressoide_11.1.0_3209/ide/plugins/com.nxp.mcuxpresso.tools.win32_11.1.0.201909161352/tools/bin/../lib/gcc/arm-none-eabi/8.3.1/../../../../arm-none-eabi/lib/thumb/v7e-m+fp/hard\libstdc++.a(snprintf_lite.o)
                              d:/programfiles/nxp/mcuxpressoide_11.1.0_3209/ide/plugins/com.nxp.mcuxpresso.tools.win32_11.1.0.201909161352/tools/bin/../lib/gcc/arm-none-eabi/8.3.1/../../../../arm-none-eabi/lib/thumb/v7e-m+fp/hard\libstdc++.a(functexcept.o) (__gnu_cxx::__snprintf_lite(char*, unsigned int, char const*, std::__va_list))
d:/programfiles/nxp/mcuxpressoide_11.1.0_3209/ide/plugins/com.nxp.mcuxpresso.tools.win32_11.1.0.201909161352/tools/bin/../lib/gcc/arm-none-eabi/8.3.1/../../../../arm-none-eabi/lib/thumb/v7e-m+fp/hard\libstdc++.a(sso_string.o)
                              d:/programfiles/nxp/mcuxpressoide_11.1.0_3209/ide/plugins/com.nxp.mcuxpresso.tools.win32_11.1.0.201909161352/tools/bin/../lib/gcc/arm-none-eabi/8.3.1/../../../../arm-none-eabi/lib/thumb/v7e-m+fp/hard\libstdc++.a(cow-stdexcept.o) (std::__sso_string::__sso_string(char const*, unsigned int))
d:/programfiles/nxp/mcuxpressoide_11.1.0_3209/ide/plugins/com.nxp.mcuxpresso.tools.win32_11.1.0.201909161352/tools/bin/../lib/gcc/arm-none-eabi/8.3.1/../../../../arm-none-eabi/lib/thumb/v7e-m+fp/hard\libm.a(lib_a-s_fabs.o)
                              ./open62541/open62541.o (fabs)
d:/programfiles/nxp/mcuxpressoide_11.1.0_3209/ide/plugins/com.nxp.mcuxpresso.tools.win32_11.1.0.201909161352/tools/bin/../lib/gcc/arm-none-eabi/8.3.1/../../../../arm-none-eabi/lib/thumb/v7e-m+fp/hard\libm.a(lib_a-w_pow.o)
                              ./source/Devices.o (pow)
d:/programfiles/nxp/mcuxpressoide_11.1.0_3209/ide/plugins/com.nxp.mcuxpresso.tools.win32_11.1.0.201909161352/tools/bin/../lib/gcc/arm-none-eabi/8.3.1/../../../../arm-none-eabi/lib/thumb/v7e-m+fp/hard\libm.a(lib_a-e_pow.o)
                              d:/programfiles/nxp/mcuxpressoide_11.1.0_3209/ide/plugins/com.nxp.mcuxpresso.tools.win32_11.1.0.201909161352/tools/bin/../lib/gcc/arm-none-eabi/8.3.1/../../../../arm-none-eabi/lib/thumb/v7e-m+fp/hard\libm.a(lib_a-w_pow.o) (__ieee754_pow)
d:/programfiles/nxp/mcuxpressoide_11.1.0_3209/ide/plugins/com.nxp.mcuxpresso.tools.win32_11.1.0.201909161352/tools/bin/../lib/gcc/arm-none-eabi/8.3.1/../../../../arm-none-eabi/lib/thumb/v7e-m+fp/hard\libm.a(lib_a-e_sqrt.o)
                              d:/programfiles/nxp/mcuxpressoide_11.1.0_3209/ide/plugins/com.nxp.mcuxpresso.tools.win32_11.1.0.201909161352/tools/bin/../lib/gcc/arm-none-eabi/8.3.1/../../../../arm-none-eabi/lib/thumb/v7e-m+fp/hard\libm.a(lib_a-e_pow.o) (__ieee754_sqrt)
d:/programfiles/nxp/mcuxpressoide_11.1.0_3209/ide/plugins/com.nxp.mcuxpresso.tools.win32_11.1.0.201909161352/tools/bin/../lib/gcc/arm-none-eabi/8.3.1/../../../../arm-none-eabi/lib/thumb/v7e-m+fp/hard\libm.a(lib_a-s_finite.o)
                              d:/programfiles/nxp/mcuxpressoide_11.1.0_3209/ide/plugins/com.nxp.mcuxpresso.tools.win32_11.1.0.201909161352/tools/bin/../lib/gcc/arm-none-eabi/8.3.1/../../../../arm-none-eabi/lib/thumb/v7e-m+fp/hard\libm.a(lib_a-w_pow.o) (finite)
d:/programfiles/nxp/mcuxpressoide_11.1.0_3209/ide/plugins/com.nxp.mcuxpresso.tools.win32_11.1.0.201909161352/tools/bin/../lib/gcc/arm-none-eabi/8.3.1/../../../../arm-none-eabi/lib/thumb/v7e-m+fp/hard\libm.a(lib_a-s_lib_ver.o)
                              d:/programfiles/nxp/mcuxpressoide_11.1.0_3209/ide/plugins/com.nxp.mcuxpresso.tools.win32_11.1.0.201909161352/tools/bin/../lib/gcc/arm-none-eabi/8.3.1/../../../../arm-none-eabi/lib/thumb/v7e-m+fp/hard\libm.a(lib_a-w_pow.o) (__fdlib_version)
d:/programfiles/nxp/mcuxpressoide_11.1.0_3209/ide/plugins/com.nxp.mcuxpresso.tools.win32_11.1.0.201909161352/tools/bin/../lib/gcc/arm-none-eabi/8.3.1/../../../../arm-none-eabi/lib/thumb/v7e-m+fp/hard\libm.a(lib_a-s_nan.o)
                              d:/programfiles/nxp/mcuxpressoide_11.1.0_3209/ide/plugins/com.nxp.mcuxpresso.tools.win32_11.1.0.201909161352/tools/bin/../lib/gcc/arm-none-eabi/8.3.1/../../../../arm-none-eabi/lib/thumb/v7e-m+fp/hard\libm.a(lib_a-e_pow.o) (nan)
d:/programfiles/nxp/mcuxpressoide_11.1.0_3209/ide/plugins/com.nxp.mcuxpresso.tools.win32_11.1.0.201909161352/tools/bin/../lib/gcc/arm-none-eabi/8.3.1/../../../../arm-none-eabi/lib/thumb/v7e-m+fp/hard\libm.a(lib_a-s_rint.o)
                              d:/programfiles/nxp/mcuxpressoide_11.1.0_3209/ide/plugins/com.nxp.mcuxpresso.tools.win32_11.1.0.201909161352/tools/bin/../lib/gcc/arm-none-eabi/8.3.1/../../../../arm-none-eabi/lib/thumb/v7e-m+fp/hard\libm.a(lib_a-w_pow.o) (rint)
d:/programfiles/nxp/mcuxpressoide_11.1.0_3209/ide/plugins/com.nxp.mcuxpresso.tools.win32_11.1.0.201909161352/tools/bin/../lib/gcc/arm-none-eabi/8.3.1/../../../../arm-none-eabi/lib/thumb/v7e-m+fp/hard\libm.a(lib_a-s_scalbn.o)
                              d:/programfiles/nxp/mcuxpressoide_11.1.0_3209/ide/plugins/com.nxp.mcuxpresso.tools.win32_11.1.0.201909161352/tools/bin/../lib/gcc/arm-none-eabi/8.3.1/../../../../arm-none-eabi/lib/thumb/v7e-m+fp/hard\libm.a(lib_a-e_pow.o) (scalbn)
d:/programfiles/nxp/mcuxpressoide_11.1.0_3209/ide/plugins/com.nxp.mcuxpresso.tools.win32_11.1.0.201909161352/tools/bin/../lib/gcc/arm-none-eabi/8.3.1/../../../../arm-none-eabi/lib/thumb/v7e-m+fp/hard\libcr_newlib_semihost.a(_cr_sbrk.o)
                              d:/programfiles/nxp/mcuxpressoide_11.1.0_3209/ide/plugins/com.nxp.mcuxpresso.tools.win32_11.1.0.201909161352/tools/bin/../lib/gcc/arm-none-eabi/8.3.1/../../../../arm-none-eabi/lib/thumb/v7e-m+fp/hard\libc.a(lib_a-sbrkr.o) (_sbrk)
d:/programfiles/nxp/mcuxpressoide_11.1.0_3209/ide/plugins/com.nxp.mcuxpresso.tools.win32_11.1.0.201909161352/tools/bin/../lib/gcc/arm-none-eabi/8.3.1/../../../../arm-none-eabi/lib/thumb/v7e-m+fp/hard\libcr_newlib_semihost.a(syscalls.o)
                              d:/programfiles/nxp/mcuxpressoide_11.1.0_3209/ide/plugins/com.nxp.mcuxpresso.tools.win32_11.1.0.201909161352/tools/bin/../lib/gcc/arm-none-eabi/8.3.1/../../../../arm-none-eabi/lib/thumb/v7e-m+fp/hard\libc.a(lib_a-readr.o) (_read)
d:/programfiles/nxp/mcuxpressoide_11.1.0_3209/ide/plugins/com.nxp.mcuxpresso.tools.win32_11.1.0.201909161352/tools/bin/../lib/gcc/arm-none-eabi/8.3.1/../../../../arm-none-eabi/lib/thumb/v7e-m+fp/hard\libcr_newlib_semihost.a(_cr_check_heap.o)
                              d:/programfiles/nxp/mcuxpressoide_11.1.0_3209/ide/plugins/com.nxp.mcuxpresso.tools.win32_11.1.0.201909161352/tools/bin/../lib/gcc/arm-none-eabi/8.3.1/../../../../arm-none-eabi/lib/thumb/v7e-m+fp/hard\libcr_newlib_semihost.a(_cr_sbrk.o) (__check_heap_overflow)
d:/programfiles/nxp/mcuxpressoide_11.1.0_3209/ide/plugins/com.nxp.mcuxpresso.tools.win32_11.1.0.201909161352/tools/bin/../lib/gcc/arm-none-eabi/8.3.1/thumb/v7e-m+fp/hard\libgcc.a(_arm_unorddf2.o)
                              d:/programfiles/nxp/mcuxpressoide_11.1.0_3209/ide/plugins/com.nxp.mcuxpresso.tools.win32_11.1.0.201909161352/tools/bin/../lib/gcc/arm-none-eabi/8.3.1/../../../../arm-none-eabi/lib/thumb/v7e-m+fp/hard\libc.a(lib_a-svfprintf.o) (__aeabi_dcmpun)
d:/programfiles/nxp/mcuxpressoide_11.1.0_3209/ide/plugins/com.nxp.mcuxpresso.tools.win32_11.1.0.201909161352/tools/bin/../lib/gcc/arm-none-eabi/8.3.1/thumb/v7e-m+fp/hard\libgcc.a(_arm_fixdfsi.o)
                              d:/programfiles/nxp/mcuxpressoide_11.1.0_3209/ide/plugins/com.nxp.mcuxpresso.tools.win32_11.1.0.201909161352/tools/bin/../lib/gcc/arm-none-eabi/8.3.1/../../../../arm-none-eabi/lib/thumb/v7e-m+fp/hard\libc.a(lib_a-svfprintf.o) (__aeabi_d2iz)
d:/programfiles/nxp/mcuxpressoide_11.1.0_3209/ide/plugins/com.nxp.mcuxpresso.tools.win32_11.1.0.201909161352/tools/bin/../lib/gcc/arm-none-eabi/8.3.1/thumb/v7e-m+fp/hard\libgcc.a(unwind-arm.o)
                              d:/programfiles/nxp/mcuxpressoide_11.1.0_3209/ide/plugins/com.nxp.mcuxpresso.tools.win32_11.1.0.201909161352/tools/bin/../lib/gcc/arm-none-eabi/8.3.1/../../../../arm-none-eabi/lib/thumb/v7e-m+fp/hard\libstdc++.a(eh_arm.o) (__aeabi_unwind_cpp_pr0)
d:/programfiles/nxp/mcuxpressoide_11.1.0_3209/ide/plugins/com.nxp.mcuxpresso.tools.win32_11.1.0.201909161352/tools/bin/../lib/gcc/arm-none-eabi/8.3.1/thumb/v7e-m+fp/hard\libgcc.a(libunwind.o)
                              d:/programfiles/nxp/mcuxpressoide_11.1.0_3209/ide/plugins/com.nxp.mcuxpresso.tools.win32_11.1.0.201909161352/tools/bin/../lib/gcc/arm-none-eabi/8.3.1/thumb/v7e-m+fp/hard\libgcc.a(unwind-arm.o) (restore_core_regs)
d:/programfiles/nxp/mcuxpressoide_11.1.0_3209/ide/plugins/com.nxp.mcuxpresso.tools.win32_11.1.0.201909161352/tools/bin/../lib/gcc/arm-none-eabi/8.3.1/thumb/v7e-m+fp/hard\libgcc.a(pr-support.o)
                              d:/programfiles/nxp/mcuxpressoide_11.1.0_3209/ide/plugins/com.nxp.mcuxpresso.tools.win32_11.1.0.201909161352/tools/bin/../lib/gcc/arm-none-eabi/8.3.1/thumb/v7e-m+fp/hard\libgcc.a(unwind-arm.o) (__gnu_unwind_execute)
d:/programfiles/nxp/mcuxpressoide_11.1.0_3209/ide/plugins/com.nxp.mcuxpresso.tools.win32_11.1.0.201909161352/tools/bin/../lib/gcc/arm-none-eabi/8.3.1/../../../../arm-none-eabi/lib/thumb/v7e-m+fp/hard\libc.a(lib_a-abort.o)
                              d:/programfiles/nxp/mcuxpressoide_11.1.0_3209/ide/plugins/com.nxp.mcuxpresso.tools.win32_11.1.0.201909161352/tools/bin/../lib/gcc/arm-none-eabi/8.3.1/../../../../arm-none-eabi/lib/thumb/v7e-m+fp/hard\libstdc++.a(eh_terminate.o) (abort)
d:/programfiles/nxp/mcuxpressoide_11.1.0_3209/ide/plugins/com.nxp.mcuxpresso.tools.win32_11.1.0.201909161352/tools/bin/../lib/gcc/arm-none-eabi/8.3.1/../../../../arm-none-eabi/lib/thumb/v7e-m+fp/hard\libc.a(lib_a-errno.o)
                              d:/programfiles/nxp/mcuxpressoide_11.1.0_3209/ide/plugins/com.nxp.mcuxpresso.tools.win32_11.1.0.201909161352/tools/bin/../lib/gcc/arm-none-eabi/8.3.1/../../../../arm-none-eabi/lib/thumb/v7e-m+fp/hard\libm.a(lib_a-w_pow.o) (__errno)
d:/programfiles/nxp/mcuxpressoide_11.1.0_3209/ide/plugins/com.nxp.mcuxpresso.tools.win32_11.1.0.201909161352/tools/bin/../lib/gcc/arm-none-eabi/8.3.1/../../../../arm-none-eabi/lib/thumb/v7e-m+fp/hard\libc.a(lib_a-fopen.o)
                              d:/programfiles/nxp/mcuxpressoide_11.1.0_3209/ide/plugins/com.nxp.mcuxpresso.tools.win32_11.1.0.201909161352/tools/bin/../lib/gcc/arm-none-eabi/8.3.1/../../../../arm-none-eabi/lib/thumb/v7e-m+fp/hard\libstdc++.a(cow-string-inst.o) (fopen)
d:/programfiles/nxp/mcuxpressoide_11.1.0_3209/ide/plugins/com.nxp.mcuxpresso.tools.win32_11.1.0.201909161352/tools/bin/../lib/gcc/arm-none-eabi/8.3.1/../../../../arm-none-eabi/lib/thumb/v7e-m+fp/hard\libc.a(lib_a-fseek.o)
                              d:/programfiles/nxp/mcuxpressoide_11.1.0_3209/ide/plugins/com.nxp.mcuxpresso.tools.win32_11.1.0.201909161352/tools/bin/../lib/gcc/arm-none-eabi/8.3.1/../../../../arm-none-eabi/lib/thumb/v7e-m+fp/hard\libc.a(lib_a-fopen.o) (_fseek_r)
d:/programfiles/nxp/mcuxpressoide_11.1.0_3209/ide/plugins/com.nxp.mcuxpresso.tools.win32_11.1.0.201909161352/tools/bin/../lib/gcc/arm-none-eabi/8.3.1/../../../../arm-none-eabi/lib/thumb/v7e-m+fp/hard\libc.a(lib_a-fseeko.o)
                              d:/programfiles/nxp/mcuxpressoide_11.1.0_3209/ide/plugins/com.nxp.mcuxpresso.tools.win32_11.1.0.201909161352/tools/bin/../lib/gcc/arm-none-eabi/8.3.1/../../../../arm-none-eabi/lib/thumb/v7e-m+fp/hard\libc.a(lib_a-fseek.o) (_fseeko_r)
d:/programfiles/nxp/mcuxpressoide_11.1.0_3209/ide/plugins/com.nxp.mcuxpresso.tools.win32_11.1.0.201909161352/tools/bin/../lib/gcc/arm-none-eabi/8.3.1/../../../../arm-none-eabi/lib/thumb/v7e-m+fp/hard\libc.a(lib_a-openr.o)
                              d:/programfiles/nxp/mcuxpressoide_11.1.0_3209/ide/plugins/com.nxp.mcuxpresso.tools.win32_11.1.0.201909161352/tools/bin/../lib/gcc/arm-none-eabi/8.3.1/../../../../arm-none-eabi/lib/thumb/v7e-m+fp/hard\libc.a(lib_a-fopen.o) (_open_r)
d:/programfiles/nxp/mcuxpressoide_11.1.0_3209/ide/plugins/com.nxp.mcuxpresso.tools.win32_11.1.0.201909161352/tools/bin/../lib/gcc/arm-none-eabi/8.3.1/../../../../arm-none-eabi/lib/thumb/v7e-m+fp/hard\libc.a(lib_a-refill.o)
                              d:/programfiles/nxp/mcuxpressoide_11.1.0_3209/ide/plugins/com.nxp.mcuxpresso.tools.win32_11.1.0.201909161352/tools/bin/../lib/gcc/arm-none-eabi/8.3.1/../../../../arm-none-eabi/lib/thumb/v7e-m+fp/hard\libc.a(lib_a-fseeko.o) (__srefill_r)
d:/programfiles/nxp/mcuxpressoide_11.1.0_3209/ide/plugins/com.nxp.mcuxpresso.tools.win32_11.1.0.201909161352/tools/bin/../lib/gcc/arm-none-eabi/8.3.1/../../../../arm-none-eabi/lib/thumb/v7e-m+fp/hard\libc.a(lib_a-signal.o)
                              d:/programfiles/nxp/mcuxpressoide_11.1.0_3209/ide/plugins/com.nxp.mcuxpresso.tools.win32_11.1.0.201909161352/tools/bin/../lib/gcc/arm-none-eabi/8.3.1/../../../../arm-none-eabi/lib/thumb/v7e-m+fp/hard\libc.a(lib_a-abort.o) (raise)
d:/programfiles/nxp/mcuxpressoide_11.1.0_3209/ide/plugins/com.nxp.mcuxpresso.tools.win32_11.1.0.201909161352/tools/bin/../lib/gcc/arm-none-eabi/8.3.1/../../../../arm-none-eabi/lib/thumb/v7e-m+fp/hard\libc.a(lib_a-signalr.o)
                              d:/programfiles/nxp/mcuxpressoide_11.1.0_3209/ide/plugins/com.nxp.mcuxpresso.tools.win32_11.1.0.201909161352/tools/bin/../lib/gcc/arm-none-eabi/8.3.1/../../../../arm-none-eabi/lib/thumb/v7e-m+fp/hard\libc.a(lib_a-signal.o) (_kill_r)
d:/programfiles/nxp/mcuxpressoide_11.1.0_3209/ide/plugins/com.nxp.mcuxpresso.tools.win32_11.1.0.201909161352/tools/bin/../lib/gcc/arm-none-eabi/8.3.1/../../../../arm-none-eabi/lib/thumb/v7e-m+fp/hard\libc.a(lib_a-strtoul.o)
                              d:/programfiles/nxp/mcuxpressoide_11.1.0_3209/ide/plugins/com.nxp.mcuxpresso.tools.win32_11.1.0.201909161352/tools/bin/../lib/gcc/arm-none-eabi/8.3.1/../../../../arm-none-eabi/lib/thumb/v7e-m+fp/hard\libstdc++.a(cow-string-inst.o) (strtoul)
d:/programfiles/nxp/mcuxpressoide_11.1.0_3209/ide/plugins/com.nxp.mcuxpresso.tools.win32_11.1.0.201909161352/tools/bin/../lib/gcc/arm-none-eabi/8.3.1/../../../../arm-none-eabi/lib/thumb/v7e-m+fp/hard\libc.a(lib_a-syswrite.o)
                              d:/programfiles/nxp/mcuxpressoide_11.1.0_3209/ide/plugins/com.nxp.mcuxpresso.tools.win32_11.1.0.201909161352/tools/bin/../lib/gcc/arm-none-eabi/8.3.1/../../../../arm-none-eabi/lib/thumb/v7e-m+fp/hard\libstdc++.a(pure.o) (write)
d:/programfiles/nxp/mcuxpressoide_11.1.0_3209/ide/plugins/com.nxp.mcuxpresso.tools.win32_11.1.0.201909161352/tools/bin/../lib/gcc/arm-none-eabi/8.3.1/../../../../arm-none-eabi/lib/thumb/v7e-m+fp/hard\libc.a(lib_a-flags.o)
                              d:/programfiles/nxp/mcuxpressoide_11.1.0_3209/ide/plugins/com.nxp.mcuxpresso.tools.win32_11.1.0.201909161352/tools/bin/../lib/gcc/arm-none-eabi/8.3.1/../../../../arm-none-eabi/lib/thumb/v7e-m+fp/hard\libc.a(lib_a-fopen.o) (__sflags)
d:/programfiles/nxp/mcuxpressoide_11.1.0_3209/ide/plugins/com.nxp.mcuxpresso.tools.win32_11.1.0.201909161352/tools/bin/../lib/gcc/arm-none-eabi/8.3.1/../../../../arm-none-eabi/lib/thumb/v7e-m+fp/hard\libcr_newlib_semihost.a(_exit.o)
                              d:/programfiles/nxp/mcuxpressoide_11.1.0_3209/ide/plugins/com.nxp.mcuxpresso.tools.win32_11.1.0.201909161352/tools/bin/../lib/gcc/arm-none-eabi/8.3.1/../../../../arm-none-eabi/lib/thumb/v7e-m+fp/hard\libc.a(lib_a-abort.o) (_exit)
d:/programfiles/nxp/mcuxpressoide_11.1.0_3209/ide/plugins/com.nxp.mcuxpresso.tools.win32_11.1.0.201909161352/tools/bin/../lib/gcc/arm-none-eabi/8.3.1/../../../../arm-none-eabi/lib/thumb/v7e-m+fp/hard\libcr_newlib_semihost.a(_kill.o)
                              d:/programfiles/nxp/mcuxpressoide_11.1.0_3209/ide/plugins/com.nxp.mcuxpresso.tools.win32_11.1.0.201909161352/tools/bin/../lib/gcc/arm-none-eabi/8.3.1/../../../../arm-none-eabi/lib/thumb/v7e-m+fp/hard\libc.a(lib_a-signalr.o) (_kill)

Allocating common symbols
Common symbol       size              file

__lock___atexit_recursive_mutex
                    0x1               d:/programfiles/nxp/mcuxpressoide_11.1.0_3209/ide/plugins/com.nxp.mcuxpresso.tools.win32_11.1.0.201909161352/tools/bin/../lib/gcc/arm-none-eabi/8.3.1/../../../../arm-none-eabi/lib/thumb/v7e-m+fp/hard\libc.a(lib_a-lock.o)
__lock___arc4random_mutex
                    0x1               d:/programfiles/nxp/mcuxpressoide_11.1.0_3209/ide/plugins/com.nxp.mcuxpresso.tools.win32_11.1.0.201909161352/tools/bin/../lib/gcc/arm-none-eabi/8.3.1/../../../../arm-none-eabi/lib/thumb/v7e-m+fp/hard\libc.a(lib_a-lock.o)
__lock___env_recursive_mutex
                    0x1               d:/programfiles/nxp/mcuxpressoide_11.1.0_3209/ide/plugins/com.nxp.mcuxpresso.tools.win32_11.1.0.201909161352/tools/bin/../lib/gcc/arm-none-eabi/8.3.1/../../../../arm-none-eabi/lib/thumb/v7e-m+fp/hard\libc.a(lib_a-lock.o)
__lock___sinit_recursive_mutex
                    0x1               d:/programfiles/nxp/mcuxpressoide_11.1.0_3209/ide/plugins/com.nxp.mcuxpresso.tools.win32_11.1.0.201909161352/tools/bin/../lib/gcc/arm-none-eabi/8.3.1/../../../../arm-none-eabi/lib/thumb/v7e-m+fp/hard\libc.a(lib_a-lock.o)
__lock___malloc_recursive_mutex
                    0x1               d:/programfiles/nxp/mcuxpressoide_11.1.0_3209/ide/plugins/com.nxp.mcuxpresso.tools.win32_11.1.0.201909161352/tools/bin/../lib/gcc/arm-none-eabi/8.3.1/../../../../arm-none-eabi/lib/thumb/v7e-m+fp/hard\libc.a(lib_a-lock.o)
__lock___at_quick_exit_mutex
                    0x1               d:/programfiles/nxp/mcuxpressoide_11.1.0_3209/ide/plugins/com.nxp.mcuxpresso.tools.win32_11.1.0.201909161352/tools/bin/../lib/gcc/arm-none-eabi/8.3.1/../../../../arm-none-eabi/lib/thumb/v7e-m+fp/hard\libc.a(lib_a-lock.o)
__lock___dd_hash_mutex
                    0x1               d:/programfiles/nxp/mcuxpressoide_11.1.0_3209/ide/plugins/com.nxp.mcuxpresso.tools.win32_11.1.0.201909161352/tools/bin/../lib/gcc/arm-none-eabi/8.3.1/../../../../arm-none-eabi/lib/thumb/v7e-m+fp/hard\libc.a(lib_a-lock.o)
__lock___tz_mutex   0x1               d:/programfiles/nxp/mcuxpressoide_11.1.0_3209/ide/plugins/com.nxp.mcuxpresso.tools.win32_11.1.0.201909161352/tools/bin/../lib/gcc/arm-none-eabi/8.3.1/../../../../arm-none-eabi/lib/thumb/v7e-m+fp/hard\libc.a(lib_a-lock.o)
__lock___sfp_recursive_mutex
                    0x1               d:/programfiles/nxp/mcuxpressoide_11.1.0_3209/ide/plugins/com.nxp.mcuxpresso.tools.win32_11.1.0.201909161352/tools/bin/../lib/gcc/arm-none-eabi/8.3.1/../../../../arm-none-eabi/lib/thumb/v7e-m+fp/hard\libc.a(lib_a-lock.o)

Discarded input sections

 .group         0x00000000        0xc ./xip/evkmimxrt1060_flexspi_nor_config.o
 .group         0x00000000        0xc ./xip/evkmimxrt1060_flexspi_nor_config.o
 .group         0x00000000        0xc ./xip/evkmimxrt1060_flexspi_nor_config.o
 .group         0x00000000        0xc ./xip/evkmimxrt1060_flexspi_nor_config.o
 .group         0x00000000        0xc ./xip/evkmimxrt1060_flexspi_nor_config.o
 .group         0x00000000        0xc ./xip/evkmimxrt1060_flexspi_nor_config.o
 .group         0x00000000        0xc ./xip/evkmimxrt1060_flexspi_nor_config.o
 .group         0x00000000        0xc ./xip/evkmimxrt1060_flexspi_nor_config.o
 .group         0x00000000        0xc ./xip/evkmimxrt1060_flexspi_nor_config.o
 .group         0x00000000        0xc ./xip/evkmimxrt1060_flexspi_nor_config.o
 .group         0x00000000        0xc ./xip/evkmimxrt1060_flexspi_nor_config.o
 .group         0x00000000        0xc ./xip/evkmimxrt1060_flexspi_nor_config.o
 .group         0x00000000        0xc ./xip/evkmimxrt1060_flexspi_nor_config.o
 .group         0x00000000        0xc ./xip/evkmimxrt1060_flexspi_nor_config.o
 .group         0x00000000        0xc ./xip/evkmimxrt1060_flexspi_nor_config.o
 .group         0x00000000        0xc ./xip/evkmimxrt1060_flexspi_nor_config.o
 .group         0x00000000        0xc ./xip/evkmimxrt1060_flexspi_nor_config.o
 .group         0x00000000        0xc ./xip/evkmimxrt1060_flexspi_nor_config.o
Memory Configuration

Name             Origin             Length             Attributes
BOARD_FLASH      0x60000000         0x00400000         xr
SRAM_OC          0x20200000         0x000c0000         xrw
SRAM_DTC         0x20000000         0x00020000         xrw
SRAM_ITC         0x00000000         0x00020000         xrw
BOARD_SDRAM      0x80000000         0x01e00000         xrw
NCACHE_REGION    0x81e00000         0x00200000         xrw
*default*        0x00000000         0xffffffff

Linker script and memory map

LOAD ./xip/evkmimxrt1060_flexspi_nor_config.o
LOAD ./xip/evkmimxrt1060_sdram_ini_dcd.o
LOAD ./xip/fsl_flexspi_nor_boot.o
LOAD ./utilities/fsl_assert.o
LOAD ./utilities/fsl_debug_console.o
LOAD ./utilities/fsl_str.o
LOAD ./startup/startup_mimxrt1062.o
LOAD ./source/Devices.o
LOAD ./source/commands.o
LOAD ./source/common.o
LOAD ./source/cpp_config.o
LOAD ./source/main_MandC.o
LOAD ./source/node.o
LOAD ./source/semihost_hardfault.o
LOAD ./open62541/open62541.o
LOAD ./nanopb/generated/RCU2.pb.o
LOAD ./nanopb/pb_common.o
LOAD ./nanopb/pb_decode.o
LOAD ./nanopb/pb_encode.o
LOAD ./lwip/src/netif/ppp/polarssl/arc4.o
LOAD ./lwip/src/netif/ppp/polarssl/des.o
LOAD ./lwip/src/netif/ppp/polarssl/md4.o
LOAD ./lwip/src/netif/ppp/polarssl/md5.o
LOAD ./lwip/src/netif/ppp/polarssl/sha1.o
LOAD ./lwip/src/netif/ppp/auth.o
LOAD ./lwip/src/netif/ppp/ccp.o
LOAD ./lwip/src/netif/ppp/chap-md5.o
LOAD ./lwip/src/netif/ppp/chap-new.o
LOAD ./lwip/src/netif/ppp/chap_ms.o
LOAD ./lwip/src/netif/ppp/demand.o
LOAD ./lwip/src/netif/ppp/eap.o
LOAD ./lwip/src/netif/ppp/eui64.o
LOAD ./lwip/src/netif/ppp/fsm.o
LOAD ./lwip/src/netif/ppp/ipcp.o
LOAD ./lwip/src/netif/ppp/ipv6cp.o
LOAD ./lwip/src/netif/ppp/lcp.o
LOAD ./lwip/src/netif/ppp/lwip_ecp.o
LOAD ./lwip/src/netif/ppp/magic.o
LOAD ./lwip/src/netif/ppp/mppe.o
LOAD ./lwip/src/netif/ppp/multilink.o
LOAD ./lwip/src/netif/ppp/ppp.o
LOAD ./lwip/src/netif/ppp/pppapi.o
LOAD ./lwip/src/netif/ppp/pppcrypt.o
LOAD ./lwip/src/netif/ppp/pppoe.o
LOAD ./lwip/src/netif/ppp/pppol2tp.o
LOAD ./lwip/src/netif/ppp/pppos.o
LOAD ./lwip/src/netif/ppp/upap.o
LOAD ./lwip/src/netif/ppp/utils.o
LOAD ./lwip/src/netif/ppp/vj.o
LOAD ./lwip/src/netif/bridgeif.o
LOAD ./lwip/src/netif/bridgeif_fdb.o
LOAD ./lwip/src/netif/ethernet.o
LOAD ./lwip/src/netif/lowpan6.o
LOAD ./lwip/src/netif/lowpan6_ble.o
LOAD ./lwip/src/netif/lowpan6_common.o
LOAD ./lwip/src/netif/slipif.o
LOAD ./lwip/src/netif/zepif.o
LOAD ./lwip/src/core/ipv6/dhcp6.o
LOAD ./lwip/src/core/ipv6/ethip6.o
LOAD ./lwip/src/core/ipv6/icmp6.o
LOAD ./lwip/src/core/ipv6/inet6.o
LOAD ./lwip/src/core/ipv6/ip6.o
LOAD ./lwip/src/core/ipv6/ip6_addr.o
LOAD ./lwip/src/core/ipv6/ip6_frag.o
LOAD ./lwip/src/core/ipv6/mld6.o
LOAD ./lwip/src/core/ipv6/nd6.o
LOAD ./lwip/src/core/ipv4/autoip.o
LOAD ./lwip/src/core/ipv4/dhcp.o
LOAD ./lwip/src/core/ipv4/etharp.o
LOAD ./lwip/src/core/ipv4/icmp.o
LOAD ./lwip/src/core/ipv4/igmp.o
LOAD ./lwip/src/core/ipv4/ip4.o
LOAD ./lwip/src/core/ipv4/ip4_addr.o
LOAD ./lwip/src/core/ipv4/ip4_frag.o
LOAD ./lwip/src/core/altcp.o
LOAD ./lwip/src/core/altcp_alloc.o
LOAD ./lwip/src/core/altcp_tcp.o
LOAD ./lwip/src/core/def.o
LOAD ./lwip/src/core/dns.o
LOAD ./lwip/src/core/inet_chksum.o
LOAD ./lwip/src/core/init.o
LOAD ./lwip/src/core/ip.o
LOAD ./lwip/src/core/mem.o
LOAD ./lwip/src/core/memp.o
LOAD ./lwip/src/core/netif.o
LOAD ./lwip/src/core/pbuf.o
LOAD ./lwip/src/core/raw.o
LOAD ./lwip/src/core/stats.o
LOAD ./lwip/src/core/sys.o
LOAD ./lwip/src/core/tcp.o
LOAD ./lwip/src/core/tcp_in.o
LOAD ./lwip/src/core/tcp_out.o
LOAD ./lwip/src/core/timeouts.o
LOAD ./lwip/src/core/udp.o
LOAD ./lwip/src/api/api_lib.o
LOAD ./lwip/src/api/api_msg.o
LOAD ./lwip/src/api/err.o
LOAD ./lwip/src/api/if_api.o
LOAD ./lwip/src/api/netbuf.o
LOAD ./lwip/src/api/netdb.o
LOAD ./lwip/src/api/netifapi.o
LOAD ./lwip/src/api/sockets.o
LOAD ./lwip/src/api/tcpip.o
LOAD ./lwip/port/enet_ethernetif.o
LOAD ./lwip/port/enet_ethernetif_kinetis.o
LOAD ./lwip/port/sys_arch.o
LOAD ./drivers/fsl_cache.o
LOAD ./drivers/fsl_clock.o
LOAD ./drivers/fsl_common.o
LOAD ./drivers/fsl_enet.o
LOAD ./drivers/fsl_flexio.o
LOAD ./drivers/fsl_flexio_i2c_master.o
LOAD ./drivers/fsl_gpio.o
LOAD ./drivers/fsl_gpt.o
LOAD ./drivers/fsl_lpi2c.o
LOAD ./drivers/fsl_lpi2c_freertos.o
LOAD ./drivers/fsl_lpuart.o
LOAD ./drivers/fsl_semc.o
LOAD ./drivers/fsl_tempmon.o
LOAD ./drivers/fsl_wdog.o
LOAD ./device/system_MIMXRT1062.o
LOAD ./component/uart/lpuart_adapter.o
LOAD ./component/timer_manager/timer_manager.o
LOAD ./component/timer/gpt_adapter.o
LOAD ./component/serial_manager/serial_manager.o
LOAD ./component/serial_manager/serial_port_uart.o
LOAD ./component/lists/generic_list.o
LOAD ./component/i2c/lpi2c_adapter.o
LOAD ./board/board.o
LOAD ./board/clock_config.o
LOAD ./board/fsl_phy.o
LOAD ./board/peripherals.o
LOAD ./board/pin_mux.o
LOAD ./amazon-freertos/freertos_kernel/portable/MemMang/heap_5.o
LOAD ./amazon-freertos/freertos_kernel/portable/GCC/ARM_CM4F/port.o
LOAD ./amazon-freertos/freertos_kernel/event_groups.o
LOAD ./amazon-freertos/freertos_kernel/list.o
LOAD ./amazon-freertos/freertos_kernel/queue.o
LOAD ./amazon-freertos/freertos_kernel/stream_buffer.o
LOAD ./amazon-freertos/freertos_kernel/tasks.o
LOAD ./amazon-freertos/freertos_kernel/timers.o
LOAD D:\projects\MCUXpresso\M_and_C\libs\libarm_cortexM7lfsp_math.a
LOAD D:\projects\MCUXpresso\M_and_C\libs\libarm_cortexM7lfdp_math.a
START GROUP
LOAD d:/programfiles/nxp/mcuxpressoide_11.1.0_3209/ide/plugins/com.nxp.mcuxpresso.tools.win32_11.1.0.201909161352/tools/bin/../lib/gcc/arm-none-eabi/8.3.1/thumb/v7e-m+fp/hard\libgcc.a
LOAD d:/programfiles/nxp/mcuxpressoide_11.1.0_3209/ide/plugins/com.nxp.mcuxpresso.tools.win32_11.1.0.201909161352/tools/bin/../lib/gcc/arm-none-eabi/8.3.1/../../../../arm-none-eabi/lib/thumb/v7e-m+fp/hard\libc.a
LOAD d:/programfiles/nxp/mcuxpressoide_11.1.0_3209/ide/plugins/com.nxp.mcuxpresso.tools.win32_11.1.0.201909161352/tools/bin/../lib/gcc/arm-none-eabi/8.3.1/../../../../arm-none-eabi/lib/thumb/v7e-m+fp/hard\libstdc++.a
LOAD d:/programfiles/nxp/mcuxpressoide_11.1.0_3209/ide/plugins/com.nxp.mcuxpresso.tools.win32_11.1.0.201909161352/tools/bin/../lib/gcc/arm-none-eabi/8.3.1/../../../../arm-none-eabi/lib/thumb/v7e-m+fp/hard\libm.a
LOAD d:/programfiles/nxp/mcuxpressoide_11.1.0_3209/ide/plugins/com.nxp.mcuxpresso.tools.win32_11.1.0.201909161352/tools/bin/../lib/gcc/arm-none-eabi/8.3.1/../../../../arm-none-eabi/lib/thumb/v7e-m+fp/hard\libcr_newlib_semihost.a
LOAD d:/programfiles/nxp/mcuxpressoide_11.1.0_3209/ide/plugins/com.nxp.mcuxpresso.tools.win32_11.1.0.201909161352/tools/bin/../lib/gcc/arm-none-eabi/8.3.1/thumb/v7e-m+fp/hard\crti.o
LOAD d:/programfiles/nxp/mcuxpressoide_11.1.0_3209/ide/plugins/com.nxp.mcuxpresso.tools.win32_11.1.0.201909161352/tools/bin/../lib/gcc/arm-none-eabi/8.3.1/thumb/v7e-m+fp/hard\crtn.o
LOAD d:/programfiles/nxp/mcuxpressoide_11.1.0_3209/ide/plugins/com.nxp.mcuxpresso.tools.win32_11.1.0.201909161352/tools/bin/../lib/gcc/arm-none-eabi/8.3.1/thumb/v7e-m+fp/hard\crtbegin.o
LOAD d:/programfiles/nxp/mcuxpressoide_11.1.0_3209/ide/plugins/com.nxp.mcuxpresso.tools.win32_11.1.0.201909161352/tools/bin/../lib/gcc/arm-none-eabi/8.3.1/thumb/v7e-m+fp/hard\crtend.o
END GROUP
                0x60000000                __base_BOARD_FLASH = 0x60000000
                0x60000000                __base_Flash = 0x60000000
                0x60400000                __top_BOARD_FLASH = 0x60400000
                0x60400000                __top_Flash = 0x60400000
                0x20200000                __base_SRAM_OC = 0x20200000
                0x20200000                __base_RAM = 0x20200000
                0x202c0000                __top_SRAM_OC = 0x202c0000
                0x202c0000                __top_RAM = 0x202c0000
                0x20000000                __base_SRAM_DTC = 0x20000000
                0x20000000                __base_RAM2 = 0x20000000
                0x20020000                __top_SRAM_DTC = 0x20020000
                0x20020000                __top_RAM2 = 0x20020000
                0x00000000                __base_SRAM_ITC = 0x0
                0x00000000                __base_RAM3 = 0x0
                0x00020000                __top_SRAM_ITC = 0x20000
                0x00020000                __top_RAM3 = 0x20000
                0x80000000                __base_BOARD_SDRAM = 0x80000000
                0x80000000                __base_RAM4 = 0x80000000
                0x81e00000                __top_BOARD_SDRAM = 0x81e00000
                0x81e00000                __top_RAM4 = 0x81e00000
                0x81e00000                __base_NCACHE_REGION = 0x81e00000
                0x81e00000                __base_RAM5 = 0x81e00000
                0x82000000                __top_NCACHE_REGION = 0x82000000
                0x82000000                __top_RAM5 = 0x82000000

.boot_hdr       0x60000000     0x2000
 FILL mask 0xff
                0x60000000                __boot_hdr_start__ = ABSOLUTE (.)
 *(SORT_BY_ALIGNMENT(.boot_hdr.conf))
 .boot_hdr.conf
                0x60000000      0x200 ./xip/evkmimxrt1060_flexspi_nor_config.o
                0x60000000                qspiflash_config
                0x00001000                . = 0x1000
 *fill*         0x60000200      0xe00 ff
 *(SORT_BY_ALIGNMENT(.boot_hdr.ivt))
 .boot_hdr.ivt  0x60001000       0x20 ./xip/fsl_flexspi_nor_boot.o
                0x60001000                image_vector_table
                0x00001020                . = 0x1020
 *(SORT_BY_ALIGNMENT(.boot_hdr.boot_data))
 .boot_hdr.boot_data
                0x60001020       0x10 ./xip/fsl_flexspi_nor_boot.o
                0x60001020                boot_data
                0x00001030                . = 0x1030
 *(SORT_BY_ALIGNMENT(.boot_hdr.dcd_data))
 .boot_hdr.dcd_data
                0x60001030      0x430 ./xip/evkmimxrt1060_sdram_ini_dcd.o
                0x60001030                dcd_data
                0x60001460                __boot_hdr_end__ = ABSOLUTE (.)
                0x00002000                . = 0x2000
 *fill*         0x60001460      0xba0 ff

.text           0x60002000    0x7b600
 FILL mask 0xff
                0x60002000                __vectors_start__ = ABSOLUTE (.)
 *(SORT_BY_ALIGNMENT(.isr_vector))
 .isr_vector    0x60002000      0x2b8 ./startup/startup_mimxrt1062.o
                0x60002000                g_pfnVectors
                0x60002000                __Vectors
                0x600022b8                . = ALIGN (0x4)
                0x600022b8                __section_table_start = .
                0x600022b8                __data_section_table = .
                0x600022b8        0x4 LONG 0x6007d9c4 LOADADDR (.data)
                0x600022bc        0x4 LONG 0x20200000 ADDR (.data)
                0x600022c0        0x4 LONG 0x1bf8 SIZEOF (.data)
                0x600022c4        0x4 LONG 0x6007d9c4 LOADADDR (.data_RAM2)
                0x600022c8        0x4 LONG 0x20000000 ADDR (.data_RAM2)
                0x600022cc        0x4 LONG 0x0 SIZEOF (.data_RAM2)
                0x600022d0        0x4 LONG 0x6007d9c4 LOADADDR (.data_RAM3)
                0x600022d4        0x4 LONG 0x0 ADDR (.data_RAM3)
                0x600022d8        0x4 LONG 0x0 SIZEOF (.data_RAM3)
                0x600022dc        0x4 LONG 0x6007d9c4 LOADADDR (.data_RAM4)
                0x600022e0        0x4 LONG 0x80000000 ADDR (.data_RAM4)
                0x600022e4        0x4 LONG 0x0 SIZEOF (.data_RAM4)
                0x600022e8        0x4 LONG 0x6007d9c4 LOADADDR (.data_RAM5)
                0x600022ec        0x4 LONG 0x81e00000 ADDR (.data_RAM5)
                0x600022f0        0x4 LONG 0x0 SIZEOF (.data_RAM5)
                0x600022f4                __data_section_table_end = .
                0x600022f4                __bss_section_table = .
                0x600022f4        0x4 LONG 0x20201c00 ADDR (.bss)
                0x600022f8        0x4 LONG 0x25cc4 SIZEOF (.bss)
                0x600022fc        0x4 LONG 0x20000000 ADDR (.bss_RAM2)
                0x60002300        0x4 LONG 0xd8 SIZEOF (.bss_RAM2)
                0x60002304        0x4 LONG 0x0 ADDR (.bss_RAM3)
                0x60002308        0x4 LONG 0x0 SIZEOF (.bss_RAM3)
                0x6000230c        0x4 LONG 0x80000000 ADDR (.bss_RAM4)
                0x60002310        0x4 LONG 0x0 SIZEOF (.bss_RAM4)
                0x60002314        0x4 LONG 0x81e00000 ADDR (.bss_RAM5)
                0x60002318        0x4 LONG 0x0 SIZEOF (.bss_RAM5)
                0x6000231c                __bss_section_table_end = .
                0x6000231c                __section_table_end = .
 *(SORT_BY_ALIGNMENT(.after_vectors*))
 .after_vectors.reset
                0x6000231c       0x4c ./startup/startup_mimxrt1062.o
                0x6000231c                ResetISR
 .after_vectors.init_data
                0x60002368       0x1e ./startup/startup_mimxrt1062.o
                0x60002368                data_init
 .after_vectors.init_bss
                0x60002386       0x12 ./startup/startup_mimxrt1062.o
                0x60002386                bss_init
 .after_vectors
                0x60002398        0xc ./startup/startup_mimxrt1062.o
                0x60002398                NMI_Handler
                0x600023a2                Reserved87_DriverIRQHandler
                0x600023a2                KPP_DriverIRQHandler
                0x600023a2                FLEXSPI2_DriverIRQHandler
                0x600023a2                LPSPI2_DriverIRQHandler
                0x600023a2                LCDIF_DriverIRQHandler
                0x600023a2                SAI3_RX_DriverIRQHandler
                0x600023a2                CCM_2_DriverIRQHandler
                0x600023a2                PIT_DriverIRQHandler
                0x600023a2                PMU_EVENT_DriverIRQHandler
                0x600023a2                PWM4_FAULT_DriverIRQHandler
                0x600023a2                DMA13_DMA29_DriverIRQHandler
                0x600023a2                FLEXRAM_DriverIRQHandler
                0x600023a2                LPSPI4_DriverIRQHandler
                0x600023a2                SEMC_DriverIRQHandler
                0x600023a2                SPDIF_DriverIRQHandler
                0x600023a2                PWM4_3_DriverIRQHandler
                0x600023a2                ACMP4_DriverIRQHandler
                0x600023a2                USB_PHY1_DriverIRQHandler
                0x600023a2                GPIO3_Combined_0_15_DriverIRQHandler
                0x600023a2                CAN3_DriverIRQHandler
                0x600023a2                Reserved171_DriverIRQHandler
                0x600023a2                DMA7_DMA23_DriverIRQHandler
                0x600023a2                BEE_DriverIRQHandler
                0x600023a2                GPR_IRQ_DriverIRQHandler
                0x600023a2                PWM2_FAULT_DriverIRQHandler
                0x600023a2                PWM3_1_DriverIRQHandler
                0x600023a2                DMA14_DMA30_DriverIRQHandler
                0x600023a2                TMR1_DriverIRQHandler
                0x600023a2                TRNG_DriverIRQHandler
                0x600023a2                PWM3_2_DriverIRQHandler
                0x600023a2                ENET_1588_Timer_DriverIRQHandler
                0x600023a2                GPIO2_Combined_16_31_DriverIRQHandler
                0x600023a2                Reserved143_DriverIRQHandler
                0x600023a2                PWM4_1_DriverIRQHandler
                0x600023a2                PWM3_3_DriverIRQHandler
                0x600023a2                DMA0_DMA16_DriverIRQHandler
                0x600023a2                IntDefaultHandler
                0x600023a2                DMA2_DMA18_DriverIRQHandler
                0x600023a2                SRC_DriverIRQHandler
                0x600023a2                GPIO1_INT4_DriverIRQHandler
                0x600023a2                Reserved144_DriverIRQHandler
                0x600023a2                USDHC1_DriverIRQHandler
                0x600023a2                ENC3_DriverIRQHandler
                0x600023a2                PWM3_FAULT_DriverIRQHandler
                0x600023a2                EWM_DriverIRQHandler
                0x600023a2                TSC_DIG_DriverIRQHandler
                0x600023a2                WDOG1_DriverIRQHandler
                0x600023a2                Reserved78_DriverIRQHandler
                0x600023a2                TMR4_DriverIRQHandler
                0x600023a2                ENC2_DriverIRQHandler
                0x600023a2                ADC_ETC_IRQ2_DriverIRQHandler
                0x600023a2                GPIO1_Combined_16_31_DriverIRQHandler
                0x600023a2                GPIO1_INT7_DriverIRQHandler
                0x600023a2                SAI1_DriverIRQHandler
                0x600023a2                DCDC_DriverIRQHandler
                0x600023a2                DMA12_DMA28_DriverIRQHandler
                0x600023a2                PWM4_0_DriverIRQHandler
                0x600023a2                ADC_ETC_ERROR_IRQ_DriverIRQHandler
                0x600023a2                ACMP2_DriverIRQHandler
                0x600023a2                GPIO5_Combined_0_15_DriverIRQHandler
                0x600023a2                GPIO1_INT0_DriverIRQHandler
                0x600023a2                GPIO1_INT2_DriverIRQHandler
                0x600023a2                RTWDOG_DriverIRQHandler
                0x600023a2                FLEXSPI_DriverIRQHandler
                0x600023a2                GPT2_DriverIRQHandler
                0x600023a2                USB_PHY2_DriverIRQHandler
                0x600023a2                DMA10_DMA26_DriverIRQHandler
                0x600023a2                PWM2_1_DriverIRQHandler
                0x600023a2                PWM1_1_DriverIRQHandler
                0x600023a2                PXP_DriverIRQHandler
                0x600023a2                ADC1_DriverIRQHandler
                0x600023a2                PWM1_0_DriverIRQHandler
                0x600023a2                SJC_DriverIRQHandler
                0x600023a2                DMA1_DMA17_DriverIRQHandler
                0x600023a2                ENC1_DriverIRQHandler
                0x600023a2                ENC4_DriverIRQHandler
                0x600023a2                CAN2_DriverIRQHandler
                0x600023a2                DCP_DriverIRQHandler
                0x600023a2                CTI0_ERROR_DriverIRQHandler
                0x600023a2                DMA8_DMA24_DriverIRQHandler
                0x600023a2                GPT1_DriverIRQHandler
                0x600023a2                ACMP3_DriverIRQHandler
                0x600023a2                DMA6_DMA22_DriverIRQHandler
                0x600023a2                CSU_DriverIRQHandler
                0x600023a2                GPIO1_INT5_DriverIRQHandler
                0x600023a2                TMR3_DriverIRQHandler
                0x600023a2                TMR2_DriverIRQHandler
                0x600023a2                CTI1_ERROR_DriverIRQHandler
                0x600023a2                GPIO1_Combined_0_15_DriverIRQHandler
                0x600023a2                USDHC2_DriverIRQHandler
                0x600023a2                PWM4_2_DriverIRQHandler
                0x600023a2                SAI2_DriverIRQHandler
                0x600023a2                CORE_DriverIRQHandler
                0x600023a2                DMA11_DMA27_DriverIRQHandler
                0x600023a2                CSI_DriverIRQHandler
                0x600023a2                PWM2_3_DriverIRQHandler
                0x600023a2                XBAR1_IRQ_2_3_DriverIRQHandler
                0x600023a2                SNVS_HP_WRAPPER_TZ_DriverIRQHandler
                0x600023a2                GPIO3_Combined_16_31_DriverIRQHandler
                0x600023a2                PWM1_FAULT_DriverIRQHandler
                0x600023a2                ENET2_1588_Timer_DriverIRQHandler
                0x600023a2                PWM2_2_DriverIRQHandler
                0x600023a2                DMA4_DMA20_DriverIRQHandler
                0x600023a2                DMA9_DMA25_DriverIRQHandler
                0x600023a2                SNVS_HP_WRAPPER_DriverIRQHandler
                0x600023a2                XBAR1_IRQ_0_1_DriverIRQHandler
                0x600023a2                ADC_ETC_IRQ1_DriverIRQHandler
                0x600023a2                LPSPI1_DriverIRQHandler
                0x600023a2                DMA3_DMA19_DriverIRQHandler
                0x600023a2                GPIO1_INT3_DriverIRQHandler
                0x600023a2                DCP_VMI_DriverIRQHandler
                0x600023a2                GPC_DriverIRQHandler
                0x600023a2                GPIO2_Combined_0_15_DriverIRQHandler
                0x600023a2                PWM1_2_DriverIRQHandler
                0x600023a2                USB_OTG1_DriverIRQHandler
                0x600023a2                TEMP_LOW_HIGH_DriverIRQHandler
                0x600023a2                SAI3_TX_DriverIRQHandler
                0x600023a2                WDOG2_DriverIRQHandler
                0x600023a2                Reserved68_DriverIRQHandler
                0x600023a2                PWM3_0_DriverIRQHandler
                0x600023a2                GPIO4_Combined_0_15_DriverIRQHandler
                0x600023a2                GPIO4_Combined_16_31_DriverIRQHandler
                0x600023a2                GPIO6_7_8_9_DriverIRQHandler
                0x600023a2                GPIO5_Combined_16_31_DriverIRQHandler
                0x600023a2                DMA5_DMA21_DriverIRQHandler
                0x600023a2                CCM_1_DriverIRQHandler
                0x600023a2                ADC2_DriverIRQHandler
                0x600023a2                Reserved115_DriverIRQHandler
                0x600023a2                TEMP_PANIC_DriverIRQHandler
                0x600023a2                DMA15_DMA31_DriverIRQHandler
                0x600023a2                LPSPI3_DriverIRQHandler
                0x600023a2                PWM1_3_DriverIRQHandler
                0x600023a2                ACMP1_DriverIRQHandler
                0x600023a2                Reserved86_DriverIRQHandler
                0x600023a2                DMA_ERROR_DriverIRQHandler
                0x600023a2                ADC_ETC_IRQ0_DriverIRQHandler
                0x600023a2                CAN1_DriverIRQHandler
                0x600023a2                GPIO1_INT6_DriverIRQHandler
                0x600023a2                GPIO1_INT1_DriverIRQHandler
                0x600023a2                PWM2_0_DriverIRQHandler
                0x600023a2                SNVS_LP_WRAPPER_DriverIRQHandler
                0x600023a2                USB_OTG2_DriverIRQHandler
 *(SORT_BY_ALIGNMENT(.text*))
 *fill*         0x600023a4       0x1c ff
 .text          0x600023c0       0xdc d:/programfiles/nxp/mcuxpressoide_11.1.0_3209/ide/plugins/com.nxp.mcuxpresso.tools.win32_11.1.0.201909161352/tools/bin/../lib/gcc/arm-none-eabi/8.3.1/../../../../arm-none-eabi/lib/thumb/v7e-m+fp/hard\libc.a(lib_a-strlen.o)
                0x600023c0                strlen
 *fill*         0x6000249c        0x4 ff
 .text          0x600024a0      0x2dc d:/programfiles/nxp/mcuxpressoide_11.1.0_3209/ide/plugins/com.nxp.mcuxpresso.tools.win32_11.1.0.201909161352/tools/bin/../lib/gcc/arm-none-eabi/8.3.1/../../../../arm-none-eabi/lib/thumb/v7e-m+fp/hard\libc.a(lib_a-strcmp.o)
                0x600024a8                strcmp
 *fill*         0x6000277c        0x4 ff
 .text.SVC_Handler
                0x60002780       0x28 ./amazon-freertos/freertos_kernel/portable/GCC/ARM_CM4F/port.o
                0x60002780                SVC_Handler
 *fill*         0x600027a8        0x8 ff
 .text.PendSV_Handler
                0x600027b0       0x68 ./amazon-freertos/freertos_kernel/portable/GCC/ARM_CM4F/port.o
                0x600027b0                PendSV_Handler
 *fill*         0x60002818        0x8 ff
 .text          0x60002820       0xa0 d:/programfiles/nxp/mcuxpressoide_11.1.0_3209/ide/plugins/com.nxp.mcuxpresso.tools.win32_11.1.0.201909161352/tools/bin/../lib/gcc/arm-none-eabi/8.3.1/../../../../arm-none-eabi/lib/thumb/v7e-m+fp/hard\libc.a(lib_a-memchr.o)
                0x60002820                memchr
 .text.UA_DateTime_fromUnixTime
                0x600028c0       0x54 ./source/commands.o
 *fill*         0x60002914        0x4 ff
 .text.UA_DateTime_fromUnixTime
                0x60002918       0x54 ./source/main_MandC.o
 *fill*         0x6000296c        0x4 ff
 .text.UA_DateTime_toStruct
                0x60002970      0x234 ./open62541/open62541.o
                0x60002970                UA_DateTime_toStruct
 *fill*         0x60002ba4        0x4 ff
 .text.UA_Timer_addRepeatedCallback
                0x60002ba8       0x94 ./open62541/open62541.o
                0x60002ba8                UA_Timer_addRepeatedCallback
 *fill*         0x60002c3c        0x4 ff
 .text.checkPreviousToken
                0x60002c40       0x84 ./open62541/open62541.o
 *fill*         0x60002cc4        0x4 ff
 .text.UA_Session_updateLifetime
                0x60002cc8       0x50 ./open62541/open62541.o
                0x60002cc8                UA_Session_updateLifetime
 .text.UA_Server_init
                0x60002d18      0x144 ./open62541/open62541.o
 *fill*         0x60002e5c        0x4 ff
 .text.setServerShutdown
                0x60002e60       0x94 ./open62541/open62541.o
 *fill*         0x60002ef4        0x4 ff
 .text.__secs_to_tm
                0x60002ef8      0x308 ./open62541/open62541.o
                0x60002ef8                __secs_to_tm
 .text.outOfPercentDeadBand
                0x60003200      0x7f8 ./open62541/open62541.o
 .text.UA_Log_Stdout_log
                0x600039f8       0xdc ./open62541/open62541.o
                0x600039f8                UA_Log_Stdout_log
 *fill*         0x60003ad4        0x4 ff
 .text.setDefaultConfig
                0x60003ad8      0x2b4 ./open62541/open62541.o
 *fill*         0x60003d8c        0x4 ff
 .text.ServerNetworkLayerTCP_listen
                0x60003d90      0x314 ./open62541/open62541.o
 *fill*         0x600040a4        0x4 ff
 .text._svfprintf_r
                0x600040a8     0x19f8 d:/programfiles/nxp/mcuxpressoide_11.1.0_3209/ide/plugins/com.nxp.mcuxpresso.tools.win32_11.1.0.201909161352/tools/bin/../lib/gcc/arm-none-eabi/8.3.1/../../../../arm-none-eabi/lib/thumb/v7e-m+fp/hard\libc.a(lib_a-svfprintf.o)
                0x600040a8                _svfprintf_r
 .text._vfprintf_r
                0x60005aa0     0x1adc d:/programfiles/nxp/mcuxpressoide_11.1.0_3209/ide/plugins/com.nxp.mcuxpresso.tools.win32_11.1.0.201909161352/tools/bin/../lib/gcc/arm-none-eabi/8.3.1/../../../../arm-none-eabi/lib/thumb/v7e-m+fp/hard\libc.a(lib_a-vfprintf.o)
                0x60005aa0                _vfprintf_r
 *fill*         0x6000757c        0x4 ff
 .text._dtoa_r  0x60007580      0xe54 d:/programfiles/nxp/mcuxpressoide_11.1.0_3209/ide/plugins/com.nxp.mcuxpresso.tools.win32_11.1.0.201909161352/tools/bin/../lib/gcc/arm-none-eabi/8.3.1/../../../../arm-none-eabi/lib/thumb/v7e-m+fp/hard\libc.a(lib_a-dtoa.o)
                0x60007580                _dtoa_r
 *fill*         0x600083d4        0x4 ff
 .text.pow      0x600083d8      0x19c d:/programfiles/nxp/mcuxpressoide_11.1.0_3209/ide/plugins/com.nxp.mcuxpresso.tools.win32_11.1.0.201909161352/tools/bin/../lib/gcc/arm-none-eabi/8.3.1/../../../../arm-none-eabi/lib/thumb/v7e-m+fp/hard\libm.a(lib_a-w_pow.o)
                0x600083d8                pow
 *fill*         0x60008574        0x4 ff
 .text.__ieee754_pow
                0x60008578      0xad8 d:/programfiles/nxp/mcuxpressoide_11.1.0_3209/ide/plugins/com.nxp.mcuxpresso.tools.win32_11.1.0.201909161352/tools/bin/../lib/gcc/arm-none-eabi/8.3.1/../../../../arm-none-eabi/lib/thumb/v7e-m+fp/hard\libm.a(lib_a-e_pow.o)
                0x60008578                __ieee754_pow
 .text.nan      0x60009050       0x10 d:/programfiles/nxp/mcuxpressoide_11.1.0_3209/ide/plugins/com.nxp.mcuxpresso.tools.win32_11.1.0.201909161352/tools/bin/../lib/gcc/arm-none-eabi/8.3.1/../../../../arm-none-eabi/lib/thumb/v7e-m+fp/hard\libm.a(lib_a-s_nan.o)
                0x60009050                nan
 .text.scalbn   0x60009060      0x124 d:/programfiles/nxp/mcuxpressoide_11.1.0_3209/ide/plugins/com.nxp.mcuxpresso.tools.win32_11.1.0.201909161352/tools/bin/../lib/gcc/arm-none-eabi/8.3.1/../../../../arm-none-eabi/lib/thumb/v7e-m+fp/hard\libm.a(lib_a-s_scalbn.o)
                0x60009060                scalbn
 .text.__assert_func
                0x60009184       0x28 ./utilities/fsl_assert.o
                0x60009184                __assert_func
 .text._ZN16monitored_device14device_readoutEP18_lpi2c_rtos_handlePf
                0x600091ac       0x20 ./source/Devices.o
                0x600091ac                monitored_device::device_readout(_lpi2c_rtos_handle*, float*)
 .text._ZN12pmbus_sensor15get_measurementEP18_lpi2c_rtos_handletRf
                0x600091cc      0x12c ./source/Devices.o
                0x600091cc                pmbus_sensor::get_measurement(_lpi2c_rtos_handle*, unsigned short, float&)
 .text._ZN16monitored_deviceC2EhNSt7__cxx1112basic_stringIcSt11char_traitsIcESaIcEEEh
                0x600092f8       0x4c ./source/Devices.o
                0x600092f8                monitored_device::monitored_device(unsigned char, std::__cxx11::basic_string<char, std::char_traits<char>, std::allocator<char> >, unsigned char)
                0x600092f8                monitored_device::monitored_device(unsigned char, std::__cxx11::basic_string<char, std::char_traits<char>, std::allocator<char> >, unsigned char)
 .text._ZN12pmbus_deviceC2EhNSt7__cxx1112basic_stringIcSt11char_traitsIcESaIcEEEPP12pmbus_sensor
                0x60009344       0x50 ./source/Devices.o
                0x60009344                pmbus_device::pmbus_device(unsigned char, std::__cxx11::basic_string<char, std::char_traits<char>, std::allocator<char> >, pmbus_sensor**)
                0x60009344                pmbus_device::pmbus_device(unsigned char, std::__cxx11::basic_string<char, std::char_traits<char>, std::allocator<char> >, pmbus_sensor**)
 .text._ZN6deviceC2Eh11device_typeNSt7__cxx1112basic_stringIcSt11char_traitsIcESaIcEEE
                0x60009394       0x48 ./source/Devices.o
                0x60009394                device::device(unsigned char, device_type, std::__cxx11::basic_string<char, std::char_traits<char>, std::allocator<char> >)
                0x60009394                device::device(unsigned char, device_type, std::__cxx11::basic_string<char, std::char_traits<char>, std::allocator<char> >)
 .text._ZN10I2C_switchC2EhNSt7__cxx1112basic_stringIcSt11char_traitsIcESaIcEEEh
                0x600093dc       0x5c ./source/Devices.o
                0x600093dc                I2C_switch::I2C_switch(unsigned char, std::__cxx11::basic_string<char, std::char_traits<char>, std::allocator<char> >, unsigned char)
                0x600093dc                I2C_switch::I2C_switch(unsigned char, std::__cxx11::basic_string<char, std::char_traits<char>, std::allocator<char> >, unsigned char)
 .text._ZN10I2C_switch11set_channelEP18_lpi2c_rtos_handleh
                0x60009438       0x6c ./source/Devices.o
                0x60009438                I2C_switch::set_channel(_lpi2c_rtos_handle*, unsigned char)
 .text._ZN10I2C_switch7set_offEP18_lpi2c_rtos_handle
                0x600094a4       0x44 ./source/Devices.o
                0x600094a4                I2C_switch::set_off(_lpi2c_rtos_handle*)
 .text._ZN11IO_ExpanderC2EhNSt7__cxx1112basic_stringIcSt11char_traitsIcESaIcEEE
                0x600094e8       0x48 ./source/Devices.o
                0x600094e8                IO_Expander::IO_Expander(unsigned char, std::__cxx11::basic_string<char, std::char_traits<char>, std::allocator<char> >)
                0x600094e8                IO_Expander::IO_Expander(unsigned char, std::__cxx11::basic_string<char, std::char_traits<char>, std::allocator<char> >)
 .text._ZN11IO_Expander9IO_configEP18_lpi2c_rtos_handlet
                0x60009530       0x40 ./source/Devices.o
                0x60009530                IO_Expander::IO_config(_lpi2c_rtos_handle*, unsigned short)
 .text.UA_Server_writeValue
                0x60009570       0x3c ./source/commands.o
 .text.UA_Server_addVariableNode
                0x600095ac       0x6c ./source/commands.o
 .text.UA_Server_addObjectNode
                0x60009618       0x6c ./source/commands.o
 .text.UA_Server_addMethodNode
                0x60009684       0xd0 ./source/commands.o
 .text._Z7test_pbv
                0x60009754       0x14 ./source/commands.o
                0x60009754                test_pb()
 .text._Z16UA_readable_timex
                0x60009768       0x84 ./source/commands.o
                0x60009768                UA_readable_time(long long)
 .text._ZN11cmd_handler14check_commandsEv
                0x600097ec       0x9c ./source/commands.o
                0x600097ec                cmd_handler::check_commands()
 .text._ZN11cmd_handler17new_deadline_unixEP9UA_ServerPK9UA_NodeIdPvS4_S5_S4_S5_jPK10UA_VariantjPS6_
                0x60009888      0x130 ./source/commands.o
                0x60009888                cmd_handler::new_deadline_unix(UA_Server*, UA_NodeId const*, void*, UA_NodeId const*, void*, UA_NodeId const*, void*, unsigned int, UA_Variant const*, unsigned int, UA_Variant*)
 .text._ZN11cmd_handler16cmd_handler_taskEv
                0x600099b8      0x184 ./source/commands.o
                0x600099b8                cmd_handler::cmd_handler_task()
 .text._ZN6deviceD2Ev
                0x60009b3c       0x28 ./source/commands.o
                0x60009b3c                device::~device()
                0x60009b3c                device::~device()
 .text._ZN10I2C_switchD2Ev
                0x60009b64       0x24 ./source/commands.o
                0x60009b64                I2C_switch::~I2C_switch()
                0x60009b64                I2C_switch::~I2C_switch()
 .text._ZN11cmd_handlerC2EP9UA_ServerhPP18_lpi2c_rtos_handle
                0x60009b88      0x1fc ./source/commands.o
                0x60009b88                cmd_handler::cmd_handler(UA_Server*, unsigned char, _lpi2c_rtos_handle**)
                0x60009b88                cmd_handler::cmd_handler(UA_Server*, unsigned char, _lpi2c_rtos_handle**)
 .text._ZN11cmd_handler14get_RCU_configE10I2C_config
                0x60009d84      0x198 ./source/commands.o
                0x60009d84                cmd_handler::get_RCU_config(I2C_config)
 .text._ZN11cmd_handler16init_OPCua_stuffEv
                0x60009f1c      0x514 ./source/commands.o
                0x60009f1c                cmd_handler::init_OPCua_stuff()
 .text._ZN3RCUC2EP10I2C_configP11cmd_handlerh
                0x6000a430      0x278 ./source/commands.o
                0x6000a430                RCU::RCU(I2C_config*, cmd_handler*, unsigned char)
                0x6000a430                RCU::RCU(I2C_config*, cmd_handler*, unsigned char)
 .text._ZN3RCU18variable_decode_pbEP12pb_istream_sPK15pb_field_iter_sPPv
                0x6000a6a8      0x24c ./source/commands.o
                0x6000a6a8                RCU::variable_decode_pb(pb_istream_s*, pb_field_iter_s const*, void**)
 .text._ZN3RCU14mode_decode_pbEP12pb_istream_sPK15pb_field_iter_sPPv
                0x6000a8f4       0x58 ./source/commands.o
                0x6000a8f4                RCU::mode_decode_pb(pb_istream_s*, pb_field_iter_s const*, void**)
 .text._ZN3RCU13spi_decode_pbEP12pb_istream_sPK15pb_field_iter_sPPv
                0x6000a94c       0x60 ./source/commands.o
                0x6000a94c                RCU::spi_decode_pb(pb_istream_s*, pb_field_iter_s const*, void**)
 .text._ZN3RCU15input_decode_pbEP12pb_istream_sPK15pb_field_iter_sPPv
                0x6000a9ac       0x6c ./source/commands.o
                0x6000a9ac                RCU::input_decode_pb(pb_istream_s*, pb_field_iter_s const*, void**)
 .text._ZN3RCU16device_decode_pbEP12pb_istream_sPK15pb_field_iter_sPPv
                0x6000aa18       0x74 ./source/commands.o
                0x6000aa18                RCU::device_decode_pb(pb_istream_s*, pb_field_iter_s const*, void**)
 .text._ZN11cmd_handler15process_RCU_cmdEP3cmd
                0x6000aa8c      0x194 ./source/commands.o
                0x6000aa8c                cmd_handler::process_RCU_cmd(cmd*)
 .text._ZN3RCU15compose_commandEP3cmdh
                0x6000ac20      0x18c ./source/commands.o
                0x6000ac20                RCU::compose_command(cmd*, unsigned char)
 .text._ZN11cmd_handler7RCU_cmdEP9UA_ServerPK9UA_NodeIdPvS4_S5_S4_S5_jPK10UA_VariantjPS6_
                0x6000adac       0x98 ./source/commands.o
                0x6000adac                cmd_handler::RCU_cmd(UA_Server*, UA_NodeId const*, void*, UA_NodeId const*, void*, UA_NodeId const*, void*, unsigned int, UA_Variant const*, unsigned int, UA_Variant*)
 .text._ZN11cmd_handler21set_RCU_read_intervalEP9UA_ServerPK9UA_NodeIdPvS4_S5_S4_S5_jPK10UA_VariantjPS6_
                0x6000ae44       0x28 ./source/commands.o
                0x6000ae44                cmd_handler::set_RCU_read_interval(UA_Server*, UA_NodeId const*, void*, UA_NodeId const*, void*, UA_NodeId const*, void*, unsigned int, UA_Variant const*, unsigned int, UA_Variant*)
 .text._ZN11cmd_handler15flush_cmd_queueEP9UA_ServerPK9UA_NodeIdPvS4_S5_S4_S5_jPK10UA_VariantjPS6_
                0x6000ae6c       0x30 ./source/commands.o
                0x6000ae6c                cmd_handler::flush_cmd_queue(UA_Server*, UA_NodeId const*, void*, UA_NodeId const*, void*, UA_NodeId const*, void*, unsigned int, UA_Variant const*, unsigned int, UA_Variant*)
 .text._ZN11cmd_handler14add_OPCua_funcEv
                0x6000ae9c      0x838 ./source/commands.o
                0x6000ae9c                cmd_handler::add_OPCua_func()
 .text.I2C_reset
                0x6000b6d4       0x80 ./source/common.o
                0x6000b6d4                I2C_reset
 .text.__NVIC_SetPriority
                0x6000b754       0x5c ./source/main_MandC.o
 .text.CLOCK_SetMux
                0x6000b7b0       0xb8 ./source/main_MandC.o
 .text.CLOCK_SetDiv
                0x6000b868       0xb8 ./source/main_MandC.o
 .text.UA_Server_writeValue
                0x6000b920       0x3c ./source/main_MandC.o
 .text.UA_Server_addVariableNode
                0x6000b95c       0x6c ./source/main_MandC.o
 .text.UA_Server_addObjectNode
                0x6000b9c8       0x6c ./source/main_MandC.o
 .text.UA_Server_addMethodNode
                0x6000ba34       0xd0 ./source/main_MandC.o
 .text.IOMUXC_EnableMode
                0x6000bb04       0x48 ./source/main_MandC.o
 .text.debug_msg_buff_init
                0x6000bb4c      0x2a4 ./source/main_MandC.o
 .text._Z24add_OPC_ua_offset_methodP9UA_Server
                0x6000bdf0      0x18c ./source/main_MandC.o
                0x6000bdf0                add_OPC_ua_offset_method(UA_Server*)
 .text._Z14get_ip_addressv
                0x6000bf7c       0x30 ./source/main_MandC.o
                0x6000bf7c                get_ip_address()
 .text._Z23set_get_cmd_handler_ptrP11cmd_handler
                0x6000bfac       0x2c ./source/main_MandC.o
                0x6000bfac                set_get_cmd_handler_ptr(cmd_handler*)
 .text._Z14BOARD_InitSEMCv
                0x6000bfd8       0xfc ./source/main_MandC.o
                0x6000bfd8                BOARD_InitSEMC()
 .text._Z5delayv
                0x6000c0d4       0x3c ./source/main_MandC.o
                0x6000c0d4                delay()
 .text._Z14RTOS_heap_initv
                0x6000c110       0x2c ./source/main_MandC.o
                0x6000c110                RTOS_heap_init()
 .text._Z25BOARD_Init_ETH_peripheralv
                0x6000c13c       0x84 ./source/main_MandC.o
                0x6000c13c                BOARD_Init_ETH_peripheral()
 .text._Z20get_readable_runtimev
                0x6000c1c0       0xf0 ./source/main_MandC.o
                0x6000c1c0                get_readable_runtime()
 .text.vApplicationMallocFailedHook
                0x6000c2b0       0x1c ./source/main_MandC.o
                0x6000c2b0                vApplicationMallocFailedHook
 .text.vApplicationStackOverflowHook
                0x6000c2cc       0x34 ./source/main_MandC.o
                0x6000c2cc                vApplicationStackOverflowHook
 .text._Z16WDOG_reset_causev
                0x6000c300       0x64 ./source/main_MandC.o
                0x6000c300                WDOG_reset_cause()
 .text._ZN16WDOG_sys_manager15WDOG_thread_addEv
                0x6000c364       0x60 ./source/main_MandC.o
                0x6000c364                WDOG_sys_manager::WDOG_thread_add()
 .text._ZN16WDOG_sys_manager17WDOG_task_refreshEh
                0x6000c3c4       0x44 ./source/main_MandC.o
                0x6000c3c4                WDOG_sys_manager::WDOG_task_refresh(unsigned char)
 .text._Z6blinkyv
                0x6000c408       0x2c ./source/main_MandC.o
                0x6000c408                blinky()
 .text._ZN14TEST_base_nodeC2EP18_lpi2c_rtos_handleP9UA_ServerhP15QueueDefinitionNSt7__cxx1112basic_stringIcSt11char_traitsIcESaIcEEE
                0x6000c434      0xfb4 ./source/main_MandC.o
                0x6000c434                TEST_base_node::TEST_base_node(_lpi2c_rtos_handle*, UA_Server*, unsigned char, QueueDefinition*, std::__cxx11::basic_string<char, std::char_traits<char>, std::allocator<char> >)
                0x6000c434                TEST_base_node::TEST_base_node(_lpi2c_rtos_handle*, UA_Server*, unsigned char, QueueDefinition*, std::__cxx11::basic_string<char, std::char_traits<char>, std::allocator<char> >)
 .text.main     0x6000d3e8       0xa0 ./source/main_MandC.o
                0x6000d3e8                main
 .text._ZL9lwip_initPv
                0x6000d488      0x218 ./source/main_MandC.o
 .text._ZL12opcua_threadPv
                0x6000d6a0      0x100 ./source/main_MandC.o
 .text._ZL21server_manager_threadPv
                0x6000d7a0      0x130 ./source/main_MandC.o
 .text._ZL18I2C_3_manager_taskPv
                0x6000d8d0      0x154 ./source/main_MandC.o
 .text._ZL11status_nodeP9UA_Server
                0x6000da24      0x870 ./source/main_MandC.o
 .text._ZNSt7__cxx119to_stringEi
                0x6000e294       0x2c ./source/node.o
                0x6000e294                std::__cxx11::to_string(int)
 .text.UA_NodeId_clear
                0x6000e2c0       0x1c ./source/node.o
 .text.UA_QualifiedName_clear
                0x6000e2dc       0x1c ./source/node.o
 .text.UA_LocalizedText_clear
                0x6000e2f8       0x1c ./source/node.o
 .text.UA_ObjectAttributes_clear
                0x6000e314       0x1c ./source/node.o
 .text.UA_VariableAttributes_clear
                0x6000e330       0x1c ./source/node.o
 .text.UA_Server_writeValue
                0x6000e34c       0x3c ./source/node.o
 .text.UA_Server_addVariableNode
                0x6000e388       0x6c ./source/node.o
 .text.UA_Server_addObjectNode
                0x6000e3f4       0x6c ./source/node.o
 .text._ZN4node9add_OPCuaEP9UA_Server9UA_NodeId
                0x6000e460      0x744 ./source/node.o
                0x6000e460                node::add_OPCua(UA_Server*, UA_NodeId)
 .text._ZN4node12update_OPCuaEP9UA_ServerRtf
                0x6000eba4       0x98 ./source/node.o
                0x6000eba4                node::update_OPCua(UA_Server*, unsigned short&, float)
 .text._ZN9base_node13update_bufferEv
                0x6000ec3c       0x68 ./source/node.o
                0x6000ec3c                base_node::update_buffer()
 .text._ZN9base_node15I2C_log_failureE14type_of_device
                0x6000eca4       0xc0 ./source/node.o
                0x6000eca4                base_node::I2C_log_failure(type_of_device)
 .text._ZN9base_node16process_I2C_logsEv
                0x6000ed64      0x1fc ./source/node.o
                0x6000ed64                base_node::process_I2C_logs()
 .text._ZN9base_node16I2C_monitor_initEv
                0x6000ef60      0x950 ./source/node.o
                0x6000ef60                base_node::I2C_monitor_init()
 .text._ZNSt7__cxx1112basic_stringIcSt11char_traitsIcESaIcEE12_M_constructIPcEEvT_S7_St20forward_iterator_tag
                0x6000f8b0       0x90 ./source/node.o
                0x6000f8b0                void std::__cxx11::basic_string<char, std::char_traits<char>, std::allocator<char> >::_M_construct<char*>(char*, char*, std::forward_iterator_tag)
 .text.UA_Boolean_new
                0x6000f940       0x14 ./open62541/open62541.o
 .text.UA_Byte_new
                0x6000f954       0x14 ./open62541/open62541.o
 .text.UA_Int32_new
                0x6000f968       0x14 ./open62541/open62541.o
 .text.UA_Int32_delete
                0x6000f97c       0x1c ./open62541/open62541.o
 .text.UA_UInt32_new
                0x6000f998       0x14 ./open62541/open62541.o
 .text.UA_String_new
                0x6000f9ac       0x14 ./open62541/open62541.o
 .text.UA_String_copy
                0x6000f9c0       0x24 ./open62541/open62541.o
 .text.UA_String_deleteMembers
                0x6000f9e4       0x1c ./open62541/open62541.o
 .text.UA_String_clear
                0x6000fa00       0x1c ./open62541/open62541.o
 .text.UA_String_delete
                0x6000fa1c       0x1c ./open62541/open62541.o
 .text.UA_Guid_new
                0x6000fa38       0x14 ./open62541/open62541.o
 .text.UA_ByteString_new
                0x6000fa4c       0x14 ./open62541/open62541.o
 .text.UA_ByteString_copy
                0x6000fa60       0x24 ./open62541/open62541.o
 .text.UA_ByteString_deleteMembers
                0x6000fa84       0x1c ./open62541/open62541.o
 .text.UA_ByteString_delete
                0x6000faa0       0x1c ./open62541/open62541.o
 .text.UA_NodeId_copy
                0x6000fabc       0x24 ./open62541/open62541.o
 .text.UA_NodeId_deleteMembers
                0x6000fae0       0x1c ./open62541/open62541.o
 .text.UA_NodeId_clear
                0x6000fafc       0x1c ./open62541/open62541.o
 .text.UA_ExpandedNodeId_copy
                0x6000fb18       0x24 ./open62541/open62541.o
 .text.UA_ExpandedNodeId_deleteMembers
                0x6000fb3c       0x1c ./open62541/open62541.o
 .text.UA_QualifiedName_copy
                0x6000fb58       0x24 ./open62541/open62541.o
 .text.UA_QualifiedName_deleteMembers
                0x6000fb7c       0x1c ./open62541/open62541.o
 .text.UA_LocalizedText_copy
                0x6000fb98       0x24 ./open62541/open62541.o
 .text.UA_LocalizedText_deleteMembers
                0x6000fbbc       0x1c ./open62541/open62541.o
 .text.UA_DataValue_copy
                0x6000fbd8       0x24 ./open62541/open62541.o
 .text.UA_DataValue_deleteMembers
                0x6000fbfc       0x1c ./open62541/open62541.o
 .text.UA_Variant_new
                0x6000fc18       0x14 ./open62541/open62541.o
 .text.UA_Variant_copy
                0x6000fc2c       0x24 ./open62541/open62541.o
 .text.UA_Variant_deleteMembers
                0x6000fc50       0x1c ./open62541/open62541.o
 .text.UA_Variant_clear
                0x6000fc6c       0x1c ./open62541/open62541.o
 .text.UA_ApplicationDescription_copy
                0x6000fc88       0x24 ./open62541/open62541.o
 .text.UA_ApplicationDescription_deleteMembers
                0x6000fcac       0x1c ./open62541/open62541.o
 .text.UA_RequestHeader_deleteMembers
                0x6000fcc8       0x1c ./open62541/open62541.o
 .text.UA_EndpointDescription_copy
                0x6000fce4       0x24 ./open62541/open62541.o
 .text.UA_EndpointDescription_deleteMembers
                0x6000fd08       0x1c ./open62541/open62541.o
 .text.UA_RegisteredServer_copy
                0x6000fd24       0x24 ./open62541/open62541.o
 .text.UA_RegisteredServer_deleteMembers
                0x6000fd48       0x1c ./open62541/open62541.o
 .text.UA_OpenSecureChannelRequest_deleteMembers
                0x6000fd64       0x1c ./open62541/open62541.o
 .text.UA_OpenSecureChannelResponse_deleteMembers
                0x6000fd80       0x1c ./open62541/open62541.o
 .text.UA_BrowseDescription_copy
                0x6000fd9c       0x24 ./open62541/open62541.o
 .text.UA_BrowseDescription_deleteMembers
                0x6000fdc0       0x1c ./open62541/open62541.o
 .text.UA_ReferenceDescription_deleteMembers
                0x6000fddc       0x1c ./open62541/open62541.o
 .text.UA_ReferenceDescription_clear
                0x6000fdf8       0x1c ./open62541/open62541.o
 .text.UA_BrowseResult_deleteMembers
                0x6000fe14       0x1c ./open62541/open62541.o
 .text.UA_BrowsePathTarget_deleteMembers
                0x6000fe30       0x1c ./open62541/open62541.o
 .text.UA_BrowsePathResult_deleteMembers
                0x6000fe4c       0x1c ./open62541/open62541.o
 .text.UA_EventFilter_copy
                0x6000fe68       0x24 ./open62541/open62541.o
 .text.UA_EventFilter_clear
                0x6000fe8c       0x1c ./open62541/open62541.o
 .text.UA_NotificationMessage_copy
                0x6000fea8       0x24 ./open62541/open62541.o
 .text.UA_NotificationMessage_deleteMembers
                0x6000fecc       0x1c ./open62541/open62541.o
 .text.UA_EventFieldList_deleteMembers
                0x6000fee8       0x1c ./open62541/open62541.o
 .text.UA_StatusChangeNotification_new
                0x6000ff04       0x14 ./open62541/open62541.o
 .text.UA_PublishResponse_deleteMembers
                0x6000ff18       0x1c ./open62541/open62541.o
 .text.UA_BuildInfo_copy
                0x6000ff34       0x24 ./open62541/open62541.o
 .text.UA_BuildInfo_deleteMembers
                0x6000ff58       0x1c ./open62541/open62541.o
 .text.UA_ServerState_new
                0x6000ff74       0x14 ./open62541/open62541.o
 .text.UA_ServerStatusDataType_new
                0x6000ff88       0x14 ./open62541/open62541.o
 .text.UA_DataChangeNotification_new
                0x6000ff9c       0x14 ./open62541/open62541.o
 .text.UA_EventNotificationList_new
                0x6000ffb0       0x14 ./open62541/open62541.o
 .text.UA_Server_writeBrowseName
                0x6000ffc4       0x3c ./open62541/open62541.o
 .text.UA_Server_writeValue
                0x60010000       0x3c ./open62541/open62541.o
 .text.UA_Server_writeValueRank
                0x6001003c       0x3c ./open62541/open62541.o
 .text.UA_Server_writeAccessLevel
                0x60010078       0x3c ./open62541/open62541.o
 .text.UA_Server_addVariableNode
                0x600100b4       0x6c ./open62541/open62541.o
 .text.UA_Server_addVariableTypeNode
                0x60010120       0x6c ./open62541/open62541.o
 .text.UA_Server_addObjectNode
                0x6001018c       0x6c ./open62541/open62541.o
 .text.UA_Server_addObjectTypeNode
                0x600101f8       0x6c ./open62541/open62541.o
 .text.UA_Server_addReferenceTypeNode
                0x60010264       0x6c ./open62541/open62541.o
 .text.UA_UInt32_decodeBinary
                0x600102d0       0x2c ./open62541/open62541.o
 .text.UA_NodeId_decodeBinary
                0x600102fc       0x2c ./open62541/open62541.o
 .text.UA_RequestHeader_decodeBinary
                0x60010328       0x2c ./open62541/open62541.o
 .text.UA_OpenSecureChannelRequest_decodeBinary
                0x60010354       0x2c ./open62541/open62541.o
 .text.UA_AsymmetricAlgorithmSecurityHeader_deleteMembers
                0x60010380       0x1c ./open62541/open62541.o
 .text.UA_TcpMessageHeader_encodeBinary
                0x6001039c       0x30 ./open62541/open62541.o
 .text.UA_TcpMessageHeader_decodeBinary
                0x600103cc       0x2c ./open62541/open62541.o
 .text.UA_TcpHelloMessage_decodeBinary
                0x600103f8       0x2c ./open62541/open62541.o
 .text.UA_TcpAcknowledgeMessage_encodeBinary
                0x60010424       0x30 ./open62541/open62541.o
 .text.UA_TcpErrorMessage_encodeBinary
                0x60010454       0x30 ./open62541/open62541.o
 .text.UA_SecureConversationMessageHeader_decodeBinary
                0x60010484       0x2c ./open62541/open62541.o
 .text.UA_AsymmetricAlgorithmSecurityHeader_decodeBinary
                0x600104b0       0x2c ./open62541/open62541.o
 .text.UA_SymmetricAlgorithmSecurityHeader_decodeBinary
                0x600104dc       0x2c ./open62541/open62541.o
 .text.UA_SequenceHeader_decodeBinary
                0x60010508       0x2c ./open62541/open62541.o
 .text.UA_findDataType
                0x60010534       0x7c ./open62541/open62541.o
                0x60010534                UA_findDataType
 .text.UA_random_seed
                0x600105b0       0x2c ./open62541/open62541.o
                0x600105b0                UA_random_seed
 .text.UA_UInt32_random
                0x600105dc       0x14 ./open62541/open62541.o
                0x600105dc                UA_UInt32_random
 .text.String_copy
                0x600105f0       0x3c ./open62541/open62541.o
 .text.String_clear
                0x6001062c       0x28 ./open62541/open62541.o
 .text.UA_Guid_random
                0x60010654       0x90 ./open62541/open62541.o
                0x60010654                UA_Guid_random
 .text.UA_ByteString_allocBuffer
                0x600106e4       0x48 ./open62541/open62541.o
                0x600106e4                UA_ByteString_allocBuffer
 .text.NodeId_copy
                0x6001072c       0xbc ./open62541/open62541.o
 .text.UA_NodeId_isNull
                0x600107e8       0x94 ./open62541/open62541.o
                0x600107e8                UA_NodeId_isNull
 .text.UA_NodeId_order
                0x6001087c      0x19c ./open62541/open62541.o
                0x6001087c                UA_NodeId_order
 .text.fnv32    0x60010a18       0x4c ./open62541/open62541.o
 .text.UA_NodeId_hash
                0x60010a64       0x88 ./open62541/open62541.o
                0x60010a64                UA_NodeId_hash
 .text.ExtensionObject_copy
                0x60010aec       0xb4 ./open62541/open62541.o
 .text.Variant_copy
                0x60010ba0       0x90 ./open62541/open62541.o
 .text.UA_Variant_setScalarCopy
                0x60010c30       0x58 ./open62541/open62541.o
                0x60010c30                UA_Variant_setScalarCopy
 .text.computeStrides
                0x60010c88      0x26c ./open62541/open62541.o
 .text.isStringLike
                0x60010ef4       0x40 ./open62541/open62541.o
 .text.copySubString
                0x60010f34       0x90 ./open62541/open62541.o
 .text.UA_Variant_copyRange
                0x60010fc4      0x38c ./open62541/open62541.o
                0x60010fc4                UA_Variant_copyRange
 .text.Variant_setRange
                0x60011350      0x198 ./open62541/open62541.o
 .text.DiagnosticInfo_copy
                0x600114e8       0xbc ./open62541/open62541.o
 .text.copyStructure
                0x600115a4      0x164 ./open62541/open62541.o
 .text.copyNotImplemented
                0x60011708       0x20 ./open62541/open62541.o
 .text.UA_copy  0x60011728       0x54 ./open62541/open62541.o
                0x60011728                UA_copy
 .text.clearStructure
                0x6001177c       0xfc ./open62541/open62541.o
 .text.UA_clear
                0x60011878       0x3c ./open62541/open62541.o
                0x60011878                UA_clear
 .text.UA_delete
                0x600118b4       0x34 ./open62541/open62541.o
                0x600118b4                UA_delete
 .text.UA_Array_copy
                0x600118e8       0xfc ./open62541/open62541.o
                0x600118e8                UA_Array_copy
 .text.UA_DataType_isNumeric
                0x600119e4       0x44 ./open62541/open62541.o
                0x600119e4                UA_DataType_isNumeric
 .text.UA_NumericRange_parseFromString
                0x60011a28       0xe4 ./open62541/open62541.o
                0x60011a28                UA_NumericRange_parseFromString
 .text.exchangeBuffer
                0x60011b0c       0x34 ./open62541/open62541.o
 .text.encodeWithExchangeBuffer
                0x60011b40       0x90 ./open62541/open62541.o
 .text.Boolean_encodeBinary
                0x60011bd0       0x44 ./open62541/open62541.o
 .text.Boolean_decodeBinary
                0x60011c14       0x50 ./open62541/open62541.o
 .text.Byte_encodeBinary
                0x60011c64       0x44 ./open62541/open62541.o
 .text.Byte_decodeBinary
                0x60011ca8       0x44 ./open62541/open62541.o
 .text.UInt16_encodeBinary
                0x60011cec       0x44 ./open62541/open62541.o
 .text.UInt16_decodeBinary
                0x60011d30       0x44 ./open62541/open62541.o
 .text.UInt32_encodeBinary
                0x60011d74       0x44 ./open62541/open62541.o
 .text.UInt32_decodeBinary
                0x60011db8       0x44 ./open62541/open62541.o
 .text.UInt64_encodeBinary
                0x60011dfc       0x48 ./open62541/open62541.o
 .text.UInt64_decodeBinary
                0x60011e44       0x48 ./open62541/open62541.o
 .text.Array_encodeBinary
                0x60011e8c       0x94 ./open62541/open62541.o
 .text.Array_decodeBinary
                0x60011f20      0x17c ./open62541/open62541.o
 .text.String_encodeBinary
                0x6001209c       0x2c ./open62541/open62541.o
 .text.String_decodeBinary
                0x600120c8       0x28 ./open62541/open62541.o
 .text.Guid_encodeBinary
                0x600120f0       0x90 ./open62541/open62541.o
 .text.Guid_decodeBinary
                0x60012180       0x90 ./open62541/open62541.o
 .text.NodeId_encodeBinaryWithEncodingMask
                0x60012210      0x244 ./open62541/open62541.o
 .text.NodeId_decodeBinary
                0x60012454      0x1b0 ./open62541/open62541.o
 .text.ExpandedNodeId_encodeBinary
                0x60012604       0x90 ./open62541/open62541.o
 .text.ExpandedNodeId_decodeBinary
                0x60012694       0x84 ./open62541/open62541.o
 .text.UA_findDataTypeByBinaryInternal
                0x60012718       0xf4 ./open62541/open62541.o
 .text.ExtensionObject_encodeBinary
                0x6001280c      0x148 ./open62541/open62541.o
 .text.ExtensionObject_decodeBinaryContent
                0x60012954       0xa0 ./open62541/open62541.o
 .text.ExtensionObject_decodeBinary
                0x600129f4      0x110 ./open62541/open62541.o
 .text.Variant_encodeBinaryWrapExtensionObject
                0x60012b04       0xb8 ./open62541/open62541.o
 .text.Variant_encodeBinary
                0x60012bbc      0x1a0 ./open62541/open62541.o
 .text.Variant_decodeBinaryUnwrapExtensionObject
                0x60012d5c       0xf0 ./open62541/open62541.o
 .text.Variant_decodeBinary
                0x60012e4c      0x154 ./open62541/open62541.o
 .text.DataValue_encodeBinary
                0x60012fa0      0x1a8 ./open62541/open62541.o
 .text.DataValue_decodeBinary
                0x60013148      0x194 ./open62541/open62541.o
 .text.DiagnosticInfo_encodeBinary
                0x600132dc      0x1b0 ./open62541/open62541.o
 .text.DiagnosticInfo_decodeBinary
                0x6001348c      0x1a0 ./open62541/open62541.o
 .text.encodeBinaryStruct
                0x6001362c      0x114 ./open62541/open62541.o
 .text.encodeBinaryNotImplemented
                0x60013740       0x20 ./open62541/open62541.o
 .text.UA_encodeBinary
                0x60013760       0x5c ./open62541/open62541.o
                0x60013760                UA_encodeBinary
 .text.decodeBinaryNotImplemented
                0x600137bc       0x20 ./open62541/open62541.o
 .text.decodeBinaryStructure
                0x600137dc      0x128 ./open62541/open62541.o
 .text.UA_decodeBinary
                0x60013904       0x94 ./open62541/open62541.o
                0x60013904                UA_decodeBinary
 .text.Array_calcSizeBinary
                0x60013998       0x88 ./open62541/open62541.o
 .text.NodeId_calcSizeBinary
                0x60013a20       0xa4 ./open62541/open62541.o
 .text.ExtensionObject_calcSizeBinary
                0x60013ac4       0xd0 ./open62541/open62541.o
 .text.Variant_calcSizeBinary
                0x60013b94      0x144 ./open62541/open62541.o
 .text.calcSizeBinaryStructure
                0x60013cd8      0x108 ./open62541/open62541.o
 .text.UA_calcSizeBinary
                0x60013de0       0x30 ./open62541/open62541.o
                0x60013de0                UA_calcSizeBinary
 .text.UA_StatusCode_name
                0x60013e10       0x54 ./open62541/open62541.o
                0x60013e10                UA_StatusCode_name
 .text.UA_readNumberWithBase
                0x60013e64       0xfc ./open62541/open62541.o
                0x60013e64                UA_readNumberWithBase
 .text.UA_ByteString_toBase64String
                0x60013f60       0x7c ./open62541/open62541.o
                0x60013f60                UA_ByteString_toBase64String
 .text.UA_NodeId_toString
                0x60013fdc      0x308 ./open62541/open62541.o
                0x60013fdc                UA_NodeId_toString
 .text.addCallback
                0x600142e4       0xc8 ./open62541/open62541.o
 .text.UA_Timer_deleteMembers
                0x600143ac       0x28 ./open62541/open62541.o
                0x600143ac                UA_Timer_deleteMembers
 .text.UA_Connection_processHELACK
                0x600143d4       0x98 ./open62541/open62541.o
                0x600143d4                UA_Connection_processHELACK
 .text.hideErrors
                0x6001446c       0x48 ./open62541/open62541.o
 .text.UA_Connection_sendError
                0x600144b4       0x84 ./open62541/open62541.o
                0x600144b4                UA_Connection_sendError
 .text.bufferIncompleteChunk
                0x60014538       0x80 ./open62541/open62541.o
 .text.processChunk
                0x600145b8      0x134 ./open62541/open62541.o
 .text.UA_Connection_processChunks
                0x600146ec      0x128 ./open62541/open62541.o
                0x600146ec                UA_Connection_processChunks
 .text.UA_SecureChannel_setSecurityPolicy
                0x60014814       0xd8 ./open62541/open62541.o
                0x60014814                UA_SecureChannel_setSecurityPolicy
 .text.UA_SecureChannel_generateLocalNonce
                0x600148ec       0x6c ./open62541/open62541.o
                0x600148ec                UA_SecureChannel_generateLocalNonce
 .text.UA_SecureChannel_generateLocalKeys
                0x60014958      0x188 ./open62541/open62541.o
 .text.UA_SecureChannel_generateRemoteKeys
                0x60014ae0      0x188 ./open62541/open62541.o
 .text.UA_SecureChannel_generateNewKeys
                0x60014c68       0x70 ./open62541/open62541.o
                0x60014c68                UA_SecureChannel_generateNewKeys
 .text.UA_SecureChannel_revolveTokens
                0x60014cd8       0x7c ./open62541/open62541.o
                0x60014cd8                UA_SecureChannel_revolveTokens
 .text.prependHeadersAsym
                0x60014d54      0x120 ./open62541/open62541.o
 .text.UA_SecureChannel_sendAsymmetricOPNMessage
                0x60014e74      0x180 ./open62541/open62541.o
                0x60014e74                UA_SecureChannel_sendAsymmetricOPNMessage
 .text.checkLimitsSym
                0x60014ff4       0x98 ./open62541/open62541.o
 .text.encodeHeadersSym
                0x6001508c       0xe0 ./open62541/open62541.o
 .text.sendSymmetricChunk
                0x6001516c      0x100 ./open62541/open62541.o
 .text.sendSymmetricEncodingCallback
                0x6001526c       0x84 ./open62541/open62541.o
 .text.UA_MessageContext_begin
                0x600152f0       0x9c ./open62541/open62541.o
                0x600152f0                UA_MessageContext_begin
 .text.UA_MessageContext_encode
                0x6001538c       0x50 ./open62541/open62541.o
                0x6001538c                UA_MessageContext_encode
 .text.UA_SecureChannel_sendSymmetricMessage
                0x600153dc      0x100 ./open62541/open62541.o
                0x600153dc                UA_SecureChannel_sendSymmetricMessage
 .text.addChunkPayload
                0x600154dc      0x190 ./open62541/open62541.o
 .text.processMessage
                0x6001566c       0xd0 ./open62541/open62541.o
 .text.decryptChunk
                0x6001573c       0xec ./open62541/open62541.o
 .text.decodeChunkPaddingSize
                0x60015828       0xd8 ./open62541/open62541.o
 .text.verifyChunk
                0x60015900       0x88 ./open62541/open62541.o
 .text.decryptAndVerifyChunk
                0x60015988      0x174 ./open62541/open62541.o
 .text.processSequenceNumberAsym
                0x60015afc       0x58 ./open62541/open62541.o
 .text.processSequenceNumberSym
                0x60015b54       0x94 ./open62541/open62541.o
 .text.checkAsymHeader
                0x60015be8       0x58 ./open62541/open62541.o
 .text.checkSymHeader
                0x60015c40      0x168 ./open62541/open62541.o
 .text.putPayload
                0x60015da8       0x64 ./open62541/open62541.o
 .text.decryptAddChunk
                0x60015e0c      0x228 ./open62541/open62541.o
 .text.UA_SecureChannel_decryptAddChunk
                0x60016034       0x54 ./open62541/open62541.o
                0x60016034                UA_SecureChannel_decryptAddChunk
 .text.UA_Session_generateNonce
                0x60016088       0x6c ./open62541/open62541.o
                0x60016088                UA_Session_generateNonce
 .text.UA_Session_deleteSubscription
                0x600160f4       0xc4 ./open62541/open62541.o
                0x600160f4                UA_Session_deleteSubscription
 .text.UA_Node_deleteMembers
                0x600161b8       0xd8 ./open62541/open62541.o
                0x600161b8                UA_Node_deleteMembers
 .text.UA_CommonVariableNode_copy
                0x60016290       0xb0 ./open62541/open62541.o
 .text.UA_Node_copy
                0x60016340      0x3ac ./open62541/open62541.o
                0x60016340                UA_Node_copy
 .text.copyCommonVariableAttributes
                0x600166ec       0xa0 ./open62541/open62541.o
 .text.UA_Node_setAttributes
                0x6001678c      0x164 ./open62541/open62541.o
                0x6001678c                UA_Node_setAttributes
 .text.addReferenceTarget
                0x600168f0      0x178 ./open62541/open62541.o
 .text.addReferenceKind
                0x60016a68       0xf0 ./open62541/open62541.o
 .text.UA_Node_addReference
                0x60016b58       0xcc ./open62541/open62541.o
                0x60016b58                UA_Node_addReference
 .text.UA_Node_deleteReference
                0x60016c24      0x1cc ./open62541/open62541.o
                0x60016c24                UA_Node_deleteReference
 .text.UA_Server_delete
                0x60016df0       0xd0 ./open62541/open62541.o
                0x60016df0                UA_Server_delete
 .text.UA_Server_run_startup
                0x60016ec0      0x1bc ./open62541/open62541.o
                0x60016ec0                UA_Server_run_startup
 .text.UA_Server_run_iterate
                0x6001707c      0x13c ./open62541/open62541.o
                0x6001707c                UA_Server_run_iterate
 .text.addObjectNode
                0x600171b8       0xfc ./open62541/open62541.o
 .text.addReferenceTypeNode
                0x600172b4      0x108 ./open62541/open62541.o
 .text.UA_Server_createNS0_base
                0x600173bc      0xab4 ./open62541/open62541.o
 .text.readStatus
                0x60017e70      0x330 ./open62541/open62541.o
 .text.readServiceLevel
                0x600181a0       0x9c ./open62541/open62541.o
 .text.readAuditing
                0x6001823c       0x9c ./open62541/open62541.o
 .text.readNamespaces
                0x600182d8       0x98 ./open62541/open62541.o
 .text.writeNamespaces
                0x60018370       0xec ./open62541/open62541.o
 .text.readCurrentTime
                0x6001845c       0x94 ./open62541/open62541.o
 .text.readMinSamplingInterval
                0x600184f0       0x8c ./open62541/open62541.o
 .text.readMonitoredItems
                0x6001857c      0x148 ./open62541/open62541.o
 .text.UA_Server_initNS0
                0x600186c4      0xbec ./open62541/open62541.o
                0x600186c4                UA_Server_initNS0
 .text.sendServiceFaultWithRequest
                0x600192b0       0xd0 ./open62541/open62541.o
 .text.getServicePointers
                0x60019380      0x564 ./open62541/open62541.o
 .text.processHEL
                0x600198e4      0x150 ./open62541/open62541.o
 .text.processOPN
                0x60019a34      0x28c ./open62541/open62541.o
 .text.sendResponse
                0x60019cc0       0xe4 ./open62541/open62541.o
 .text.processMSGDecoded
                0x60019da4      0x370 ./open62541/open62541.o
 .text.processMSG
                0x6001a114      0x304 ./open62541/open62541.o
 .text.processSecureChannelMessage
                0x6001a418      0x17c ./open62541/open62541.o
 .text.createSecureChannel
                0x6001a594       0xa4 ./open62541/open62541.o
 .text.processCompleteChunkWithoutChannel
                0x6001a638      0x138 ./open62541/open62541.o
 .text.UA_Server_processBinaryMessage
                0x6001a770       0xb8 ./open62541/open62541.o
                0x6001a770                UA_Server_processBinaryMessage
 .text.isNodeInTreeNoCircular
                0x6001a828      0x1d0 ./open62541/open62541.o
 .text.getNodeType
                0x6001a9f8      0x190 ./open62541/open62541.o
                0x6001a9f8                getNodeType
 .text.getParentTypeAndInterfaceHierarchy
                0x6001ab88      0x22c ./open62541/open62541.o
                0x6001ab88                getParentTypeAndInterfaceHierarchy
 .text.UA_Server_editNode
                0x6001adb4       0x54 ./open62541/open62541.o
                0x6001adb4                UA_Server_editNode
 .text.UA_Server_processServiceOperations
                0x6001ae08       0xa4 ./open62541/open62541.o
                0x6001ae08                UA_Server_processServiceOperations
 .text.removeSecureChannel
                0x6001aeac       0x78 ./open62541/open62541.o
 .text.UA_SecureChannelManager_cleanupTimedOut
                0x6001af24      0x11c ./open62541/open62541.o
                0x6001af24                UA_SecureChannelManager_cleanupTimedOut
 .text.purgeFirstChannelWithoutSession
                0x6001b040       0x70 ./open62541/open62541.o
 .text.UA_SecureChannelManager_create
                0x6001b0b0      0x10c ./open62541/open62541.o
                0x6001b0b0                UA_SecureChannelManager_create
 .text.UA_SecureChannelManager_open
                0x6001b1bc      0x17c ./open62541/open62541.o
                0x6001b1bc                UA_SecureChannelManager_open
 .text.UA_SecureChannelManager_renew
                0x6001b338      0x140 ./open62541/open62541.o
                0x6001b338                UA_SecureChannelManager_renew
 .text.UA_SecureChannelManager_close
                0x6001b478       0x4c ./open62541/open62541.o
                0x6001b478                UA_SecureChannelManager_close
 .text.removeSession
                0x6001b4c4       0xe8 ./open62541/open62541.o
 .text.UA_SessionManager_cleanupTimedOut
                0x6001b5ac       0xc8 ./open62541/open62541.o
                0x6001b5ac                UA_SessionManager_cleanupTimedOut
 .text.UA_SessionManager_getSessionByToken
                0x6001b674      0x120 ./open62541/open62541.o
                0x6001b674                UA_SessionManager_getSessionByToken
 .text.UA_SessionManager_getSessionById
                0x6001b794      0x120 ./open62541/open62541.o
                0x6001b794                UA_SessionManager_getSessionById
 .text.UA_SessionManager_createSession
                0x6001b8b4      0x148 ./open62541/open62541.o
                0x6001b8b4                UA_SessionManager_createSession
 .text.UA_SessionManager_removeSession
                0x6001b9fc       0x54 ./open62541/open62541.o
                0x6001b9fc                UA_SessionManager_removeSession
 .text.RefTree_init
                0x6001ba50       0x48 ./open62541/open62541.o
 .text.RefTree_double
                0x6001ba98      0x18c ./open62541/open62541.o
 .text.addRelevantReferences
                0x6001bc24       0xf4 ./open62541/open62541.o
 .text.referenceSubtypes
                0x6001bd18      0x154 ./open62541/open62541.o
                0x6001bd18                referenceSubtypes
 .text.RefResult_init
                0x6001be6c       0x4c ./open62541/open62541.o
 .text.RefResult_double
                0x6001beb8       0x78 ./open62541/open62541.o
 .text.RefResult_clear
                0x6001bf30       0x68 ./open62541/open62541.o
 .text.ContinuationPoint_clear
                0x6001bf98       0x3c ./open62541/open62541.o
                0x6001bf98                ContinuationPoint_clear
 .text.browseReferences
                0x6001bfd4      0x1e4 ./open62541/open62541.o
 .text.browseWithContinuation
                0x6001c1b8      0x170 ./open62541/open62541.o
 .text.Operation_Browse
                0x6001c328      0x2ac ./open62541/open62541.o
                0x6001c328                Operation_Browse
 .text.Service_Browse
                0x6001c5d4       0x94 ./open62541/open62541.o
                0x6001c5d4                Service_Browse
 .text.Operation_BrowseNext
                0x6001c668       0xe0 ./open62541/open62541.o
 .text.Service_BrowseNext
                0x6001c748       0x54 ./open62541/open62541.o
                0x6001c748                Service_BrowseNext
 .text.walkBrowsePathElementReferenceTargets
                0x6001c79c      0x138 ./open62541/open62541.o
 .text.walkBrowsePathElement
                0x6001c8d4      0x1f8 ./open62541/open62541.o
 .text.walkBrowsePath
                0x6001cacc      0x25c ./open62541/open62541.o
 .text.Operation_TranslateBrowsePathToNodeIds
                0x6001cd28      0x228 ./open62541/open62541.o
 .text.Service_TranslateBrowsePathsToNodeIds
                0x6001cf50       0x74 ./open62541/open62541.o
                0x6001cf50                Service_TranslateBrowsePathsToNodeIds
 .text.Service_RegisterNodes
                0x6001cfc4       0x7c ./open62541/open62541.o
                0x6001cfc4                Service_RegisterNodes
 .text.Service_UnregisterNodes
                0x6001d040       0x50 ./open62541/open62541.o
                0x6001d040                Service_UnregisterNodes
 .text.typeCheckArguments
                0x6001d090      0x148 ./open62541/open62541.o
 .text.validMethodArguments
                0x6001d1d8       0x7c ./open62541/open62541.o
 .text.callWithMethodAndObject
                0x6001d254      0x2f0 ./open62541/open62541.o
 .text.Operation_CallMethod
                0x6001d544       0x98 ./open62541/open62541.o
 .text.Service_Call
                0x6001d5dc       0x6c ./open62541/open62541.o
                0x6001d5dc                Service_Call
 .text.Service_CreateSession
                0x6001d648      0x568 ./open62541/open62541.o
                0x6001d648                Service_CreateSession
 .text.checkSignature
                0x6001dbb0       0xcc ./open62541/open62541.o
 .text.Service_ActivateSession
                0x6001dc7c      0x528 ./open62541/open62541.o
                0x6001dc7c                Service_ActivateSession
 .text.Service_CloseSession
                0x6001e1a4       0xac ./open62541/open62541.o
                0x6001e1a4                Service_CloseSession
 .text.readIsAbstractAttribute
                0x6001e250       0x68 ./open62541/open62541.o
 .text.readValueAttributeFromNode
                0x6001e2b8       0xac ./open62541/open62541.o
 .text.readValueAttributeFromDataSource
                0x6001e364       0xd4 ./open62541/open62541.o
 .text.ReadWithNode
                0x6001e438      0x560 ./open62541/open62541.o
                0x6001e438                ReadWithNode
 .text.Operation_Read
                0x6001e998       0x70 ./open62541/open62541.o
 .text.Service_Read
                0x6001ea08       0x9c ./open62541/open62541.o
                0x6001ea08                Service_Read
 .text.UA_Server_readWithSession
                0x6001eaa4       0xac ./open62541/open62541.o
                0x6001eaa4                UA_Server_readWithSession
 .text.__UA_Server_read
                0x6001eb50       0xc4 ./open62541/open62541.o
                0x6001eb50                __UA_Server_read
 .text.compatibleDataType
                0x6001ec14       0xf4 ./open62541/open62541.o
                0x6001ec14                compatibleDataType
 .text.compatibleValueRankArrayDimensions
                0x6001ed08      0x1b0 ./open62541/open62541.o
                0x6001ed08                compatibleValueRankArrayDimensions
 .text.compatibleValueRanks
                0x6001eeb8       0x7c ./open62541/open62541.o
                0x6001eeb8                compatibleValueRanks
 .text.compatibleValueRankValue
                0x6001ef34       0xb4 ./open62541/open62541.o
 .text.compatibleValueArrayDimensions
                0x6001efe8       0x7c ./open62541/open62541.o
                0x6001efe8                compatibleValueArrayDimensions
 .text.compatibleValue
                0x6001f064      0x124 ./open62541/open62541.o
                0x6001f064                compatibleValue
 .text.adjustValue
                0x6001f188       0x98 ./open62541/open62541.o
 .text.writeArrayDimensionsAttribute
                0x6001f220      0x1a0 ./open62541/open62541.o
 .text.writeValueRankAttribute
                0x6001f3c0      0x128 ./open62541/open62541.o
 .text.writeDataTypeAttribute
                0x6001f4e8      0x164 ./open62541/open62541.o
 .text.writeValueAttributeWithRange
                0x6001f64c      0x15c ./open62541/open62541.o
 .text.writeValueAttribute
                0x6001f7a8      0x240 ./open62541/open62541.o
 .text.writeIsAbstractAttribute
                0x6001f9e8       0x68 ./open62541/open62541.o
 .text.copyAttributeIntoNode
                0x6001fa50      0x94c ./open62541/open62541.o
 .text.Operation_Write
                0x6002039c       0x30 ./open62541/open62541.o
 .text.Service_Write
                0x600203cc       0x6c ./open62541/open62541.o
                0x600203cc                Service_Write
 .text.UA_Server_writeWithSession
                0x60020438       0x2c ./open62541/open62541.o
                0x60020438                UA_Server_writeWithSession
 .text.UA_Server_write
                0x60020464       0x2c ./open62541/open62541.o
                0x60020464                UA_Server_write
 .text.__UA_Server_write
                0x60020490       0x84 ./open62541/open62541.o
                0x60020490                __UA_Server_write
 .text.setApplicationDescriptionFromRegisteredServer
                0x60020514      0x1d0 ./open62541/open62541.o
 .text.setApplicationDescriptionFromServer
                0x600206e4       0xc4 ./open62541/open62541.o
 .text.Service_FindServers
                0x600207a8      0x1e8 ./open62541/open62541.o
                0x600207a8                Service_FindServers
 .text.Service_GetEndpoints
                0x60020990      0x26c ./open62541/open62541.o
                0x60020990                Service_GetEndpoints
 .text.process_RegisterServer
                0x60020bfc      0x3b0 ./open62541/open62541.o
 .text.UA_Discovery_cleanupTimedOut
                0x60020fac      0x18c ./open62541/open62541.o
                0x60020fac                UA_Discovery_cleanupTimedOut
 .text.Service_CreateSubscription
                0x60021138      0x184 ./open62541/open62541.o
                0x60021138                Service_CreateSubscription
 .text.Service_ModifySubscription
                0x600212bc       0x94 ./open62541/open62541.o
                0x600212bc                Service_ModifySubscription
 .text.Operation_SetPublishingMode
                0x60021350       0x44 ./open62541/open62541.o
 .text.Service_SetPublishingMode
                0x60021394       0x54 ./open62541/open62541.o
                0x60021394                Service_SetPublishingMode
 .text.subscriptionSendError
                0x600213e8       0x50 ./open62541/open62541.o
 .text.Service_Publish
                0x60021438      0x218 ./open62541/open62541.o
                0x60021438                Service_Publish
 .text.Service_DeleteSubscriptions
                0x60021650       0x5c ./open62541/open62541.o
                0x60021650                Service_DeleteSubscriptions
 .text.Service_Republish
                0x600216ac       0x8c ./open62541/open62541.o
                0x600216ac                Service_Republish
 .text.setMonitoredItemSettings
                0x60021738      0x260 ./open62541/open62541.o
 .text.Operation_CreateMonitoredItem
                0x60021998      0x4a0 ./open62541/open62541.o
 .text.Service_CreateMonitoredItems
                0x60021e38       0xb0 ./open62541/open62541.o
                0x60021e38                Service_CreateMonitoredItems
 .text.Operation_ModifyMonitoredItem
                0x60021ee8       0xd8 ./open62541/open62541.o
 .text.Service_ModifyMonitoredItems
                0x60021fc0       0xa4 ./open62541/open62541.o
                0x60021fc0                Service_ModifyMonitoredItems
 .text.Operation_SetMonitoringMode
                0x60022064      0x1ac ./open62541/open62541.o
 .text.Service_SetMonitoringMode
                0x60022210       0x9c ./open62541/open62541.o
                0x60022210                Service_SetMonitoringMode
 .text.Service_DeleteMonitoredItems
                0x600222ac       0x90 ./open62541/open62541.o
                0x600222ac                Service_DeleteMonitoredItems
 .text.Service_OpenSecureChannel
                0x6002233c      0x130 ./open62541/open62541.o
                0x6002233c                Service_OpenSecureChannel
 .text.Service_CloseSecureChannel
                0x6002246c       0x58 ./open62541/open62541.o
                0x6002246c                Service_CloseSecureChannel
 .text.UA_Server_getNodeContext
                0x600224c4       0x5c ./open62541/open62541.o
                0x600224c4                UA_Server_getNodeContext
 .text.checkParentReference
                0x60022520      0x554 ./open62541/open62541.o
 .text.typeCheckVariableNode
                0x60022a74      0x500 ./open62541/open62541.o
 .text.useVariableTypeAttributes
                0x60022f74      0x29c ./open62541/open62541.o
 .text.isMandatoryChild
                0x60023210       0xdc ./open62541/open62541.o
 .text.addTypeChildren
                0x600232ec       0xa8 ./open62541/open62541.o
 .text.AddNode_addRefs
                0x60023394      0xebc ./open62541/open62541.o
                0x60023394                AddNode_addRefs
 .text.AddNode_raw
                0x60024250      0x3c0 ./open62541/open62541.o
                0x60024250                AddNode_raw
 .text.recursiveTypeCheckAddChildren
                0x60024610      0x380 ./open62541/open62541.o
 .text.findDefaultInstanceBrowseNameNode
                0x60024990       0xd4 ./open62541/open62541.o
 .text.checkValidBrowseName
                0x60024a64      0x114 ./open62541/open62541.o
 .text.recursiveCallConstructors
                0x60024b78      0x31c ./open62541/open62541.o
 .text.AddNode_finish
                0x60024e94      0x284 ./open62541/open62541.o
                0x60024e94                AddNode_finish
 .text.Service_AddNodes
                0x60025118       0x6c ./open62541/open62541.o
                0x60025118                Service_AddNodes
 .text.recursiveDeconstructNode
                0x60025184      0x20c ./open62541/open62541.o
 .text.deleteNodeOperation
                0x60025390      0x230 ./open62541/open62541.o
 .text.Service_DeleteNodes
                0x600255c0       0x6c ./open62541/open62541.o
                0x600255c0                Service_DeleteNodes
 .text.Operation_addReference
                0x6002562c      0x1f8 ./open62541/open62541.o
 .text.Service_AddReferences
                0x60025824       0x6c ./open62541/open62541.o
                0x60025824                Service_AddReferences
 .text.Operation_deleteReference
                0x60025890      0x11c ./open62541/open62541.o
 .text.Service_DeleteReferences
                0x600259ac       0x6c ./open62541/open62541.o
                0x600259ac                Service_DeleteReferences
 .text.setDataSource
                0x60025a18       0x54 ./open62541/open62541.o
 .text.UA_Server_setVariableNode_dataSource
                0x60025a6c       0x40 ./open62541/open62541.o
                0x60025a6c                UA_Server_setVariableNode_dataSource
 .text.UA_Server_addMethodNodeEx_finish
                0x60025aac      0x598 ./open62541/open62541.o
 .text.UA_Server_addMethodNode_finish
                0x60026044       0x78 ./open62541/open62541.o
                0x60026044                UA_Server_addMethodNode_finish
 .text.UA_Server_addMethodNodeEx
                0x600260bc      0x13c ./open62541/open62541.o
                0x600260bc                UA_Server_addMethodNodeEx
 .text.editMethodCallback
                0x600261f8       0x38 ./open62541/open62541.o
 .text.UA_Server_setMethodNode_callback
                0x60026230       0x3c ./open62541/open62541.o
                0x60026230                UA_Server_setMethodNode_callback
 .text.pcg32_random_r
                0x6002626c       0xa8 ./open62541/open62541.o
                0x6002626c                pcg32_random_r
 .text.UA_base64
                0x60026314      0x18c ./open62541/open62541.o
                0x60026314                UA_base64
 .text.function_namespace0_generated_0_begin
                0x600264a0      0x124 ./open62541/open62541.o
 .text.function_namespace0_generated_1_begin
                0x600265c4      0x124 ./open62541/open62541.o
 .text.function_namespace0_generated_2_begin
                0x600266e8      0x120 ./open62541/open62541.o
 .text.function_namespace0_generated_3_begin
                0x60026808      0x120 ./open62541/open62541.o
 .text.function_namespace0_generated_4_begin
                0x60026928      0x120 ./open62541/open62541.o
 .text.function_namespace0_generated_5_begin
                0x60026a48      0x120 ./open62541/open62541.o
 .text.function_namespace0_generated_6_begin
                0x60026b68      0x120 ./open62541/open62541.o
 .text.function_namespace0_generated_7_begin
                0x60026c88      0x104 ./open62541/open62541.o
 .text.function_namespace0_generated_8_begin
                0x60026d8c      0x104 ./open62541/open62541.o
 .text.function_namespace0_generated_9_begin
                0x60026e90      0x10c ./open62541/open62541.o
 .text.function_namespace0_generated_10_begin
                0x60026f9c      0x108 ./open62541/open62541.o
 .text.function_namespace0_generated_11_begin
                0x600270a4      0x108 ./open62541/open62541.o
 .text.function_namespace0_generated_12_begin
                0x600271ac      0x108 ./open62541/open62541.o
 .text.function_namespace0_generated_13_begin
                0x600272b4      0x108 ./open62541/open62541.o
 .text.function_namespace0_generated_14_begin
                0x600273bc      0x108 ./open62541/open62541.o
 .text.function_namespace0_generated_15_begin
                0x600274c4      0x108 ./open62541/open62541.o
 .text.function_namespace0_generated_16_begin
                0x600275cc      0x108 ./open62541/open62541.o
 .text.function_namespace0_generated_17_begin
                0x600276d4      0x104 ./open62541/open62541.o
 .text.function_namespace0_generated_18_begin
                0x600277d8      0x104 ./open62541/open62541.o
 .text.function_namespace0_generated_19_begin
                0x600278dc      0x104 ./open62541/open62541.o
 .text.function_namespace0_generated_20_begin
                0x600279e0      0x104 ./open62541/open62541.o
 .text.function_namespace0_generated_21_begin
                0x60027ae4      0x104 ./open62541/open62541.o
 .text.function_namespace0_generated_22_begin
                0x60027be8      0x104 ./open62541/open62541.o
 .text.function_namespace0_generated_23_begin
                0x60027cec      0x104 ./open62541/open62541.o
 .text.function_namespace0_generated_24_begin
                0x60027df0      0x10c ./open62541/open62541.o
 .text.function_namespace0_generated_25_begin
                0x60027efc      0x104 ./open62541/open62541.o
 .text.function_namespace0_generated_26_begin
                0x60028000      0x104 ./open62541/open62541.o
 .text.function_namespace0_generated_27_begin
                0x60028104      0x108 ./open62541/open62541.o
 .text.function_namespace0_generated_28_begin
                0x6002820c      0x104 ./open62541/open62541.o
 .text.function_namespace0_generated_29_begin
                0x60028310      0x108 ./open62541/open62541.o
 .text.function_namespace0_generated_30_begin
                0x60028418      0x104 ./open62541/open62541.o
 .text.function_namespace0_generated_31_begin
                0x6002851c      0x10c ./open62541/open62541.o
 .text.function_namespace0_generated_32_begin
                0x60028628      0x104 ./open62541/open62541.o
 .text.function_namespace0_generated_33_begin
                0x6002872c      0x2c4 ./open62541/open62541.o
 .text.function_namespace0_generated_34_begin
                0x600289f0      0x108 ./open62541/open62541.o
 .text.function_namespace0_generated_35_begin
                0x60028af8      0x268 ./open62541/open62541.o
 .text.function_namespace0_generated_36_begin
                0x60028d60      0x108 ./open62541/open62541.o
 .text.function_namespace0_generated_37_begin
                0x60028e68      0x10c ./open62541/open62541.o
 .text.function_namespace0_generated_38_begin
                0x60028f74      0x10c ./open62541/open62541.o
 .text.function_namespace0_generated_39_begin
                0x60029080      0x104 ./open62541/open62541.o
 .text.function_namespace0_generated_40_begin
                0x60029184      0x104 ./open62541/open62541.o
 .text.function_namespace0_generated_41_begin
                0x60029288      0x104 ./open62541/open62541.o
 .text.function_namespace0_generated_42_begin
                0x6002938c      0x104 ./open62541/open62541.o
 .text.function_namespace0_generated_43_begin
                0x60029490      0x10c ./open62541/open62541.o
 .text.function_namespace0_generated_44_begin
                0x6002959c      0x104 ./open62541/open62541.o
 .text.function_namespace0_generated_45_begin
                0x600296a0      0x104 ./open62541/open62541.o
 .text.function_namespace0_generated_46_begin
                0x600297a4      0x104 ./open62541/open62541.o
 .text.function_namespace0_generated_47_begin
                0x600298a8      0x104 ./open62541/open62541.o
 .text.function_namespace0_generated_48_begin
                0x600299ac      0x104 ./open62541/open62541.o
 .text.function_namespace0_generated_49_begin
                0x60029ab0      0x108 ./open62541/open62541.o
 .text.function_namespace0_generated_50_begin
                0x60029bb8      0x104 ./open62541/open62541.o
 .text.function_namespace0_generated_51_begin
                0x60029cbc      0x104 ./open62541/open62541.o
 .text.function_namespace0_generated_52_begin
                0x60029dc0      0x128 ./open62541/open62541.o
 .text.function_namespace0_generated_53_begin
                0x60029ee8      0x17c ./open62541/open62541.o
 .text.function_namespace0_generated_54_begin
                0x6002a064      0x17c ./open62541/open62541.o
 .text.function_namespace0_generated_55_begin
                0x6002a1e0      0x17c ./open62541/open62541.o
 .text.function_namespace0_generated_56_begin
                0x6002a35c      0x17c ./open62541/open62541.o
 .text.function_namespace0_generated_57_begin
                0x6002a4d8      0x17c ./open62541/open62541.o
 .text.function_namespace0_generated_58_begin
                0x6002a654      0x110 ./open62541/open62541.o
 .text.function_namespace0_generated_59_begin
                0x6002a764      0x17c ./open62541/open62541.o
 .text.function_namespace0_generated_60_begin
                0x6002a8e0      0x17c ./open62541/open62541.o
 .text.function_namespace0_generated_61_begin
                0x6002aa5c      0x17c ./open62541/open62541.o
 .text.function_namespace0_generated_62_begin
                0x6002abd8      0x17c ./open62541/open62541.o
 .text.function_namespace0_generated_63_begin
                0x6002ad54      0x114 ./open62541/open62541.o
 .text.function_namespace0_generated_64_begin
                0x6002ae68      0x18c ./open62541/open62541.o
 .text.function_namespace0_generated_65_begin
                0x6002aff4      0x140 ./open62541/open62541.o
 .text.function_namespace0_generated_66_begin
                0x6002b134      0x160 ./open62541/open62541.o
 .text.function_namespace0_generated_67_begin
                0x6002b294      0x160 ./open62541/open62541.o
 .text.function_namespace0_generated_68_begin
                0x6002b3f4      0x160 ./open62541/open62541.o
 .text.function_namespace0_generated_69_begin
                0x6002b554      0x160 ./open62541/open62541.o
 .text.function_namespace0_generated_70_begin
                0x6002b6b4      0x160 ./open62541/open62541.o
 .text.function_namespace0_generated_71_begin
                0x6002b814      0x160 ./open62541/open62541.o
 .text.function_namespace0_generated_72_begin
                0x6002b974      0x160 ./open62541/open62541.o
 .text.function_namespace0_generated_73_begin
                0x6002bad4      0x160 ./open62541/open62541.o
 .text.function_namespace0_generated_74_begin
                0x6002bc34      0x160 ./open62541/open62541.o
 .text.function_namespace0_generated_75_begin
                0x6002bd94      0x160 ./open62541/open62541.o
 .text.function_namespace0_generated_76_begin
                0x6002bef4      0x160 ./open62541/open62541.o
 .text.function_namespace0_generated_77_begin
                0x6002c054      0x160 ./open62541/open62541.o
 .text.function_namespace0_generated_78_begin
                0x6002c1b4      0x140 ./open62541/open62541.o
 .text.function_namespace0_generated_79_begin
                0x6002c2f4      0x140 ./open62541/open62541.o
 .text.function_namespace0_generated_80_begin
                0x6002c434      0x108 ./open62541/open62541.o
 .text.function_namespace0_generated_81_begin
                0x6002c53c      0x160 ./open62541/open62541.o
 .text.function_namespace0_generated_82_begin
                0x6002c69c      0x160 ./open62541/open62541.o
 .text.function_namespace0_generated_83_begin
                0x6002c7fc      0x160 ./open62541/open62541.o
 .text.function_namespace0_generated_84_begin
                0x6002c95c      0x160 ./open62541/open62541.o
 .text.function_namespace0_generated_85_begin
                0x6002cabc      0x160 ./open62541/open62541.o
 .text.function_namespace0_generated_86_begin
                0x6002cc1c      0x160 ./open62541/open62541.o
 .text.function_namespace0_generated_87_begin
                0x6002cd7c      0x160 ./open62541/open62541.o
 .text.function_namespace0_generated_88_begin
                0x6002cedc      0x160 ./open62541/open62541.o
 .text.function_namespace0_generated_89_begin
                0x6002d03c      0x108 ./open62541/open62541.o
 .text.function_namespace0_generated_90_begin
                0x6002d144      0x160 ./open62541/open62541.o
 .text.function_namespace0_generated_91_begin
                0x6002d2a4      0x108 ./open62541/open62541.o
 .text.function_namespace0_generated_92_begin
                0x6002d3ac      0x108 ./open62541/open62541.o
 .text.function_namespace0_generated_93_begin
                0x6002d4b4      0x108 ./open62541/open62541.o
 .text.function_namespace0_generated_94_begin
                0x6002d5bc      0x118 ./open62541/open62541.o
 .text.function_namespace0_generated_95_begin
                0x6002d6d4      0x108 ./open62541/open62541.o
 .text.function_namespace0_generated_96_begin
                0x6002d7dc      0x118 ./open62541/open62541.o
 .text.function_namespace0_generated_97_begin
                0x6002d8f4      0x11c ./open62541/open62541.o
 .text.function_namespace0_generated_98_begin
                0x6002da10      0x164 ./open62541/open62541.o
 .text.function_namespace0_generated_99_begin
                0x6002db74      0x160 ./open62541/open62541.o
 .text.function_namespace0_generated_100_begin
                0x6002dcd4      0x160 ./open62541/open62541.o
 .text.function_namespace0_generated_101_begin
                0x6002de34      0x160 ./open62541/open62541.o
 .text.function_namespace0_generated_102_begin
                0x6002df94      0x160 ./open62541/open62541.o
 .text.function_namespace0_generated_103_begin
                0x6002e0f4      0x164 ./open62541/open62541.o
 .text.function_namespace0_generated_104_begin
                0x6002e258      0x164 ./open62541/open62541.o
 .text.function_namespace0_generated_105_begin
                0x6002e3bc      0x160 ./open62541/open62541.o
 .text.function_namespace0_generated_106_begin
                0x6002e51c      0x160 ./open62541/open62541.o
 .text.function_namespace0_generated_107_begin
                0x6002e67c      0x160 ./open62541/open62541.o
 .text.function_namespace0_generated_108_begin
                0x6002e7dc      0x160 ./open62541/open62541.o
 .text.function_namespace0_generated_109_begin
                0x6002e93c      0x160 ./open62541/open62541.o
 .text.function_namespace0_generated_110_begin
                0x6002ea9c      0x160 ./open62541/open62541.o
 .text.function_namespace0_generated_111_begin
                0x6002ebfc      0x118 ./open62541/open62541.o
 .text.function_namespace0_generated_112_begin
                0x6002ed14      0x118 ./open62541/open62541.o
 .text.function_namespace0_generated_113_begin
                0x6002ee2c      0x160 ./open62541/open62541.o
 .text.function_namespace0_generated_114_begin
                0x6002ef8c      0x114 ./open62541/open62541.o
 .text.function_namespace0_generated_115_begin
                0x6002f0a0      0x160 ./open62541/open62541.o
 .text.function_namespace0_generated_116_begin
                0x6002f200      0x160 ./open62541/open62541.o
 .text.function_namespace0_generated_117_begin
                0x6002f360      0x160 ./open62541/open62541.o
 .text.function_namespace0_generated_118_begin
                0x6002f4c0      0x118 ./open62541/open62541.o
 .text.function_namespace0_generated_119_begin
                0x6002f5d8      0x160 ./open62541/open62541.o
 .text.function_namespace0_generated_120_begin
                0x6002f738      0x160 ./open62541/open62541.o
 .text.function_namespace0_generated_121_begin
                0x6002f898      0x160 ./open62541/open62541.o
 .text.function_namespace0_generated_122_begin
                0x6002f9f8      0x160 ./open62541/open62541.o
 .text.function_namespace0_generated_123_begin
                0x6002fb58      0x160 ./open62541/open62541.o
 .text.function_namespace0_generated_124_begin
                0x6002fcb8      0x160 ./open62541/open62541.o
 .text.function_namespace0_generated_125_begin
                0x6002fe18      0x160 ./open62541/open62541.o
 .text.function_namespace0_generated_126_begin
                0x6002ff78      0x160 ./open62541/open62541.o
 .text.function_namespace0_generated_127_begin
                0x600300d8      0x178 ./open62541/open62541.o
 .text.function_namespace0_generated_128_begin
                0x60030250      0x178 ./open62541/open62541.o
 .text.function_namespace0_generated_129_begin
                0x600303c8      0x178 ./open62541/open62541.o
 .text.function_namespace0_generated_130_begin
                0x60030540      0x114 ./open62541/open62541.o
 .text.function_namespace0_generated_131_begin
                0x60030654      0x160 ./open62541/open62541.o
 .text.function_namespace0_generated_132_begin
                0x600307b4      0x118 ./open62541/open62541.o
 .text.function_namespace0_generated_133_begin
                0x600308cc      0x164 ./open62541/open62541.o
 .text.function_namespace0_generated_134_begin
                0x60030a30      0x160 ./open62541/open62541.o
 .text.function_namespace0_generated_135_begin
                0x60030b90      0x160 ./open62541/open62541.o
 .text.function_namespace0_generated_136_begin
                0x60030cf0      0x160 ./open62541/open62541.o
 .text.function_namespace0_generated_137_begin
                0x60030e50      0x160 ./open62541/open62541.o
 .text.function_namespace0_generated_138_begin
                0x60030fb0      0x160 ./open62541/open62541.o
 .text.function_namespace0_generated_139_begin
                0x60031110      0x160 ./open62541/open62541.o
 .text.function_namespace0_generated_140_begin
                0x60031270      0x160 ./open62541/open62541.o
 .text.function_namespace0_generated_141_begin
                0x600313d0      0x160 ./open62541/open62541.o
 .text.function_namespace0_generated_142_begin
                0x60031530      0x160 ./open62541/open62541.o
 .text.function_namespace0_generated_143_begin
                0x60031690      0x160 ./open62541/open62541.o
 .text.function_namespace0_generated_144_begin
                0x600317f0      0x160 ./open62541/open62541.o
 .text.function_namespace0_generated_145_begin
                0x60031950      0x160 ./open62541/open62541.o
 .text.function_namespace0_generated_146_begin
                0x60031ab0      0x160 ./open62541/open62541.o
 .text.function_namespace0_generated_147_begin
                0x60031c10      0x120 ./open62541/open62541.o
 .text.function_namespace0_generated_148_begin
                0x60031d30      0x2b8 ./open62541/open62541.o
 .text.function_namespace0_generated_149_begin
                0x60031fe8      0x210 ./open62541/open62541.o
 .text.function_namespace0_generated_150_begin
                0x600321f8      0x178 ./open62541/open62541.o
 .text.function_namespace0_generated_151_begin
                0x60032370      0x118 ./open62541/open62541.o
 .text.function_namespace0_generated_152_begin
                0x60032488      0x160 ./open62541/open62541.o
 .text.function_namespace0_generated_153_begin
                0x600325e8      0x178 ./open62541/open62541.o
 .text.function_namespace0_generated_154_begin
                0x60032760      0x160 ./open62541/open62541.o
 .text.function_namespace0_generated_155_begin
                0x600328c0      0x104 ./open62541/open62541.o
 .text.function_namespace0_generated_156_begin
                0x600329c4      0x1a4 ./open62541/open62541.o
 .text.function_namespace0_generated_157_begin
                0x60032b68      0xf9c ./open62541/open62541.o
 .text.function_namespace0_generated_158_begin
                0x60033b04      0x1a4 ./open62541/open62541.o
 .text.function_namespace0_generated_159_begin
                0x60033ca8      0x6f0 ./open62541/open62541.o
 .text.function_namespace0_generated_160_begin
                0x60034398      0x1a4 ./open62541/open62541.o
 .text.function_namespace0_generated_161_begin
                0x6003453c      0x104 ./open62541/open62541.o
 .text.function_namespace0_generated_162_begin
                0x60034640      0x190 ./open62541/open62541.o
 .text.function_namespace0_generated_163_begin
                0x600347d0      0x190 ./open62541/open62541.o
 .text.function_namespace0_generated_164_begin
                0x60034960      0x104 ./open62541/open62541.o
 .text.function_namespace0_generated_165_begin
                0x60034a64      0x110 ./open62541/open62541.o
 .text.function_namespace0_generated_166_begin
                0x60034b74      0x110 ./open62541/open62541.o
 .text.function_namespace0_generated_167_begin
                0x60034c84      0x13c ./open62541/open62541.o
 .text.function_namespace0_generated_168_begin
                0x60034dc0      0x230 ./open62541/open62541.o
 .text.function_namespace0_generated_169_begin
                0x60034ff0      0x1c0 ./open62541/open62541.o
 .text.function_namespace0_generated_170_begin
                0x600351b0      0x24c ./open62541/open62541.o
 .text.function_namespace0_generated_171_begin
                0x600353fc      0x13c ./open62541/open62541.o
 .text.function_namespace0_generated_172_begin
                0x60035538      0x230 ./open62541/open62541.o
 .text.function_namespace0_generated_173_begin
                0x60035768      0x290 ./open62541/open62541.o
 .text.function_namespace0_generated_174_begin
                0x600359f8      0x290 ./open62541/open62541.o
 .text.function_namespace0_generated_175_begin
                0x60035c88      0x230 ./open62541/open62541.o
 .text.function_namespace0_generated_176_begin
                0x60035eb8      0x114 ./open62541/open62541.o
 .text.function_namespace0_generated_177_begin
                0x60035fcc      0x114 ./open62541/open62541.o
 .text.namespace0_generated
                0x600360e0     0x1eb8 ./open62541/open62541.o
                0x600360e0                namespace0_generated
 .text.UA_Subscription_deleteMembers
                0x60037f98      0x244 ./open62541/open62541.o
                0x60037f98                UA_Subscription_deleteMembers
 .text.UA_Subscription_deleteMonitoredItem
                0x600381dc      0x158 ./open62541/open62541.o
                0x600381dc                UA_Subscription_deleteMonitoredItem
 .text.removeOldestRetransmissionMessage
                0x60038334       0xf4 ./open62541/open62541.o
 .text.UA_Subscription_addRetransmissionMessage
                0x60038428      0x108 ./open62541/open62541.o
 .text.UA_Subscription_removeRetransmissionMessage
                0x60038530       0x9c ./open62541/open62541.o
                0x60038530                UA_Subscription_removeRetransmissionMessage
 .text.prepareNotificationMessage
                0x600385cc      0x33c ./open62541/open62541.o
 .text.UA_Subscription_publish
                0x60038908      0x44c ./open62541/open62541.o
                0x60038908                UA_Subscription_publish
 .text.UA_Subscription_reachedPublishReqLimit
                0x60038d54      0x128 ./open62541/open62541.o
                0x60038d54                UA_Subscription_reachedPublishReqLimit
 .text.Subscription_registerPublishCallback
                0x60038e7c       0x5c ./open62541/open62541.o
                0x60038e7c                Subscription_registerPublishCallback
 .text.UA_Subscription_answerPublishRequestsNoSubscription
                0x60038ed8       0x7c ./open62541/open62541.o
                0x60038ed8                UA_Subscription_answerPublishRequestsNoSubscription
 .text.UA_Notification_isOverflowEvent
                0x60038f54       0x70 ./open62541/open62541.o
 .text.createEventOverflowNotification
                0x60038fc4      0x120 ./open62541/open62541.o
 .text.UA_MonitoredItem_delete
                0x600390e4      0x160 ./open62541/open62541.o
                0x600390e4                UA_MonitoredItem_delete
 .text.UA_MonitoredItem_ensureQueueSpace
                0x60039244      0x248 ./open62541/open62541.o
                0x60039244                UA_MonitoredItem_ensureQueueSpace
 .text.UA_MonitoredItem_registerSampleCallback
                0x6003948c       0x5c ./open62541/open62541.o
                0x6003948c                UA_MonitoredItem_registerSampleCallback
 .text.outOfDeadBand
                0x600394e8      0x58c ./open62541/open62541.o
 .text.detectValueChangeWithFilter
                0x60039a74      0x338 ./open62541/open62541.o
 .text.sampleCallbackWithValue
                0x60039dac      0x2ac ./open62541/open62541.o
 .text.UA_MonitoredItem_sampleCallback
                0x6003a058      0x208 ./open62541/open62541.o
                0x6003a058                UA_MonitoredItem_sampleCallback
 .text.UA_MonitoredItem_removeNodeEventCallback
                0x6003a260       0x98 ./open62541/open62541.o
                0x6003a260                UA_MonitoredItem_removeNodeEventCallback
 .text.activateSession_default
                0x6003a2f8      0x16c ./open62541/open62541.o
 .text.deleteMembers_default
                0x6003a464       0x90 ./open62541/open62541.o
 .text.UA_AccessControl_default
                0x6003a4f4      0x290 ./open62541/open62541.o
                0x6003a4f4                UA_AccessControl_default
 .text.UA_CertificateVerification_AcceptAll
                0x6003a784       0x34 ./open62541/open62541.o
                0x6003a784                UA_CertificateVerification_AcceptAll
 .text.UA_Nodestore_releaseNode
                0x6003a7b8       0x54 ./open62541/open62541.o
                0x6003a7b8                UA_Nodestore_releaseNode
 .text.UA_Nodestore_getNodeCopy
                0x6003a80c       0x88 ./open62541/open62541.o
                0x6003a80c                UA_Nodestore_getNodeCopy
 .text.UA_Nodestore_insertNode
                0x6003a894       0xe4 ./open62541/open62541.o
                0x6003a894                UA_Nodestore_insertNode
 .text.UA_Nodestore_removeNode
                0x6003a978       0x68 ./open62541/open62541.o
                0x6003a978                UA_Nodestore_removeNode
 .text.UA_Nodestore_new
                0x6003a9e0       0x34 ./open62541/open62541.o
                0x6003a9e0                UA_Nodestore_new
 .text.UA_Nodestore_delete
                0x6003aa14       0x34 ./open62541/open62541.o
                0x6003aa14                UA_Nodestore_delete
 .text.createEndpoint
                0x6003aa48       0xb4 ./open62541/open62541.o
 .text.UA_ServerConfig_addNetworkLayerTCP
                0x6003aafc       0xf8 ./open62541/open62541.o
                0x6003aafc                UA_ServerConfig_addNetworkLayerTCP
 .text.UA_ServerConfig_addSecurityPolicyNone
                0x6003abf4       0xa8 ./open62541/open62541.o
                0x6003abf4                UA_ServerConfig_addSecurityPolicyNone
 .text.UA_ServerConfig_addEndpoint
                0x6003ac9c       0xec ./open62541/open62541.o
                0x6003ac9c                UA_ServerConfig_addEndpoint
 .text.UA_ServerConfig_setMinimalCustomBuffer
                0x6003ad88       0xdc ./open62541/open62541.o
                0x6003ad88                UA_ServerConfig_setMinimalCustomBuffer
 .text.generateNonce_none
                0x6003ae64       0x8c ./open62541/open62541.o
 .text.UA_SecurityPolicy_None
                0x6003aef0      0x1b4 ./open62541/open62541.o
                0x6003aef0                UA_SecurityPolicy_None
 .text.UA_DateTime_offset
                0x6003b0a4       0x3c ./open62541/open62541.o
                0x6003b0a4                UA_DateTime_offset
 .text.UA_DateTime_now
                0x6003b0e0      0x110 ./open62541/open62541.o
                0x6003b0e0                UA_DateTime_now
 .text.UA_socket_set_nonblocking
                0x6003b1f0       0x38 ./open62541/open62541.o
                0x6003b1f0                UA_socket_set_nonblocking
 .text.connection_getsendbuffer
                0x6003b228       0x30 ./open62541/open62541.o
 .text.connection_write
                0x6003b258       0xa8 ./open62541/open62541.o
 .text.connection_recv
                0x6003b300      0x1d4 ./open62541/open62541.o
 .text.ServerNetworkLayerTCP_add
                0x6003b4d4      0x134 ./open62541/open62541.o
 .text.addServerSocket
                0x6003b608      0x15c ./open62541/open62541.o
 .text.ServerNetworkLayerTCP_start
                0x6003b764      0x1a8 ./open62541/open62541.o
 .text.ServerNetworkLayerTCP_stop
                0x6003b90c       0x94 ./open62541/open62541.o
 .text.UA_ServerNetworkLayerTCP
                0x6003b9a0       0xb8 ./open62541/open62541.o
                0x6003b9a0                UA_ServerNetworkLayerTCP
 .text.pb_read  0x6003ba58       0xd8 ./nanopb/pb_decode.o
                0x6003ba58                pb_read
 .text.pb_readbyte
                0x6003bb30       0x78 ./nanopb/pb_decode.o
 .text.pb_istream_from_buffer
                0x6003bba8       0x3c ./nanopb/pb_decode.o
                0x6003bba8                pb_istream_from_buffer
 .text.pb_decode_varint32_eof
                0x6003bbe4      0x134 ./nanopb/pb_decode.o
 .text.pb_decode_varint
                0x6003bd18       0xc4 ./nanopb/pb_decode.o
                0x6003bd18                pb_decode_varint
 .text.pb_skip_field
                0x6003bddc       0x84 ./nanopb/pb_decode.o
                0x6003bddc                pb_skip_field
 .text.read_raw_value
                0x6003be60       0xd0 ./nanopb/pb_decode.o
 .text.pb_make_string_substream
                0x6003bf30       0x74 ./nanopb/pb_decode.o
                0x6003bf30                pb_make_string_substream
 .text.decode_basic_field
                0x6003bfa4      0x1ec ./nanopb/pb_decode.o
 .text.decode_static_field
                0x6003c190      0x204 ./nanopb/pb_decode.o
 .text.decode_pointer_field
                0x6003c394       0x34 ./nanopb/pb_decode.o
 .text.decode_callback_field
                0x6003c3c8      0x10c ./nanopb/pb_decode.o
 .text.decode_field
                0x6003c4d4       0x74 ./nanopb/pb_decode.o
 .text.default_extension_decoder
                0x6003c548       0x74 ./nanopb/pb_decode.o
 .text.pb_decode_inner
                0x6003c5bc      0x378 ./nanopb/pb_decode.o
 .text.pb_dec_varint
                0x6003c934      0x234 ./nanopb/pb_decode.o
 .text.pb_dec_bytes
                0x6003cb68       0xe8 ./nanopb/pb_decode.o
 .text.pb_dec_string
                0x6003cc50       0xf8 ./nanopb/pb_decode.o
 .text.pb_dec_submessage
                0x6003cd48      0x120 ./nanopb/pb_decode.o
 .text.pb_dec_fixed_length_bytes
                0x6003ce68       0xa8 ./nanopb/pb_decode.o
 .text.ethernet_input
                0x6003cf10      0x154 ./lwip/src/netif/ethernet.o
                0x6003cf10                ethernet_input
 .text.ethernet_output
                0x6003d064       0x94 ./lwip/src/netif/ethernet.o
                0x6003d064                ethernet_output
 .text.etharp_free_entry
                0x6003d0f8       0xc0 ./lwip/src/core/ipv4/etharp.o
 .text.etharp_tmr
                0x6003d1b8      0x150 ./lwip/src/core/ipv4/etharp.o
                0x6003d1b8                etharp_tmr
 .text.etharp_find_entry
                0x6003d308      0x2c0 ./lwip/src/core/ipv4/etharp.o
 .text.etharp_update_arp_entry
                0x6003d5c8      0x13c ./lwip/src/core/ipv4/etharp.o
 .text.etharp_input
                0x6003d704      0x150 ./lwip/src/core/ipv4/etharp.o
                0x6003d704                etharp_input
 .text.etharp_output_to_arp_index
                0x6003d854      0x124 ./lwip/src/core/ipv4/etharp.o
 .text.etharp_output
                0x6003d978      0x1e4 ./lwip/src/core/ipv4/etharp.o
                0x6003d978                etharp_output
 .text.etharp_query
                0x6003db5c      0x254 ./lwip/src/core/ipv4/etharp.o
                0x6003db5c                etharp_query
 .text.etharp_raw
                0x6003ddb0      0x114 ./lwip/src/core/ipv4/etharp.o
 .text.etharp_request_dst
                0x6003dec4       0x44 ./lwip/src/core/ipv4/etharp.o
 .text.etharp_request
                0x6003df08       0x24 ./lwip/src/core/ipv4/etharp.o
                0x6003df08                etharp_request
 .text.icmp_input
                0x6003df2c      0x248 ./lwip/src/core/ipv4/icmp.o
                0x6003df2c                icmp_input
 .text.icmp_send_response
                0x6003e174       0xd8 ./lwip/src/core/ipv4/icmp.o
 .text.ip4_route
                0x6003e24c      0x110 ./lwip/src/core/ipv4/ip4.o
                0x6003e24c                ip4_route
 .text.ip4_input_accept
                0x6003e35c       0x54 ./lwip/src/core/ipv4/ip4.o
 .text.ip4_input
                0x6003e3b0      0x338 ./lwip/src/core/ipv4/ip4.o
                0x6003e3b0                ip4_input
 .text.ip4_output_if_src
                0x6003e6e8      0x23c ./lwip/src/core/ipv4/ip4.o
                0x6003e6e8                ip4_output_if_src
 .text.ip4addr_aton
                0x6003e924      0x248 ./lwip/src/core/ipv4/ip4_addr.o
                0x6003e924                ip4addr_aton
 .text.ip_reass_tmr
                0x6003eb6c       0x58 ./lwip/src/core/ipv4/ip4_frag.o
                0x6003eb6c                ip_reass_tmr
 .text.ip_reass_free_complete_datagram
                0x6003ebc4      0x120 ./lwip/src/core/ipv4/ip4_frag.o
 .text.ip_reass_remove_oldest_datagram
                0x6003ece4       0xc4 ./lwip/src/core/ipv4/ip4_frag.o
 .text.ip_reass_enqueue_new_datagram
                0x6003eda8       0x74 ./lwip/src/core/ipv4/ip4_frag.o
 .text.ip_reass_dequeue_datagram
                0x6003ee1c       0x4c ./lwip/src/core/ipv4/ip4_frag.o
 .text.ip_reass_chain_frag_into_datagram_and_validate
                0x6003ee68      0x2a4 ./lwip/src/core/ipv4/ip4_frag.o
 .text.ip4_reass
                0x6003f10c      0x31c ./lwip/src/core/ipv4/ip4_frag.o
                0x6003f10c                ip4_reass
 .text.ip_frag_free_pbuf_custom_ref
                0x6003f428       0x28 ./lwip/src/core/ipv4/ip4_frag.o
 .text.ipfrag_free_pbuf_custom
                0x6003f450       0x50 ./lwip/src/core/ipv4/ip4_frag.o
 .text.ip4_frag
                0x6003f4a0      0x284 ./lwip/src/core/ipv4/ip4_frag.o
                0x6003f4a0                ip4_frag
 .text.dns_lookup
                0x6003f724       0x84 ./lwip/src/core/dns.o
 .text.dns_compare_name
                0x6003f7a8      0x11c ./lwip/src/core/dns.o
 .text.dns_send
                0x6003f8c4      0x1d0 ./lwip/src/core/dns.o
 .text.dns_alloc_random_port
                0x6003fa94       0x78 ./lwip/src/core/dns.o
 .text.dns_alloc_pcb
                0x6003fb0c       0xa4 ./lwip/src/core/dns.o
 .text.dns_call_found
                0x6003fbb0      0x180 ./lwip/src/core/dns.o
 .text.dns_create_txid
                0x6003fd30       0x60 ./lwip/src/core/dns.o
 .text.dns_backupserver_available
                0x6003fd90       0x40 ./lwip/src/core/dns.o
 .text.dns_check_entry
                0x6003fdd0      0x188 ./lwip/src/core/dns.o
 .text.dns_correct_response
                0x6003ff58       0x6c ./lwip/src/core/dns.o
 .text.dns_recv
                0x6003ffc4      0x2a0 ./lwip/src/core/dns.o
 .text.dns_enqueue
                0x60040264      0x26c ./lwip/src/core/dns.o
 .text.dns_gethostbyname_addrtype
                0x600404d0       0x88 ./lwip/src/core/dns.o
                0x600404d0                dns_gethostbyname_addrtype
 .text.ptr_to_mem
                0x60040558       0x24 ./lwip/src/core/mem.o
 .text.mem_to_ptr
                0x6004057c       0x24 ./lwip/src/core/mem.o
 .text.plug_holes
                0x600405a0      0x11c ./lwip/src/core/mem.o
 .text.mem_init
                0x600406bc       0x94 ./lwip/src/core/mem.o
                0x600406bc                mem_init
 .text.mem_link_valid
                0x60040750       0x78 ./lwip/src/core/mem.o
 .text.mem_free
                0x600407c8      0x14c ./lwip/src/core/mem.o
                0x600407c8                mem_free
 .text.mem_trim
                0x60040914      0x200 ./lwip/src/core/mem.o
                0x60040914                mem_trim
 .text.mem_malloc
                0x60040b14      0x1f4 ./lwip/src/core/mem.o
                0x60040b14                mem_malloc
 .text.memp_init
                0x60040d08       0x34 ./lwip/src/core/memp.o
                0x60040d08                memp_init
 .text.do_memp_malloc_pool
                0x60040d3c       0x70 ./lwip/src/core/memp.o
 .text.memp_malloc
                0x60040dac       0x48 ./lwip/src/core/memp.o
                0x60040dac                memp_malloc
 .text.do_memp_free_pool
                0x60040df4       0x48 ./lwip/src/core/memp.o
 .text.memp_free
                0x60040e3c       0x4c ./lwip/src/core/memp.o
                0x60040e3c                memp_free
 .text.netif_add
                0x60040e88      0x180 ./lwip/src/core/netif.o
                0x60040e88                netif_add
 .text.netif_do_set_ipaddr
                0x60041008       0x7c ./lwip/src/core/netif.o
 .text.netif_set_addr
                0x60041084       0x94 ./lwip/src/core/netif.o
                0x60041084                netif_set_addr
 .text.netif_set_default
                0x60041118       0x20 ./lwip/src/core/netif.o
                0x60041118                netif_set_default
 .text.netif_set_up
                0x60041138       0x54 ./lwip/src/core/netif.o
                0x60041138                netif_set_up
 .text.netif_issue_reports
                0x6004118c       0x70 ./lwip/src/core/netif.o
 .text.netif_get_by_index
                0x600411fc       0x4c ./lwip/src/core/netif.o
                0x600411fc                netif_get_by_index
 .text.netif_find
                0x60041248       0x70 ./lwip/src/core/netif.o
                0x60041248                netif_find
 .text.pbuf_alloc
                0x600412b8      0x1bc ./lwip/src/core/pbuf.o
                0x600412b8                pbuf_alloc
 .text.pbuf_alloc_reference
                0x60041474       0x84 ./lwip/src/core/pbuf.o
                0x60041474                pbuf_alloc_reference
 .text.pbuf_alloced_custom
                0x600414f8       0x80 ./lwip/src/core/pbuf.o
                0x600414f8                pbuf_alloced_custom
 .text.pbuf_realloc
                0x60041578       0xf0 ./lwip/src/core/pbuf.o
                0x60041578                pbuf_realloc
 .text.pbuf_add_header_impl
                0x60041668       0xc0 ./lwip/src/core/pbuf.o
 .text.pbuf_remove_header
                0x60041728       0x94 ./lwip/src/core/pbuf.o
                0x60041728                pbuf_remove_header
 .text.pbuf_free
                0x600417bc      0x108 ./lwip/src/core/pbuf.o
                0x600417bc                pbuf_free
 .text.pbuf_ref
                0x600418c4       0x40 ./lwip/src/core/pbuf.o
                0x600418c4                pbuf_ref
 .text.pbuf_cat
                0x60041904       0x94 ./lwip/src/core/pbuf.o
                0x60041904                pbuf_cat
 .text.pbuf_copy
                0x60041998      0x188 ./lwip/src/core/pbuf.o
                0x60041998                pbuf_copy
 .text.pbuf_copy_partial
                0x60041b20       0xdc ./lwip/src/core/pbuf.o
                0x60041b20                pbuf_copy_partial
 .text.pbuf_take
                0x60041bfc      0x10c ./lwip/src/core/pbuf.o
                0x60041bfc                pbuf_take
 .text.pbuf_take_at
                0x60041d08       0xc4 ./lwip/src/core/pbuf.o
                0x60041d08                pbuf_take_at
 .text.pbuf_clone
                0x60041dcc       0x54 ./lwip/src/core/pbuf.o
                0x60041dcc                pbuf_clone
 .text.tcp_init
                0x60041e20       0x24 ./lwip/src/core/tcp.o
                0x60041e20                tcp_init
 .text.tcp_free
                0x60041e44       0x2c ./lwip/src/core/tcp.o
                0x60041e44                tcp_free
 .text.tcp_free_listen
                0x60041e70       0x2c ./lwip/src/core/tcp.o
 .text.tcp_tmr  0x60041e9c       0x2c ./lwip/src/core/tcp.o
                0x60041e9c                tcp_tmr
 .text.tcp_remove_listener
                0x60041ec8       0x44 ./lwip/src/core/tcp.o
 .text.tcp_listen_closed
                0x60041f0c       0x5c ./lwip/src/core/tcp.o
 .text.tcp_close_shutdown
                0x60041f68      0x1a8 ./lwip/src/core/tcp.o
 .text.tcp_close_shutdown_fin
                0x60042110       0xbc ./lwip/src/core/tcp.o
 .text.tcp_close
                0x600421cc       0x5c ./lwip/src/core/tcp.o
                0x600421cc                tcp_close
 .text.tcp_shutdown
                0x60042228       0xb0 ./lwip/src/core/tcp.o
                0x60042228                tcp_shutdown
 .text.tcp_abandon
                0x600422d8      0x15c ./lwip/src/core/tcp.o
                0x600422d8                tcp_abandon
 .text.tcp_bind
                0x60042434      0x150 ./lwip/src/core/tcp.o
                0x60042434                tcp_bind
 .text.tcp_accept_null
                0x60042584       0x30 ./lwip/src/core/tcp.o
 .text.tcp_listen_with_backlog_and_err
                0x600425b4      0x18c ./lwip/src/core/tcp.o
                0x600425b4                tcp_listen_with_backlog_and_err
 .text.tcp_update_rcv_ann_wnd
                0x60042740       0x9c ./lwip/src/core/tcp.o
                0x60042740                tcp_update_rcv_ann_wnd
 .text.tcp_recved
                0x600427dc       0x94 ./lwip/src/core/tcp.o
                0x600427dc                tcp_recved
 .text.tcp_new_port
                0x60042870       0x8c ./lwip/src/core/tcp.o
 .text.tcp_slowtmr
                0x600428fc      0x5f0 ./lwip/src/core/tcp.o
                0x600428fc                tcp_slowtmr
 .text.tcp_fasttmr
                0x60042eec       0xc8 ./lwip/src/core/tcp.o
                0x60042eec                tcp_fasttmr
 .text.tcp_process_refused_data
                0x60042fb4       0xf4 ./lwip/src/core/tcp.o
                0x60042fb4                tcp_process_refused_data
 .text.tcp_recv_null
                0x600430a8       0x64 ./lwip/src/core/tcp.o
                0x600430a8                tcp_recv_null
 .text.tcp_kill_prio
                0x6004310c       0x9c ./lwip/src/core/tcp.o
 .text.tcp_kill_state
                0x600431a8       0x84 ./lwip/src/core/tcp.o
 .text.tcp_kill_timewait
                0x6004322c       0x60 ./lwip/src/core/tcp.o
 .text.tcp_handle_closepend
                0x6004328c       0x4c ./lwip/src/core/tcp.o
 .text.tcp_alloc
                0x600432d8      0x108 ./lwip/src/core/tcp.o
                0x600432d8                tcp_alloc
 .text.tcp_recv
                0x600433e0       0x34 ./lwip/src/core/tcp.o
                0x600433e0                tcp_recv
 .text.tcp_sent
                0x60043414       0x30 ./lwip/src/core/tcp.o
                0x60043414                tcp_sent
 .text.tcp_err  0x60043444       0x34 ./lwip/src/core/tcp.o
                0x60043444                tcp_err
 .text.tcp_poll
                0x60043478       0x50 ./lwip/src/core/tcp.o
                0x60043478                tcp_poll
 .text.tcp_pcb_purge
                0x600434c8       0x8c ./lwip/src/core/tcp.o
                0x600434c8                tcp_pcb_purge
 .text.tcp_pcb_remove
                0x60043554       0xf8 ./lwip/src/core/tcp.o
                0x60043554                tcp_pcb_remove
 .text.tcp_next_iss
                0x6004364c       0x3c ./lwip/src/core/tcp.o
                0x6004364c                tcp_next_iss
 .text.tcp_eff_send_mss_netif
                0x60043688       0x64 ./lwip/src/core/tcp.o
                0x60043688                tcp_eff_send_mss_netif
 .text.tcp_netif_ip_addr_changed_pcblist
                0x600436ec       0x54 ./lwip/src/core/tcp.o
 .text.tcp_netif_ip_addr_changed
                0x60043740       0x7c ./lwip/src/core/tcp.o
                0x60043740                tcp_netif_ip_addr_changed
 .text.tcp_pcbs_sane
                0x600437bc       0x88 ./lwip/src/core/tcp.o
                0x600437bc                tcp_pcbs_sane
 .text.tcp_input
                0x60043844      0x850 ./lwip/src/core/tcp_in.o
                0x60043844                tcp_input
 .text.tcp_input_delayed_close
                0x60044094       0x70 ./lwip/src/core/tcp_in.o
 .text.tcp_listen_input
                0x60044104      0x1ec ./lwip/src/core/tcp_in.o
 .text.tcp_timewait_input
                0x600442f0       0xe8 ./lwip/src/core/tcp_in.o
 .text.tcp_process
                0x600443d8      0x7a8 ./lwip/src/core/tcp_in.o
 .text.tcp_free_acked_segments
                0x60044b80       0xe0 ./lwip/src/core/tcp_in.o
 .text.tcp_receive
                0x60044c60      0x878 ./lwip/src/core/tcp_in.o
 .text.tcp_get_next_optbyte
                0x600454d8       0x6c ./lwip/src/core/tcp_in.o
 .text.tcp_parseopt
                0x60045544       0xd4 ./lwip/src/core/tcp_in.o
 .text.tcp_trigger_input_pcb_close
                0x60045618       0x20 ./lwip/src/core/tcp_in.o
                0x60045618                tcp_trigger_input_pcb_close
 .text.tcp_create_segment
                0x60045638      0x14c ./lwip/src/core/tcp_out.o
 .text.tcp_pbuf_prealloc
                0x60045784       0xd8 ./lwip/src/core/tcp_out.o
 .text.tcp_write_checks
                0x6004585c      0x11c ./lwip/src/core/tcp_out.o
 .text.tcp_write
                0x60045978      0x748 ./lwip/src/core/tcp_out.o
                0x60045978                tcp_write
 .text.tcp_split_unsent_seg
                0x600460c0      0x29c ./lwip/src/core/tcp_out.o
                0x600460c0                tcp_split_unsent_seg
 .text.tcp_send_fin
                0x6004635c       0x90 ./lwip/src/core/tcp_out.o
                0x6004635c                tcp_send_fin
 .text.tcp_enqueue_flags
                0x600463ec      0x1a4 ./lwip/src/core/tcp_out.o
                0x600463ec                tcp_enqueue_flags
 .text.tcp_output
                0x60046590      0x3cc ./lwip/src/core/tcp_out.o
                0x60046590                tcp_output
 .text.tcp_output_segment_busy
                0x6004695c       0x30 ./lwip/src/core/tcp_out.o
 .text.tcp_output_segment
                0x6004698c      0x1cc ./lwip/src/core/tcp_out.o
 .text.tcp_rexmit_rto_prepare
                0x60046b58       0xe4 ./lwip/src/core/tcp_out.o
                0x60046b58                tcp_rexmit_rto_prepare
 .text.tcp_rexmit_rto_commit
                0x60046c3c       0x40 ./lwip/src/core/tcp_out.o
                0x60046c3c                tcp_rexmit_rto_commit
 .text.tcp_rexmit_rto
                0x60046c7c       0x34 ./lwip/src/core/tcp_out.o
                0x60046c7c                tcp_rexmit_rto
 .text.tcp_rexmit
                0x60046cb0       0xc8 ./lwip/src/core/tcp_out.o
                0x60046cb0                tcp_rexmit
 .text.tcp_rexmit_fast
                0x60046d78       0xb4 ./lwip/src/core/tcp_out.o
                0x60046d78                tcp_rexmit_fast
 .text.tcp_output_alloc_header_common
                0x60046e2c       0xd4 ./lwip/src/core/tcp_out.o
 .text.tcp_output_alloc_header
                0x60046f00       0x6c ./lwip/src/core/tcp_out.o
 .text.tcp_output_fill_options
                0x60046f6c       0x68 ./lwip/src/core/tcp_out.o
 .text.tcp_output_control_segment
                0x60046fd4       0xa4 ./lwip/src/core/tcp_out.o
 .text.tcp_rst  0x60047078       0x8c ./lwip/src/core/tcp_out.o
                0x60047078                tcp_rst
 .text.tcp_send_empty_ack
                0x60047104       0xb4 ./lwip/src/core/tcp_out.o
                0x60047104                tcp_send_empty_ack
 .text.tcp_keepalive
                0x600471b8       0x70 ./lwip/src/core/tcp_out.o
                0x600471b8                tcp_keepalive
 .text.tcp_zero_window_probe
                0x60047228      0x144 ./lwip/src/core/tcp_out.o
                0x60047228                tcp_zero_window_probe
 .text.tcpip_tcp_timer
                0x6004736c       0x4c ./lwip/src/core/timeouts.o
 .text.tcp_timer_needed
                0x600473b8       0x48 ./lwip/src/core/timeouts.o
                0x600473b8                tcp_timer_needed
 .text.sys_timeout_abs
                0x60047400       0xd8 ./lwip/src/core/timeouts.o
 .text.lwip_cyclic_timer
                0x600474d8       0x6c ./lwip/src/core/timeouts.o
 .text.sys_timeouts_init
                0x60047544       0x54 ./lwip/src/core/timeouts.o
                0x60047544                sys_timeouts_init
 .text.sys_timeout_debug
                0x60047598       0x40 ./lwip/src/core/timeouts.o
                0x60047598                sys_timeout_debug
 .text.sys_check_timeouts
                0x600475d8       0x74 ./lwip/src/core/timeouts.o
                0x600475d8                sys_check_timeouts
 .text.sys_timeouts_sleeptime
                0x6004764c       0x60 ./lwip/src/core/timeouts.o
                0x6004764c                sys_timeouts_sleeptime
 .text.udp_init
                0x600476ac       0x24 ./lwip/src/core/udp.o
                0x600476ac                udp_init
 .text.udp_new_port
                0x600476d0       0x70 ./lwip/src/core/udp.o
 .text.udp_input_local_match
                0x60047740       0xb4 ./lwip/src/core/udp.o
 .text.udp_input
                0x600477f4      0x270 ./lwip/src/core/udp.o
                0x600477f4                udp_input
 .text.udp_send
                0x60047a64       0x60 ./lwip/src/core/udp.o
                0x60047a64                udp_send
 .text.udp_sendto
                0x60047ac4      0x114 ./lwip/src/core/udp.o
                0x60047ac4                udp_sendto
 .text.udp_sendto_if
                0x60047bd8       0xdc ./lwip/src/core/udp.o
                0x60047bd8                udp_sendto_if
 .text.udp_sendto_if_src
                0x60047cb4      0x208 ./lwip/src/core/udp.o
                0x60047cb4                udp_sendto_if_src
 .text.udp_bind
                0x60047ebc      0x124 ./lwip/src/core/udp.o
                0x60047ebc                udp_bind
 .text.udp_recv
                0x60047fe0       0x3c ./lwip/src/core/udp.o
                0x60047fe0                udp_recv
 .text.udp_remove
                0x6004801c       0x7c ./lwip/src/core/udp.o
                0x6004801c                udp_remove
 .text.udp_netif_ip_addr_changed
                0x60048098       0x60 ./lwip/src/core/udp.o
                0x60048098                udp_netif_ip_addr_changed
 .text.netconn_new_with_proto_and_callback
                0x600480f8       0xbc ./lwip/src/api/api_lib.o
                0x600480f8                netconn_new_with_proto_and_callback
 .text.netconn_prepare_delete
                0x600481b4       0x48 ./lwip/src/api/api_lib.o
                0x600481b4                netconn_prepare_delete
 .text.netconn_getaddr
                0x600481fc       0x9c ./lwip/src/api/api_lib.o
                0x600481fc                netconn_getaddr
 .text.netconn_bind
                0x60048298       0x6c ./lwip/src/api/api_lib.o
                0x60048298                netconn_bind
 .text.netconn_listen_with_backlog
                0x60048304       0x54 ./lwip/src/api/api_lib.o
                0x60048304                netconn_listen_with_backlog
 .text.netconn_accept
                0x60048358      0x11c ./lwip/src/api/api_lib.o
                0x60048358                netconn_accept
 .text.netconn_recv_data
                0x60048474      0x190 ./lwip/src/api/api_lib.o
 .text.netconn_tcp_recvd_msg
                0x60048604       0x5c ./lwip/src/api/api_lib.o
 .text.netconn_tcp_recvd
                0x60048660       0x58 ./lwip/src/api/api_lib.o
                0x60048660                netconn_tcp_recvd
 .text.netconn_recv_tcp_pbuf_flags
                0x600486b8       0x50 ./lwip/src/api/api_lib.o
                0x600486b8                netconn_recv_tcp_pbuf_flags
 .text.netconn_recv_udp_raw_netbuf_flags
                0x60048708       0x50 ./lwip/src/api/api_lib.o
                0x60048708                netconn_recv_udp_raw_netbuf_flags
 .text.netconn_send
                0x60048758       0x54 ./lwip/src/api/api_lib.o
                0x60048758                netconn_send
 .text.netconn_write_vectors_partly
                0x600487ac      0x160 ./lwip/src/api/api_lib.o
                0x600487ac                netconn_write_vectors_partly
 .text.netconn_close_shutdown
                0x6004890c       0x5c ./lwip/src/api/api_lib.o
 .text.netconn_gethostbyname
                0x60048968       0xb0 ./lwip/src/api/api_lib.o
                0x60048968                netconn_gethostbyname
 .text.lwip_netconn_err_to_msg
                0x60048a18       0x58 ./lwip/src/api/api_msg.o
 .text.lwip_netconn_is_err_msg
                0x60048a70       0x68 ./lwip/src/api/api_msg.o
                0x60048a70                lwip_netconn_is_err_msg
 .text.recv_udp
                0x60048ad8       0xd8 ./lwip/src/api/api_msg.o
 .text.recv_tcp
                0x60048bb0       0xdc ./lwip/src/api/api_msg.o
 .text.poll_tcp
                0x60048c8c       0xc0 ./lwip/src/api/api_msg.o
 .text.sent_tcp
                0x60048d4c       0xa0 ./lwip/src/api/api_msg.o
 .text.err_tcp  0x60048dec      0x178 ./lwip/src/api/api_msg.o
 .text.setup_tcp
                0x60048f64       0x50 ./lwip/src/api/api_msg.o
 .text.accept_function
                0x60048fb4      0x15c ./lwip/src/api/api_msg.o
 .text.pcb_new  0x60049110       0xc4 ./lwip/src/api/api_msg.o
 .text.netconn_alloc
                0x600491d4       0xd0 ./lwip/src/api/api_msg.o
                0x600491d4                netconn_alloc
 .text.netconn_free
                0x600492a4       0x60 ./lwip/src/api/api_msg.o
                0x600492a4                netconn_free
 .text.lwip_netconn_do_close_internal
                0x60049304      0x28c ./lwip/src/api/api_msg.o
 .text.lwip_netconn_do_delconn
                0x60049590      0x190 ./lwip/src/api/api_msg.o
                0x60049590                lwip_netconn_do_delconn
 .text.lwip_netconn_do_listen
                0x60049720      0x11c ./lwip/src/api/api_msg.o
                0x60049720                lwip_netconn_do_listen
 .text.lwip_netconn_do_writemore
                0x6004983c      0x364 ./lwip/src/api/api_msg.o
 .text.lwip_netconn_do_write
                0x60049ba0       0xf0 ./lwip/src/api/api_msg.o
                0x60049ba0                lwip_netconn_do_write
 .text.lwip_netconn_do_getaddr
                0x60049c90       0xfc ./lwip/src/api/api_msg.o
                0x60049c90                lwip_netconn_do_getaddr
 .text.lwip_netconn_do_close
                0x60049d8c       0xf8 ./lwip/src/api/api_msg.o
                0x60049d8c                lwip_netconn_do_close
 .text.lwip_netconn_do_gethostbyname
                0x60049e84       0x7c ./lwip/src/api/api_msg.o
                0x60049e84                lwip_netconn_do_gethostbyname
 .text.err_to_errno
                0x60049f00       0x3c ./lwip/src/api/err.o
                0x60049f00                err_to_errno
 .text.lwip_strerr
                0x60049f3c       0x40 ./lwip/src/api/err.o
                0x60049f3c                lwip_strerr
 .text.netbuf_free
                0x60049f7c       0x4c ./lwip/src/api/netbuf.o
                0x60049f7c                netbuf_free
 .text.netbuf_ref
                0x60049fc8       0x90 ./lwip/src/api/netbuf.o
                0x60049fc8                netbuf_ref
 .text.lwip_getaddrinfo
                0x6004a058      0x1e4 ./lwip/src/api/netdb.o
                0x6004a058                lwip_getaddrinfo
 .text.tryget_socket_unconn_nouse
                0x6004a23c       0x34 ./lwip/src/api/sockets.o
 .text.get_socket
                0x6004a270       0x30 ./lwip/src/api/sockets.o
 .text.alloc_socket
                0x6004a2a0       0xc8 ./lwip/src/api/sockets.o
